:1080000018520020A5E40100BDE40100BFE4010016
:10801000C1E40100C1E40100C1E40100000000006E
:10802000000000000000000000000000C1E40100AA
:10803000C1E4010000000000C1E401003FD30000E2
:10804000C1E40100C1E40100C1E40100C1E4010098
:10805000C1E40100C1E4010043CF0000C1E401001C
:10806000C1E40100C1E40100C1E40100C1E4010078
:10807000C1E40100C1E40100C1E40100C1E4010068
:10808000C1E40100C1E40100C1E40100C1E4010058
:10809000C1E40100C1E40100C1E40100C1E4010048
:1080A000C1E40100C1E40100C1E40100C1E4010038
:1080B000C1E40100C1E40100C1E40100C1E4010028
:1080C000C1E40100C1E40100C1E40100C1E4010018
:1080D000C1E40100C1E40100C1E40100C1E4010008
:1080E000C1E40100C1E4010000000000C1E401009E
:1080F000C1E40100C1E40100C1E40100C1E40100E8
:10810000C1E40100C1E40100C1E40100C1E40100D7
:108110000000000000000000C1E40100C1E4010013
:10812000C1E40100C1E40100C1E40100C1E40100B7
:10813000C1E40100C1E40100C1E40100C1E40100A7
:10814000000000000000000000000000000000002F
:10815000C1E40100C1E40100C1E40100C1E4010087
:10816000000000000000000000000000000000000F
:1081700000000000000000000000000000000000FF
:1081800000000000000000000000000000000000EF
:1081900000000000000000000000000000000000DF
:1081A00000000000000000000000000000000000CF
:1081B000C1E40100C1E40100C1E40100C1E4010027
:1081C000C1E40100C1E40100C1E40100C1E4010017
:1081D000C1E40100C1E40100C1E40100C1E4010007
:1081E000C1E40100C1E40100C1E40100000000009D
:1081F00000000000C1E40100C1E40100C1E401008D
:10820000C1E40100C1E40100000000000000000022
:10821000C1E40100C1E40100C1E40100C1E40100C6
:10822000C1E40100C1E40100C1E40100C1E40100B6
:10823000C1E40100C1E40100C1E40100C1E40100A6
:10824000C1E40100C1E40100C1E40100C1E4010096
:10825000C1E40100C1E40100C1E40100C1E4010086
:10826000C1E40100C1E40100C1E4010078B5C9B076
:108270000400DFF8A006002101F079FE1622DFF8E5
:10828000981601A802F04AFFDFF86C3BDFF86C2B70
:10829000162107A803F09DF8DFF8643BDFF8642B94
:1082A00016210DF1320003F094F8DFF85C3BDFF8A3
:1082B0005C2B162112A803F08CF8DFF8543BDFF892
:1082C000542B16210DF15E0003F083F8DFF8483BD4
:1082D000DFF8482B16211DA803F07BF8DFF8403BA0
:1082E000DFF8402B16210DF18A0003F072F8DFF859
:1082F000383BDFF8382B162128A803F06AF8DFF89E
:10830000303BDFF8302B16210DF1B60003F061F899
:10831000DFF8245BDFF8240B00902B00DFF8202B24
:10832000162133A803F055F8DFF8180B00902B0046
:10833000DFF8142B16210DF1E20003F04AF8DFF804
:108340000C3BDFF80C2B16213EA803F042F8DFF8B7
:10835000043BDFF8042B16210DF5877003F039F884
:108360000C2003F0C1F8032003F0D9FB042003F034
:108370002EFC002003F0E7F8401C03F0D4FB01A919
:10838000002003F001FC022003F0DDF805001626B2
:1083900007A806FB05F10144012003F0F5FB07A83F
:1083A00006FB05F1084410F11601022003F0ECFB76
:1083B00007A806FB05F1084410F12C01032003F087
:1083C000E3FB07A87543284410F14201042003F0A1
:1083D000DBFB012003F0B0FA002802D003F045F9DE
:1083E0007DE0082003F0A8FA002875D0012003F0F2
:1083F000AAF8002814D1002004F094FA10F001002B
:108400002063206B002802D00120206301E00020BF
:108410002063206BE0630121312003F0CEF85EE0A1
:10842000012806D101202063206B08284DD20025A9
:1084300044E0022802D102202063F5E7032802D19C
:1084400003202063F0E7042802D104202063EBE737
:10845000052802D105202063E6E7062802D1062080
:108460002063E1E7072802D100202063DCE7082829
:1084700002D108202063D7E7092802D10920206310
:10848000D2E70A2802D107202063CDE70121362058
:1084900003F093F8002406E0200004F043FADFF82C
:1084A000BC190855641C202CF6D318E02900206B59
:1084B00004F048FADFF8541D48556D1C202DF5D303
:1084C0000121322003F079F809E001F080FA01215E
:1084D000322003F072F802E00C2003F0DEF84AB01C
:1084E00070BD70B58EB00400DFF82804002101F0E3
:1084F0003EFD1622DFF8001908A802F00FFE206BDF
:10850000002806D11622DFF8B01B02A802F006FEF2
:1085100005E01622DFF8A41B02A802F0FFFD0420EC
:1085200003F0FDFA042003F052FB002003F0FBFAF5
:1085300008A9002003F028FB02A9012003F024FB76
:108540002CA63100022003F01FFB3100032003F0B2
:108550001BFB3100042003F017FB3100052003F062
:1085600013FB3100062003F00FFB3100072003F05E
:108570000BFB3100082003F007FB082003F0DCF9B7
:10858000002822D0206BE16B884213D0002004F039
:10859000C9F90500206B00280AD0572004F0FDF926
:1085A000022802D30020206322E055F0010501E0FB
:1085B0006D086D002900002004F0AFF90020402173
:1085C00001F0D5FC03F051F812E0012003F0B4F9FA
:1085D000002802D003F049F80AE0002001900120B1
:1085E0000090012300220121206B03F0C9F82063D1
:1085F0000EB070BD0000000070B5A8B004000320EC
:1086000003F08DFAC348002101F0B1FC206B012872
:1086100006D11622DFF8E81701A802F07FFD5FE01F
:10862000206B022806D11622DFF8DC1701A802F021
:1086300075FD55E0206B032806D11622DFF8D01710
:1086400001A802F06BFD4BE0206B042806D1162236
:10865000DFF8C41701A802F061FD41E0206B052896
:1086600006D11622DFF8B81701A802F057FD37E04F
:10867000206B062806D11622DFF8AC1701A802F0FD
:108680004DFD2DE0206B072806D11622DFF8BC1720
:1086900001A802F043FD23E0206B08280BD1DFF88E
:1086A0009C070090DFF89037DFF8642B162101A8B3
:1086B00002F08FFE14E0206B09280BD1DFF884074D
:1086C0000090DFF87437DFF8482B162101A802F07C
:1086D00080FE05E01622DFF8581701A802F01EFD03
:1086E00001A9002003F050FA206B082880F0918047
:1086F0000021206B04F026F9002808D1DFF8143B94
:10870000DFF8142B162107A802F063FE07E0DFF85C
:10871000043BDFF8082B162107A802F05AFE0521BA
:10872000206B04F00FF9002809D1DFF8E83ADFF8F0
:108730002C2C16210DF1320002F04BFE08E0DFF880
:10874000D43ADFF81C2C16210DF1320002F041FE64
:108750000A21206B04F0F6F8002808D1DFF8B43ABB
:10876000DFF8002C162112A802F033FE07E0DFF834
:10877000A43ADFF8F42B162112A802F02AFE0F21EA
:10878000206B04F0DFF8002809D1DFF8883ADFF821
:10879000DC2B16210DF15E0002F01BFE08E0DFF875
:1087A000743ADFF8CC2B16210DF15E0002F011FEB9
:1087B0001421206B04F0C6F8002808D1DFF8543AE1
:1087C000DFF8B02B16211DA802F003FE07E0DFF84A
:1087D000443ADFF8A42B16211DA802F0FAFD192156
:1087E000206B04F0AFF8002809D1DFF8283ADFF851
:1087F0008C2B16210DF18A0002F0EBFD38E0DFF83A
:10880000143ADFF87C2B16210DF18A0002F0E1FD0D
:108810002EE0DFF8005A2B00DFF8682B162107A89E
:1088200002F0D7FD2B00DFF8602B16210DF132008E
:1088300002F0CFFD2B00DFF86C2C162112A802F0FD
:10884000C8FD2B00DFF8602C16210DF15E0002F050
:10885000C0FD2B00DFF8542C16211DA802F0B9FD35
:108860002B00DFF84C2C16210DF18A0002F0B1FD2F
:10887000062002F039FE022002F065FE05001626F1
:1088800007A806FB05F10144012003F07DF907A8C4
:1088900006FB05F1084410F11601022003F074F9FB
:1088A00007A806FB05F1084410F12C01032003F092
:1088B0006BF907A87543284410F14201042003F026
:1088C00063F9002002F03FFE401C03F02CF9042065
:1088D00003F07DF9082003F02FF800280CD00120C8
:1088E00002F031FE60630121342002F066FE0020B8
:1088F000DFF8C01B08600AE0012003F01DF8002823
:1089000002D002F0B2FE02E0062002F0C6FE28B05D
:1089100070BD000000F10F00E0D203002DE9F0412E
:10892000BAB00400DFF8900B002101F020FB606B6F
:10893000401C0090DFF8DC38DFF8802B162108A8F7
:1089400002F047FDDFF8C458616B0520414305EB99
:1089500001004078182817DA616B0520414305EBC8
:10896000010080783C280FDA616B0520414305EB5C
:108970000100C078182807DA616B0520414305EB38
:10898000010000793C281BDB616B0520414305EBAE
:10899000010000214170616B0520414305EB01009E
:1089A00000218170616B0520414305EB010000212E
:1089B000C170616B0520414305EB0100002101718D
:1089C0000623162202A9DFF8FC0A02F07BFF17A794
:1089D00002AB3A0016210EA802F0FBFCDFF8E86AB1
:1089E000616B0520414305EB0100437832001621FD
:1089F0000DF14E0002F0EDFC0FF234084246162154
:108A000019A802F0E6FC616B0520414305EB01006B
:108A10008378320016210DF17A0002F0DAFC062389
:108A2000162202A9DFF8A40A04E000BF25730000A3
:108A30003A00000002F046FF02AB3A00162124A8DB
:108A400002F0C7FC616B0520414305EB0100C378D0
:108A5000320016210DF1A60002F0BBFC42461621A1
:108A60002FA802F0B6FC616B0520414305EB010025
:108A70000379320016210DF1D20002F0AAFC042085
:108A800003F04DF8042003F0A2F8DFF8286A3068FC
:108A9000400003F048F808A9002003F075F80EA97B
:108AA000012003F071F80DF14E01022003F06CF883
:108AB00019A9032003F068F80DF17A01042003F0EE
:108AC00063F824A9052003F05FF80DF1A601062044
:108AD00003F05AF82FA9072003F056F80DF1D20140
:108AE000082003F051F8306800280DD1022002F070
:108AF0001EFF002804D1042002F019FF002803D033
:108B00003068401C306074E1012002F015FF00283D
:108B10000FD0206B082809D2002605E03100206B19
:108B200003F010FFA855761C202EF7D302F09DFD10
:108B30005FE1082002F000FF002800F0C9803068E3
:108B4000042870D1606B00F04BFF002804D1022193
:108B5000392002F032FD4CE1206B08285ED200265D
:108B600000E0761C202E06D23100206B03F0EAFED6
:108B7000A95D8842F5D0202E4DD2002605E0AA5DE1
:108B80003100206B03F0D5FE761C202EF7D3206B2E
:108B9000002805D100205FF0807101F0E8F93AE08B
:108BA000206B012805D100205FF0007101F0DFF992
:108BB00031E0206B022805D100205FF0806101F0D8
:108BC000D6F928E0206B032805D100205FF0006172
:108BD00001F0CDF91FE0206B042805D100205FF0E3
:108BE000805101F0C4F916E0206B052805D1002062
:108BF0005FF0005101F0BBF90DE0206B062805D1B4
:108C000000205FF0804101F0B2F904E000205FF045
:108C1000004101F0ACF902F028FDEAE00221352024
:108C200002F0CBFCE5E0306802284DD1616B0520F5
:108C3000414305EB01008378616B0520414305EB5F
:108C400001004278616B0520414305EB0100017989
:108C5000676B0520474305EB0700C07800F09AFFDB
:108C6000012831D0616B0520414305EB0100837879
:108C7000616B0520414305EB01004278616B0520E3
:108C8000414305EB01000179676B0520474305EB84
:108C90000700C07800F08CFF012815D0616B05201B
:108CA00041432944626B0520424305EB02004078B2
:108CB000C870616B052041432944626B0520424323
:108CC00005EB0200807808713068401C306090E04D
:108CD0003068012815D10120019001200090012366
:108CE00000221721666B0520464305EB06004078FD
:108CF00002F046FD626B05214A4305EB0201487014
:108D000077E03068022815D1012001900120009001
:108D1000012300223B21666B0520464305EB06003C
:108D2000807802F02DFD626B05214A4305EB0201BC
:108D300088705EE0306803281AD10120019001207C
:108D400000900123616B0520414305EB010042784F
:108D50001721666B0520464305EB0600C07802F03C
:108D60000FFD626B05214A4305EB0201C87040E02C
:108D7000306804283DD1616B0520414305EB0100BB
:108D8000C178626B0520424305EB020040788142C6
:108D90001AD101200190012000900123616B052070
:108DA000414305EB010082783B21666B0520464379
:108DB00005EB0600007902F0E3FC626B05214A43F3
:108DC00005EB0201087114E00120019001200090E0
:108DD000012300223B21666B0520464305EB06007C
:108DE000007902F0CDFC626B05214A4305EB0201DC
:108DF00008713AB0BDE8F081A0F10300E0EE010097
:108E000020EF0300E8EE010040EF0300F0EE010068
:108E100060EF0300F8EE010080EF030000EF0100B7
:108E2000A0EF030008EF0100C0EF030010EF010006
:108E3000E0EF030018EF010000EB0300C0EB0300BC
:108E400018EA010080EB030024EA010000F00300AF
:108E500020EF010020F0030028EF0100481000205F
:108E6000F0B593B00400DFF85006002101F07FF860
:108E7000606B401C0090DFF89C33DFF84026162121
:108E800002A802F0A6FADFF88453616B0520414383
:108E90006E5C0096DFF8FC3BDFF8FC2B162108A87F
:108EA00002F097FA0DF136013000C0B203F00CFD6C
:108EB000042002F034FE042002F089FE002002F0BB
:108EC00032FE02A9002002F05FFE08A9012002F094
:108ED0005BFE0DF13601052002F056FE75A7390044
:108EE000022002F051FE3900032002F04DFE39004D
:108EF000042002F049FE3900062002F045FE390048
:108F0000072002F041FE3900082002F03DFE01205A
:108F100002F012FD00280FD0206B082809D200268D
:108F200005E03100206B03F00DFDA855761C202EC6
:108F3000F7D302F09AFBBBE0082002F0FDFC00280A
:108F400000F08380616B05204143685C002804D0F9
:108F50000221332002F031FBAAE0206B082871D2F5
:108F6000616B05204143206B03F0ECFC002869D0C5
:108F7000616B0520414305EB010000214170616BED
:108F80000520414305EB010000218170616B052044
:108F9000414305EB01000021C170616B0520414395
:108FA00005EB010000210171002605E0AA5D3100FA
:108FB000206B03F0BEFC761C202EF7D3206B00281C
:108FC00005D100205FF0807100F0D1FF3AE0206B06
:108FD000012805D100205FF0007100F0C8FF31E0EA
:108FE000206B022805D100205FF0806100F0BFFFF8
:108FF00028E0206B032805D100205FF0006100F01D
:10900000B6FF1FE0206B042805D100205FF08051DF
:1090100000F0ADFF16E0206B052805D100205FF0C1
:10902000005100F0A4FF0DE0206B062805D10020C0
:109030005FF0804100F09BFF04E000205FF0004102
:1090400000F095FF02F011FB32E003F058FD01281B
:1090500001D1062100E00E210020019001200090A6
:1090600001230022300002F08BFB060003F04FFDCD
:1090700001280FD003F083FD012815D10AE000205C
:10908000019001200090012300220E21300002F007
:1090900077FB0600032EF2D0062EF0D0042EEED081
:1090A000082EECD00A2EEAD0616B052041436E54A5
:1090B00013B0F0BD0000000080E60300E0D903001B
:1090C000F8B592B004004FF48070002100F04FFF1B
:1090D000206B082814D1DFF8705ADFF8706A009608
:1090E0002B004B4A16210CA802F073F900962B00B6
:1090F000DFF85C2A16210DF11A0002F06AF913E07C
:10910000DFF8506ADFF8405A00962B00404A1621DB
:109110000CA802F05EF900962B00DFF8342A162125
:109120000DF11A0002F055F91622DFF82C1A01A8E9
:1091300001F0F4FF042002F0F2FC032002F047FDEE
:10914000002002F0F0FC0CA9002002F01DFD01A996
:10915000012002F019FD0DF11A01052002F014FDA5
:109160007DA52900022002F00FFD2900032002F056
:109170000BFD2900042002F007FD2900062002F063
:1091800003FD2900072002F0FFFC2900082002F05F
:10919000FBFC012002F0D0FB002802D002F065FAAF
:1091A00031E0082002F0C8FB00282CD0206B0828F2
:1091B00002D10627002601E00527012610E0C44958
:1091C000626B052000FB02528A5C616B052000FB8C
:1091D0000151300003F0ADFB6D1C052DEFD3761C63
:1091E000B74201D30025F8E700205FF0785100F086
:1091F000BEFE206B082804D100205FF0824100F001
:10920000B6FE02F032FA13B0F0BD000028100020C4
:1092100030EF0100C0DD030030EA01003CEA01004C
:1092200078B5A7B004001622DFF83019684601F0BF
:1092300075FFDFF82C592B00524A162106A802F0C0
:10924000C8F82B00504A16210DF12E0002F0C1F88B
:109250002B00944A162111A802F0BBF82B00924A69
:1092600016210DF15A0002F0B4F82B008F4A162196
:109270001CA802F0AEF82B008D4A16210DF18600D5
:1092800002F0A7F8062002F02FF9032002F047FCB5
:10929000042002F09CFC6946002002F075FC0020CE
:1092A00002F051F9401C02F03EFC022002F04BF9A2
:1092B0000500162606A806FB05F10144012002F070
:1092C00063FC06A806FB05F1084410F11601022014
:1092D00002F05AFC06A806FB05F1084410F12C0127
:1092E000032002F051FC06A87543284410F1420106
:1092F000042002F049FC082002F01EFB00281DD0CB
:10930000012002F020F9062801D2606302E001206A
:1093100003F0C8FCDFF84C0801780222606B824041
:10932000114202D00120206301E000202063206B65
:10933000E0630121372002F040F90AE0012002F049
:10934000FBFA002802D002F090F902E0062002F0B9
:10935000A4F928B070BD00000000000048EA010038
:1093600054EA010060EA01006CEA010078EA0100B9
:1093700084EA010090EA01009CEA0100A8EA0100E9
:10938000B4EA010038EF010040EF010038B58EB0BB
:109390000400606B401C0090DFF8C437474A162178
:1093A00008A802F016F8206B002806D11622DFF874
:1093B000B81702A801F0B2FE05E01622DFF8AC17DC
:1093C00002A801F0ABFE042002F0A9FB042002F089
:1093D000FEFB002002F0A7FB08A9002002F0D4FB4E
:1093E00002A9012002F0D0FB35A52900022002F0DD
:1093F000CBFB2900032002F0C7FB2900042002F068
:10940000C3FB2900052002F0BFFB2900062002F063
:10941000BBFB2900072002F0B7FB2900082002F05F
:10942000B3FB012002F088FA002802D002F01DF9F7
:1094300035E0082002F080FA002825D0206BE16B8F
:10944000884219D0002003F06DFA0100206B00283B
:1094500004D00222606B8240114303E00222606B61
:1094600082409143DFF8FC060170002003F055FABA
:109470000020402100F07BFD0221382002F09DF801
:1094800000200C4908600AE00020019001200090B3
:10949000012300220121206B02F072F920630FB03A
:1094A00030BD000048EF010050EF010058EF01000F
:1094B00060EF01007C11002000F10F0068EF010057
:1094C0000000000000EE030070EF010020EE03003A
:1094D000281000202DE9F041BAB00400DFF8900612
:1094E000002100F044FD606B401C0090DFF87036F6
:1094F000DFF88026162108A801F06BFFDFF864561C
:10950000606B05EB80000079202811DA606B05EBB9
:10951000800040790D280BDA606B05EB80008079C4
:10952000202805DA606B05EB8000C0790D2813DB7D
:10953000606B05EB800000210171606B05EB800022
:1095400000214171606B05EB800000218171606B2F
:1095500005EB80000021C1710623162202A9DFF865
:10956000180602F0AFF915A602AB320016210EA8BC
:1095700001F02FFFDFF80476606B05EB80000379C4
:109580003A0016210DF14E0001F023FF0FF23008D2
:109590004246162119A801F01CFF606B05EB800004
:1095A00043793A0016210DF17A0001F012FF0623EB
:1095B000162202A9DFF8C80504E000BF25730000E9
:1095C0002F00000002F07EF902AB3200162124A821
:1095D00001F0FFFE606B05EB800083793A001621F5
:1095E0000DF1A60001F0F5FE424616212FA801F06C
:1095F000F0FE606B05EB8000C3793A0016210DF197
:10960000D20001F0E6FE042002F089FA042002F004
:10961000DEFADFF870653068400002F084FA08A9CD
:10962000002002F0B1FA0EA9012002F0ADFA0DF10E
:109630004E01022002F0A8FA19A9032002F0A4FAB0
:109640000DF17A01042002F09FFA24A9052002F00E
:109650009BFA0DF1A601062002F096FA2FA9072029
:1096600002F092FA0DF1D201082002F08DFA306872
:1096700000280DD1022002F05AF9002804D104205C
:1096800002F055F9002803D03068401C30603EE1FC
:10969000012002F051F900280BD0002404E0200042
:1096A00003F040F92855641C202CF8D301F0DDFFAD
:1096B0002DE1082002F040F9002800F0A580306874
:1096C000002802D101F0D1FF21E13068012802D049
:1096D0003068032803D13068401C306017E13068DF
:1096E000022837D1606B05EB8000407902280AD14F
:1096F000606B05EB800000791E2880F208813068DD
:10970000401C306003E1606B05EB80004079042869
:1097100011D0606B05EB8000407906280BD0606BA0
:1097200005EB80004079092805D0606B05EB8000CF
:1097300040790B280AD1606B05EB800000791F2867
:1097400080F2E5803068401C3060E0E03068401C0A
:109750003060DCE0606B05EB8000C079022809D145
:10976000606B05EB800080791E2828DA3068401C89
:10977000306024E0606B05EB8000C079042811D0D4
:10978000606B05EB8000C07906280BD0606B05EBA1
:109790008000C079092805D0606B05EB8000C07996
:1097A0000B2809D1606B05EB800080791F2806DA51
:1097B0003068401C306002E03068401C3060306827
:1097C0000528C0F0A4800020306000F067F9002474
:1097D00000E0641C202C05D2200003F0A3F8295DD2
:1097E0008142F6D0202C0CD0002404E0295D20001A
:1097F00003F093F8641C202CF8D30020402100F0E3
:10980000B6FB01F032FF82E0306801281DD1606BA9
:1098100005EB80000079002805D1606B05EB800026
:109820000121017173E001200190012000900123CA
:1098300001221F21606B05EB8000007901F0A0FF81
:10984000616B05EB8101087161E0306802281DD170
:10985000606B05EB80004079002805D1606B05EB5B
:1098600080000121417152E001200190012000900F
:10987000012301220C21606B05EB8000407901F08F
:109880007FFF616B05EB8101487140E03068032880
:109890001DD1606B05EB80008079002805D1606BDD
:1098A00005EB80000121817131E001200190012050
:1098B0000090012301221F21606B05EB800080795D
:1098C00001F05EFF616B05EB810188711FE030687C
:1098D00004281CD1606B05EB8000C079002805D1FD
:1098E000606B05EB80000121C17110E00120019047
:1098F00001200090012301220C21606B05EB800008
:10990000C07901F03DFF616B05EB8101C8713AB090
:10991000BDE8F08118B58DB0040001F0B7FE322823
:1099200009D1606B401C0090974B924A162107A802
:1099300001F04FFD0EE0362809D1606B401C00900D
:10994000874B8C4A162107A801F043FD02E0012055
:1099500003F0A8F98D4B7AA2162101A801F039FD78
:10996000042002F0DCF8012002F031F9002002F0BE
:10997000DAF807A9002002F007F901A9012002F096
:1099800003F970A42100022002F0FEF82100032058
:1099900002F0FAF82100042002F0F6F82100052078
:1099A00002F0F2F82100062002F0EEF82100072074
:1099B00002F0EAF82100082002F0E6F8082001F0A1
:1099C000BBFF002801D001F050FE0EB010BD0020FA
:1099D00003E000216E4A1154401C2028F9D370473F
:1099E00070B5040001266A4D052000FB04F0285CD8
:1099F00000284DD0052000FB04F028448378052082
:109A000000FB04F028444278052000FB04F02844C1
:109A10000179052000FB04F02844C07800F0BAF872
:109A2000012835D0052000FB04F028448378052068
:109A300000FB04F028444278052000FB04F0284491
:109A40000179052000FB04F02844C07800F0B0F84C
:109A500001281DD00020052101FB04F168540020DD
:109A6000052101FB04F1294448700020052101FB78
:109A700004F1294488700020052101FB04F12944E8
:109A8000C87000210520444305EB04000171002645
:109A9000300070BD40D8030078EF010038B50024D5
:109AA0004AE0304D05EB8400007900282ED005EB0C
:109AB00084004079002829D005EB840080790028B3
:109AC00024D005EB8400C07900281FD005EB84006A
:109AD000037905EB8400427905EB8400817905EB7D
:109AE0008400C07900F056F8012824D005EB8400EA
:109AF000037905EB8400427905EB8400817905EB5D
:109B00008400C07900F054F8012814D0002005EB3F
:109B100084010871002005EB84014871002005EBE9
:109B200084018871002005EB8401C8712878022126
:109B3000A14088432870641C062CB2D331BD0000BC
:109B4000257300000000000000EB0300C0EB0300E1
:109B5000C0EA010080EB030040F0030020F00300A6
:109B6000C0ED03004810002080E60300E0D90300A8
:109B700000F10F0068EF010000EE030070EF01003C
:109B800020EE03007C110020C0DD0300C0F10300C3
:109B900028100020824201D2012008E0904205D125
:109BA0008B4201D2012002E0002000E0002070473B
:109BB000904203D1994201D1012000E0002070477A
:109BC00001200021DFF8742BC2E900010020DFF83A
:109BD000701B0860704738B503F0F7F8002840F0B4
:109BE000B881DFF85C0B0068012805D101F044FA68
:109BF000DFF8482BC2E90001DFF8400BD0E9002371
:109C000001240025AB4204D1A24202D100F0BEF9EA
:109C1000A9E1D0E90023002B04D1022A02D100F0EF
:109C20006DFAA0E1D0E90023B3F5807F05D1002AC9
:109C300003D1012000F002FB95E1D0E90023B3F548
:109C4000007F05D1002A03D1022000F0F7FA8AE153
:109C5000D0E9002300240125AB4204D1A24202D165
:109C600000F0A5FA7FE1D0E90023002B04D1042AFB
:109C700002D100F04FFB76E1D0E90023002B04D1A4
:109C8000082A02D100F093FB6DE1D0E90023002BFC
:109C900005D1B2F5807F02D100F068FC63E1D0E924
:109CA0000023802B04D1002A02D100F00DFC5AE1E0
:109CB000D0E90023002B05D1102A03D1012000F0A8
:109CC000A1FC50E1D0E90023022B05D1002A03D1E9
:109CD000012000F037FD46E1D0E90023002B05D13B
:109CE000202A03D1022000F08DFC3CE1D0E90023C2
:109CF000042B05D1002A03D1022000F023FD32E11C
:109D0000D0E90023002B05D1402A03D1032000F025
:109D100079FC28E1D0E90023082B05D1002A03D1E2
:109D2000032000F00FFD1EE1D0E90023002B05D138
:109D3000B2F5800F02D100F06CFD14E1D0E90023F0
:109D4000002B06D1B2F5801F03D1012000F015FED3
:109D500009E1D0E90023002B06D1B2F5001F03D1A1
:109D6000022000F00AFEFEE0D0E90023B3F5806F88
:109D700004D1002A02D100F055FEF4E0D0E900231E
:109D8000202B04D1002A02D100F08DFEEBE0D0E9B7
:109D9000002300245FF08075AB4205D1A24203D1BD
:109DA000002000F019FFDEE0D0E9002300245FF07E
:109DB0000075AB4205D1A24203D1012000F00CFF97
:109DC000D1E0D0E9002300245FF08065AB4205D1EB
:109DD000A24203D1022000F0FFFEC4E0D0E900233C
:109DE00000245FF00065AB4205D1A24203D10320FD
:109DF00000F0F2FEB7E0D0E9002300245FF08055C8
:109E0000AB4205D1A24203D1042000F0E5FEAAE056
:109E1000D0E9002300245FF00055AB4205D1A242F7
:109E200003D1052000F0D8FE9DE0D0E900230024F6
:109E30005FF08045AB4205D1A24203D1062000F07D
:109E4000CBFE90E0D0E9002300245FF00045AB4258
:109E500005D1A24203D1072000F0BEFE83E0D0E985
:109E60000023002B06D1B2F5805F03D1002000F063
:109E70001EFF78E0D0E90023002B06D1B2F5005F89
:109E800003D1012000F013FF6DE0D0E90023002B87
:109E900006D1B2F5804F03D1022000F008FF62E046
:109EA000D0E90023002B06D1B2F5004F03D10320E7
:109EB00000F0FDFE57E0D0E90023002B06D1B2F5FB
:109EC000803F03D1042000F0F2FE4CE0D0E90023F3
:109ED000002B06D1B2F5003F03D1052000F0E7FECC
:109EE00041E0D0E90023002B06D1B2F5802F03D149
:109EF000062000F0DCFE36E0D0E90023002B06D17E
:109F0000B2F5002F03D1072000F0D1FE2BE0D0E9FD
:109F10000023402B04D1002A02D100F013FE22E0DE
:109F2000D0E90023002B05D1B2F5007F02D100F06B
:109F300053FF18E0D0E90023002B05D1B2F5006FE4
:109F400002D100F00AFF0EE001220023C0E9002345
:109F500009E003F047F9DFF8E41B0968401A6528B7
:109F600001D303F048F9082003F03FF931BD30B4C4
:109F7000DFF8CC2BD2E9004520432943C2E9000198
:109F800030BC7047DFF8401C0860704770B5DFF8E0
:109F90003C0C0068002851D1DFF8344C2920207097
:109FA000002060708820A0705320E0704420207151
:109FB0004B2060714520A0715620E0714F20207227
:109FC000002060720020A0720020E0720020207348
:109FD000002060730020A0730020E0730020207434
:109FE0000E2003F0DFF860740F2003F0DBF8A0749C
:109FF000FF20E074207560758420A0757B20E075DB
:10A00000002004E0002104EB00021176401C13281C
:10A01000F8D3042002F04BFE002806D1332084F848
:10A020002200342084F8230005E0302084F8220048
:10A03000302084F8230000F045FF5EE0DFF8944B09
:10A04000200002F002FF012855D16078BB2802D120
:10A0500003F0D1F851E0A078882849D1A07DE17DB6
:10A0600071F0FF01C94388423FD102F000FD0A268A
:10A0700094F8220003F092F90500754394F8230048
:10A0800003F08CF955FA80F002F008FD607C03F0D3
:10A0900085F905007543A07C03F080F955FA80F03E
:10A0A00002F0FFFC02F02BFD002803D102F005FDB9
:10A0B000202807D302F023FD012813D102F0FDFC74
:10A0C0001E280FD294F82700000694F8281010EBF1
:10A0D000014094F8291010EB012094F82A10401840
:10A0E00003F007FC00F0DDFE07E000F0DAFE04E01C
:10A0F00000F0B2FE01E000F0BEFE70BD38B5DFF842
:10A10000CC0A006800280CD1DFF8C40A05210170D0
:10A11000002141702F21817000F0EAFE00F0D2FE94
:10A1200044E0DFF8B04A200002F08FFE01283BD166
:10A130006078BB2802D100F0D5FF37E0A078A128D5
:10A1400028D1DFF8FC59D5E9000110F0000011F426
:10A15000807100220023994207D1904205D1A37952
:10A1600062792179E07803F04DFCD5E9000110F027
:10A17000000011F4007100220023994207D190429F
:10A1800005D1A37A627A217AE07903F04EFC00F0DF
:10A1900088FE0BE0F92804D100F083FE00F0A2FF56
:10A1A00004E000F059FE01E000F065FE31BD10B59D
:10A1B000DFF8180A0068002813D1DFF8144A0720D6
:10A1C0002070002060705220A07000F091FE7F206F
:10A1D00003F0A0FCE071E079C043207200F072FE51
:10A1E0002BE0DFF8F049200002F02FFE012822D1F9
:10A1F0006078BB2802D100F075FF1EE0A0788628A9
:10A2000004D100F0A5FE00F04CFE16E0F02808D1C5
:10A21000E078522802D100F044FE0EE000F01CFE6F
:10A220000BE0F92804D100F03CFE00F05BFF04E0F5
:10A2300000F012FE01E000F01EFE10BD38B5040073
:10A24000DFF888090068002835D1DFF884590A2032
:10A250002870002068708720A870012C14D100F0AD
:10A2600064FE0120E871002003F001FC2872012047
:10A2700003F0FDFB6872022003F0F9FBA8720320D3
:10A2800003F0F5FBE87213E000F03CFE0220E871F9
:10A29000002003F0FAFB2872012003F0F6FB68723D
:10A2A000022003F0F2FBA872032003F0EEFBE87239
:10A2B00000F008FE2DE0DFF81C59280002F0C5FD73
:10A2C000012824D16878BB2802D100F00BFF20E0E0
:10A2D000A878F02811D1E87887280BD1012C02D179
:10A2E00003F098FB03E0022C01D103F0AEFB00F079
:10A2F000D8FD0EE000F0B0FD0BE0F92804D100F02D
:10A30000D0FD00F0EFFE04E000F0A6FD01E000F05B
:10A31000B2FD31BD10B5DFF8B4080068002824D1C3
:10A32000DFF8AC480E202070002060700620A0707E
:10A3300000F0DEFD0020E0715FF0FF3002F0B7FCBE
:10A340000100090E21720100090C61720100090A65
:10A35000A172E07200202073002060730020A073BF
:10A360000020E07300F0AEFD20E0DFF86848200038
:10A3700002F06BFD012817D16078BB2802D100F0F4
:10A38000B1FE13E0A078862804D100F0E1FD00F0D2
:10A3900088FD0BE0F92804D100F083FD00F0A2FE57
:10A3A00004E000F059FD01E000F065FD10BD10B5BE
:10A3B000DFF818080068002824D1DFF814480E20C0
:10A3C0002070002060700720A07000F091FD002038
:10A3D000E0715FF0FF3002F06AFC0100090E2172AB
:10A3E0000100090C61720100090AA172E0720020EB
:10A3F0002073002060730020A0730020E07300F041
:10A4000061FD60E0DFF8CC47200002F01EFD01286E
:10A4100057D16078BB2802D100F064FE53E0A078E9
:10A42000772844D1E078217910EB012003F022FC59
:10A430006079A17910EB012003F02BFC607AA17AFE
:10A4400010EB012003F02BFC607BA17B10EB0120C3
:10A4500003F019FCE07B217C10EB012003F025FCCC
:10A46000E07D00F0FF00217E10EB012003F005FCF1
:10A4700002F045FB002803D102F01FFB202807D281
:10A4800002F03DFB01280FD102F017FB1E280BD371
:10A49000E07E0006217F50EA0140617F50EA012002
:10A4A000A17F084303F025FA00F0FBFC0BE0F9283C
:10A4B00004D100F0F6FC00F015FE04E000F0CCFC46
:10A4C00001E000F0D8FC10BD10B5DFF8000700680F
:10A4D000002823D1DFF8F8460D202070002060709E
:10A4E0008520A07000F004FD03F0F3FB0100090ECD
:10A4F000E1710100090C21720100090A6172A07268
:10A50000C0430100090EE1720100090C2173010032
:10A51000090A6173A07300F0D5FC26E0DFF8B446A9
:10A52000200002F092FC01281DD16078BB2802D1E6
:10A5300000F0D8FD19E0A078F0280AD1E07885284D
:10A5400004D103F0C9FB00F0ACFC0EE000F084FC89
:10A550000BE0F92804D100F0A4FC00F0C3FD04E0F6
:10A5600000F07AFC01E000F086FC10BD38B5DFF8A1
:10A570005C06006800280CD1DFF854060521017044
:10A58000002141700D21817000F0B2FC00F09AFCB6
:10A5900037E0DFF84046200002F057FC01282ED1BA
:10A5A0006078BB2802D100F09DFD2AE0A0789D28AC
:10A5B0001BD1DFF88C05D0E9000110F0000011F08C
:10A5C00040010022002399420CD190420AD100257B
:10A5D00006E004EB0500C178280002F09EF96D1C2E
:10A5E0001F2DF6D300F05DFC0BE0F92804D100F03C
:10A5F00058FC00F077FD04E000F02EFC01E000F0D4
:10A600003AFC31BD38B50400DFF8C0050068002809
:10A6100016D1DFF8BC050521017000214170012C25
:10A6200002D10121817006E0022C02D10221817049
:10A6300001E00321817000F05BFC00F043FC7BE053
:10A64000DFF89055280002F000FC012872D16878EC
:10A65000BB2802D100F046FD6EE0A87883281ED109
:10A66000032C1CD1DFF8D804D0E9000110F0000061
:10A6700011F008010022002399420DD190420BD124
:10A68000002407E005EB0400C17814F1400002F05B
:10A6900099F9641C1F2CF5D300F003FC4CE08228D0
:10A6A0001ED1022C1CD1DFF89804D0E9000110F073
:10A6B000000011F004010022002399420DD19042C4
:10A6C0000BD1002407E005EB0400C17814F1200051
:10A6D00002F078F9641C1F2CF5D300F0E2FB2BE0AC
:10A6E00081281DD1012C1BD1DFF85404D0E90001D1
:10A6F00010F0000011F002010022002399420CD159
:10A7000090420AD1002406E005EB0400C178200045
:10A7100002F058F9641C1F2CF6D300F0C2FB0BE0CA
:10A72000F92804D100F0BDFB00F0DCFC04E000F0EF
:10A7300093FB01E000F09FFB31BD0000C81000203A
:10A740002811002070B50400DFF88004006800289C
:10A750002AD1DFF87C542420287000206870012C56
:10A7600002D18120A87006E0022C02D18220A870BC
:10A7700001E08320A87000F0D8FB012C01D1002457
:10A7800004E0022C01D1202400E04024002606E051
:10A79000301902F014F905EB0601C871761C1F2E62
:10A7A000F6D300F08FFB33E0DFF82854280002F0E6
:10A7B0004CFB01282AD16878BB2802D100F092FC1A
:10A7C00026E0A878E978F02816D1012C03D10800FA
:10A7D000C0B281280AD0022C03D10800C0B282285E
:10A7E00004D0032C05D1C9B2832902D100F059FB52
:10A7F0000EE000F031FB0BE0F92804D100F051FB32
:10A8000000F070FC04E000F027FB01E000F033FBF7
:10A8100070BD38B5DFF8B403006800280ED1DFF84A
:10A82000B00302210170002141700B218170DFF81B
:10A8300098130968C17000F045FB9DE0DFF8944370
:10A84000200002F002FB012840F094806078BB28D1
:10A8500002D100F047FC8FE0A0788B2840F0808088
:10A86000DFF86453E0782968884276D12179286836
:10A8700003F08AFB6179A07951EA0021E07951EA7D
:10A880000041207A51EA0061286803F008FB627AEF
:10A890000023A07A0021090241EA1061000202436C
:10A8A0000B43E07A0021090441EA1041000402430D
:10A8B0000B43207B0021090641EA102100060243D8
:10A8C0000B43607C00210100002002430B43A07C6D
:10A8D00000210102002002430B43E07C002101041F
:10A8E000002002430B43207D00210106002002438B
:10A8F0000B43286803F0EDFA617BA07B51EA00214D
:10A90000E07B51EA0041207C51EA0061286803F0B5
:10A91000F5FA8B48D0E9000110F0000011F48061D5
:10A9200000220023994209D1904207D1617D286815
:10A9300003F048FBA17D286803F0EEFAE27D0021D8
:10A94000286803F00BFB227E0121286803F006FB38
:10A950000020286000F0A5FA0EE000F07DFA0BE080
:10A96000F92804D100F09DFA00F0BCFB04E000F0EF
:10A9700073FA01E000F07FFA31BD70B5040093482E
:10A98000006800280AD1924802210170002141701C
:10A990000C218170C47000F095FA42E08D4D2800C2
:10A9A00002F053FA01283AD16878BB2802D100F0AE
:10A9B00099FB36E0A978E8788C2926D1A04224D1E9
:10A9C0002879697910EB012003F039FAA879E9793F
:10A9D00010EB012003F030FA287A697A10EB01209D
:10A9E00003F030FA00260BE003F0ECFA07E0B01CAD
:10A9F00005EB0601897A012CF6D103F0C5FA761C25
:10AA00000E2EF4D300F04DFA0BE0F92904D100F03A
:10AA100048FA00F067FB04E000F01EFA01E000F0E5
:10AA20002AFA70BD38B569480068002816D1684C0C
:10AA300007202070002060708A20A070624D286876
:10AA4000E070286803F0A8FA20710020607128687F
:10AA500003F059FAA07100F035FA23E05D4C2000B4
:10AA600002F0F3F901281BD16078BB2802D100F075
:10AA700039FB17E0A078E178F02807D18A2902D1C4
:10AA800000F00FFA0EE000F0E7F90BE0F92804D12E
:10AA900000F007FA00F026FB04E000F0DDF901E029
:10AAA00000F0E9F931BD10B54848006800281FD111
:10AAB000474C0B202070002060708F20A07000F0A9
:10AAC00017FA002003F0A0FAE071012003F09CFACD
:10AAD0002072022003F098FA6072042003F094FAC6
:10AAE000E072052003F090FA207300F0EBF924E007
:10AAF000384C200002F0A9F901281CD16078BB284D
:10AB000002D100F0EFFA18E0A078E178F02808D13F
:10AB1000C9B28F2902D100F0C4F90EE000F09CF90F
:10AB20000BE0F92804D100F0BCF900F0DBFA04E0F6
:10AB300000F092F901E000F09EF910BD3011002004
:10AB4000D010002038B521480068002816D1204DCB
:10AB500025202870002068709D20A87000F0E5F97D
:10AB6000002406E0200001F0DDFE05EB0401C871C1
:10AB7000641C202CF6D300F0A5F924E0154C20002D
:10AB800002F063F901281CD16078BB2802D100F0E3
:10AB9000A9FA18E0A078E178F02808D1C9B29D2977
:10ABA00002D100F07EF90EE000F056F90BE0F92832
:10ABB00004D100F076F900F095FA04E000F04CF9C9
:10ABC00001E000F058F931BD3C1100202C110020AB
:10ABD000200E0020A00D002070B50400DFF818053D
:10ABE000006800283DD1DFF8145526202870002089
:10ABF00068709020A87000F098F9012C02D1012013
:10AC0000E8711FE0022C02D10220E8711AE0032C47
:10AC100002D10320E87115E0042C02D10420E87170
:10AC200010E0052C02D10520E8710BE0062C02D1C2
:10AC30000620E87106E0072C02D10720E87101E048
:10AC40000020E871002607E03100200001F07AFEC4
:10AC500005EB06010872761C1F2EF5D300F032F9C1
:10AC600024E0DFF89C54280002F0EFF801281BD103
:10AC70006878BB2802D100F035FA17E0AA78E878A6
:10AC80002979F02A06D1902804D1A14202D100F0FE
:10AC900008F90BE0F92804D100F003F900F022FADA
:10ACA00004E000F0D9F801E000F0E5F870BD70B5FF
:10ACB0000400DFF84404006800280DD1DFF83C549C
:10ACC00006202870002068701020A87000F010F98D
:10ACD000EC7100F0F7F83FE0DFF82454280002F0B0
:10ACE000B4F8012836D16878BB2802D100F0FAF90F
:10ACF00032E0A878902823D100205FF080712200F4
:10AD000003F0EAF9DFF8FC23D2E9002310401940F0
:10AD100000220023994210D190420ED1E87884425B
:10AD20000BD1002607E005EB060002793100200078
:10AD300001F0FFFD761C202EF5D300F0B2F80BE0F9
:10AD4000F92804D100F0ADF800F0CCF904E000F0EF
:10AD500083F801E000F08FF870BD10B5DFF89803BC
:10AD6000006800280CD1DFF8940305210170002150
:10AD700041700E21817000F0BBF800F0A3F82AE0CA
:10AD8000DFF87C43200002F060F8012821D16078D0
:10AD9000BB2802D100F0A6F91DE0A07891280ED1C1
:10ADA0002079617950EA0120A17950EA0140E179E6
:10ADB00050EA016003F0C1F900F073F80BE0F928E4
:10ADC00004D100F06EF800F08DF904E000F044F8D2
:10ADD00001E000F050F810BD38B5C7480068002801
:10ADE0000BD1C64805210170002141700F218170EF
:10ADF00000F07EF800F066F82DE0C14D280002F06A
:10AE000024F8012825D16878BB2802D100F06AF91E
:10AE100021E0A878782812D1E87801F045FE287959
:10AE200002F0BCFA04000A204443687902F0B6FA42
:10AE300054FA80F001F03BFE00F033F80BE0F92803
:10AE400004D100F02EF800F04DF904E000F004F811
:10AE500001E000F010F831BD80B5AB480168491C35
:10AE600001600021A44A116000680B2802D3102061
:10AE700001F018FF01BD80B502F0B4F9A3490968DB
:10AE8000401A65280CD300209B490860A04801683F
:10AE9000491C016000680A2802D3102001F002FF5B
:10AEA00001BD80B5002098490860002098490860DD
:10AEB000002091490860102001F0EEFE0120954924
:10AEC000086001BD38B58D4801F082FF01208A4934
:10AED000086002F087F98D4908608A48D0E90023AC
:10AEE0008D49D1E90045A243AB43C0E9002331BD00
:10AEF00082483321C17031210171302141713121EA
:10AF00008171704710B57D4C002002F0B7FDE070F4
:10AF1000012002F0B3FD2071022002F0AFFD60714C
:10AF2000032002F0ABFDA07110BD10B5734C0020E2
:10AF300002F096FDE070012002F092FD20710220E7
:10AF400002F08EFD6071032002F08AFDA07110BD39
:10AF500038B56B4CE0780006217910EB014061793F
:10AF600010EB0120A179401803F0E4F8E07903F038
:10AF7000A1F9627A00231B0643EA12231206A07A83
:10AF80000021090441EA1041000402430B43E07A26
:10AF90000021090241EA1061000202430B43207BB9
:10AFA000002102430B43607B002101020020024389
:10AFB0000B43A07B0021010000201043194303F044
:10AFC000D9F8E07C0006217D10EB0140617D10EB9B
:10AFD0000120A17D401803F069F9E07D0006217E83
:10AFE00010EB0140617E10EB0120A17E401802F0C1
:10AFF0007DFC444DD5E9000110F0000011F0010185
:10B0000000220023994205D1904203D1217FE07EA6
:10B0100002F05DFD607F02F027FE94F8200003F04F
:10B02000B3F8D5E9000110F0000011F02001002272
:10B03000002399421FD190421DD194F82310002083
:10B0400002F0DEFF94F82410012002F0D9FF94F8FA
:10B050002510022002F0D4FF94F82610032002F0FD
:10B06000CFFF94F82710042002F0CAFF94F82810AC
:10B07000052002F0C5FF31BDF0B42748D0E900013A
:10B08000204AD2E9004554F0040455F00005C2E915
:10B090000045002300E05B1C402B1ED200245FF023
:10B0A0000045A94208D801D3A04205D200240025BA
:10B0B000A94204D1A04202D10120002103E04900AD
:10B0C00041EAD0714000D2E9004504400D4000261D
:10B0D0000027BD4201D1B442DDD000220D4B1A60E1
:10B0E000F0BC7047012000210B4AC2E9000100209A
:10B0F00008490860704700002C110020200E002035
:10B10000A00D0020D01000203811002030110020A8
:10B110003411002028110020C810002010B4002491
:10B1200003E00B5D0355641C521E002A02D00B5D28
:10B13000002BF6D1002A04D000210155641C521EB8
:10B14000F8E710BC70472DE9F0470C000021002CF7
:10B1500000D0641E5FF00009804616001F000AE060
:10B1600038683F1D002C04D088F8000018F1010851
:10B17000641E19F101093078002800F019810025BA
:10B1800000E06D1C705D252802D0705D0028F8D1AC
:10B19000AC4207D2220031004046FFF7BFFFA04477
:10B1A000002406E02A0031004046FFF7B7FFA8441C
:10B1B000641B15EB09092E4430782528DBD1761C59
:10B1C000002520220CE016F8010C302802D1002DB9
:10B1D00000D130220A20454316F8010C30384519B9
:10B1E0003000461C0078253800F0BF800B38092855
:10B1F000E9D9283856D00B38B2D0401E0AD0401FAB
:10B2000008D0C01F4ED0C01E0FD0801E44D0C01E1C
:10B2100048D0B6E03B683F1D002B02D55B420120C1
:10B2200000E000205FF00A0C41E039683F1D5FF04C
:10B23000000A01E01AF1010A11F80A000028F9D108
:10B24000AA4503D215EB0909B9EB0A09544506D200
:10B2500022004046FFF762FFA044002418E0524657
:10B260004046FFF75BFFD044B4EB0A04AA450FD277
:10B27000B5EB0A05AC4200D225006C4204E0202068
:10B2800088F8000018F101082800451E0028F6D1B2
:10B290001AEB090AD1466EE73B683F1D5FF00A0CC6
:10B2A000002004E03B683F1D5FF0100C00200121EE
:10B2B00002E00CFB01F16D1E0CFB01FE734505D392
:10B2C0000CFB01FEBEFBFCFE8E45F2D0002800D038
:10B2D0006D1E002810D0002C0ED096465FFA8EFE10
:10B2E000BEF1300F08D12D2088F8000018F10108B8
:10B2F000641E19F101090020B5F1020E4FF6FE7A25
:10B30000D6450DD26D1E09E0002C04D088F800202F
:10B3100018F10108641E19F101096D1E002DF3D109
:10B3200000281FD0002C1DD02D2088F8000018F117
:10B330000108641E19F1010914E0002C0ED0B3FBC2
:10B34000F1F0B0FBFCF20CFB1200DFF8F820126801
:10B35000105C88F8000018F10108641E19F1010959
:10B36000B1FBFCF10029E8D105E7002C06D016F866
:10B37000010C88F8000018F10108641E19F1010998
:10B38000F9E6052C09D30522DFF8BC104046FFF78B
:10B39000C5FE18F10508641F07E02200DFF8A810B9
:10B3A0004046FFF7BBFEA044002419F10509E2E680
:10B3B000002088F800004846BDE8F0870CB480B54E
:10B3C0000A0002AB4FF6FF71FFF7BDFE02BC5DF84D
:10B3D0000CFB08B400B501ABFFF7B5FE5DF808FB48
:10B3E00070B406E0DBB2E4B2A34224D3401C491C93
:10B3F000521E002A22D00378002B02D10B78002B9A
:10B400000CD00378413B1A2B0AD2037820330C78F6
:10B41000413C1A2C06D20C78203404E000200EE0C7
:10B420000378F4E70C7825001E00EDB2F6B2B542C1
:10B43000D8D2012003E05FF0FF3000E0002070BCB4
:10B44000704700007CF0010068F0010010B5DFF8E3
:10B45000F444002060610321002000F0AEF80120D8
:10B46000206010BD80B51F2003F06FF9DFF8D41401
:10B470008A6C42400A650A6D82430A658A6C4240C2
:10B48000CA64CA6C0240CA64886401BD10B5102049
:10B4900003F05BF9002801D0002400E0012403F050
:10B4A00047FE00280BD1DFF89C0400218160012CAD
:10B4B00002D1002141600DE0012141600AE0DFF886
:10B4C000840400214160012C02D10121816001E04E
:10B4D00000218160DFF86C044068012803D103215A
:10B4E000012000F06AF810BD30B4DFF85814DFF81E
:10B4F0005824031F4C6952F82440A34203D2031F6F
:10B500004C6942F82430DFF844244B6952F8233068
:10B51000042B03D303234C6942F82430DFF8303482
:10B520004C6953F82440844203D3441E4D6943F8C8
:10B530002540052805D2486953F82000496942F89A
:10B54000210030BC7047002807D1DFF80004DFF885
:10B55000F413496950F8210010E0012807D1DFF801
:10B56000F003DFF8E013496950F8210006E0DFF846
:10B57000D803DFF8D013496950F82100704700283C
:10B5800007D1DFF8C803DFF8BC23526940F8221066
:10B5900012E0012807D1DFF8B803DFF8A8235269C9
:10B5A00040F8221008E0022806D1DFF89C03DFF8FB
:10B5B0009423526940F82210704738B504000800FF
:10B5C000C0B201280BD1DFF87C034169072903D2FF
:10B5D0004169491C416109E00021416106E0C9B2AD
:10B5E000022903D00020DFF85C134861DFF85453D0
:10B5F000DFF860036969445401F0F4FDA86101F0CB
:10B60000F1FDE8610020DFF840136A6941F822008B
:10B610000020DFF838136A6941F822000020DFF8C3
:10B6200030136A6941F822000020E8622000C0B2AD
:10B63000122819D02000C0B2132815D02000C0B2A3
:10B64000142811D0E4B2152C0ED000200AE03021CD
:10B6500005EB000282F82010302105EB000282F891
:10B660002510401C0528F2D331BDB6494869002891
:10B6700002D04869401E48610020C8627047B54842
:10B68000B0494969405C7047AE487047B148AD4920
:10B690004969084410F8010C704738B504000325C7
:10B6A000641EAC4200D22500042000F040F90028BE
:10B6B00030D00020FFF747FFA84215D30120FFF745
:10B6C00042FFA0425BD20120FFF73DFF0100491C71
:10B6D0000120FFF754FF0220FFF735FF0100491C4E
:10B6E0000220FFF74CFF4AE00120FFF72CFFA042A9
:10B6F00045D20120FFF727FF0100491C0120FFF779
:10B700003EFF0020FFF71FFF0100491C0020FFF74C
:10B7100036FF34E0022000F00AF900282FD0002084
:10B72000FFF711FF002815D00120FFF70CFF0028BC
:10B7300025D00120FFF707FF0100491E0120FFF778
:10B740001EFF0020FFF7FFFE0100491E0020FFF74B
:10B7500016FF14E00120FFF7F6FE00280FD00120AD
:10B76000FFF7F1FE0100491E0120FFF708FF02204C
:10B77000FFF7E9FE0100491E0220FFF700FF31BD7F
:10B780002DE9F84F81460C0015001F000B98C0B240
:10B7900000280DD101F026FD6F49086001F022FD5F
:10B7A0006E4908604FF4FA706D4908606D49086091
:10B7B000022000F0BCF800280AD05FF001084FF426
:10B7C000FA706749086001F00DFD6449086021E0E6
:10B7D000022000F0A7F8002816D001F003FD604E0B
:10B7E000DFF878A1DAF80010401A3168884208D3EF
:10B7F0005FF0010801F0F6FCCAF800009620306006
:10B8000008E05FF0000805E05FF0000801F0EAFCE6
:10B81000524908600A9EB8F1010F0CD1A14505D22A
:10B8200017EB09094C454AD2A14648E0F6B2012E71
:10B8300045D1A94643E0042000F079F800280AD059
:10B840005FF0010B4FF4FA704649086001F0CAFC42
:10B850004149086024E0042000F064F8002819D071
:10B8600001F0C0FCDFF8FC80DFF8ECA0DAF8001093
:10B87000401AD8F80010884209D35FF0010B01F09C
:10B88000B1FCCAF800009620C8F8000008E05FF09C
:10B89000000B05E05FF0000B01F0A4FC2E490860EE
:10B8A000BBF1010F0BD14D4505D2B9EB0709A945F5
:10B8B00005D2A94603E0F6B2012E00D1A1464846C2
:10B8C000BDE8F28F70B404000026002500E0761C6D
:10B8D000A05D0028FBD1D01A864215D2D21A921B45
:10B8E00002E0605D48556D1CB542FAD3002003E0CC
:10B8F00020234B556D1C401C9042F9D30020485525
:10B900000CE0605D48556D1CD01A8542F9D30020CB
:10B910004855202001EB050202F8010C0020887533
:10B9200070BC70470749896CC0B208407047054930
:10B93000C96CC0B2084070470249096DC0B20840E6
:10B9400070470000000F0020C80F0020E80F002003
:10B9500008100020D81000206C1100206811002071
:10B96000701100207411002010B5DFF8384A102142
:10B97000200003F0A1FC10221021200003F08CFC19
:10B98000DFF8504C04222821200003F072FD2068CB
:10B99000002804D02068012801D00020206003F096
:10B9A000F3FD0020DFF8301C087001F01BFC0A38A2
:10B9B000DFF8281C08600120DFF8241C086010BD97
:10B9C00010B5DFF81C0C0068002800F08D8001F035
:10B9D00009FCDFF8084C2168401A0A28C0F0818071
:10B9E00001F000FC20604FF48040002102F0C6FB13
:10B9F00000220023994206D1904204D1DFF8D40BF3
:10BA00000068012830D1012002F09FFE00280ED1ED
:10BA1000022002F09AFE002809D1042002F095FECF
:10BA2000002804D1082002F090FE002804D001F084
:10BA3000D9FBDFF8641C086001F0D4FBDFF8581C68
:10BA40000968401ADFF8541C884206D300221021EE
:10BA5000DFF8500903F020FC11E010221021DFF87C
:10BA6000440903F019FC0AE010221021DFF8340920
:10BA700003F012FC01F0B6FBDFF81C1C0860DFF8D5
:10BA8000201C0868401C086064200A680968B1FB33
:10BA9000F0F100FB1120002801D104F095F8DFF847
:10BAA000380B0178012902D100F03BF919E0017847
:10BAB000022902D100F071FA13E00178032902D1C2
:10BAC00000F08EFB0DE00178042902D100F019FC92
:10BAD00007E00078052802D100F066FC01E000F0E4
:10BAE000B1F8042001F081FB10BDDFF8E80A00681E
:10BAF000704780B5002801D0012806D1DFF8D42A8C
:10BB000010602821106803F015FD01BDDFF8940BCB
:10BB10000068002801D0012000E000207047DFF815
:10BB2000B81A08707047DFF8B01A0A78032A0AD1E9
:10BB3000052803D2DFF8081D086024E00020DFF8A4
:10BB4000001D08601FE00A78042A0AD1092803D2E0
:10BB5000DFF8EC1C086016E00020DFF8E41C086049
:10BB600011E00A78052A03D1DFF8D41C08600AE046
:10BB70000978012903D1DFF8C81C086003E0002020
:10BB8000DFF8BC1C0860704730B400230AE0DFF81F
:10BB9000B44C0500EDB21622554304EB0502CC5C13
:10BBA000D4545B1CCA5C002A01D0152BEFD316219C
:10BBB000DFF8902C0400E4B24C4314440025E55413
:10BBC000C0B2484310440021417530BC704780B575
:10BBD000DFF8741CC0B208600868002805D1DFF8DF
:10BBE0006C0CDFF86C1C08602BE00868012805D19C
:10BBF000DFF8600CDFF8581C086022E008680228B3
:10BC000005D1DFF8540CDFF8481C086019E008681B
:10BC1000032805D1DFF8440CDFF8341C086010E07D
:10BC20000868042805D1DFF8380CDFF8241C086008
:10BC300007E0DFF8180CDFF8181C0860012001F09D
:10BC400031F801BDF0B585B0DFF8184C03F0BEFC4B
:10BC50002060002005E0DFF8101C095C2268115408
:10BC6000401CB0F5806FF6D3DFF8004C25000021B2
:10BC7000686840686A68126A9047686125007FF0CA
:10BC80007F41686840686A68126A904728612500A9
:10BC9000DFF8DC6BA86904F06EFA07005FF0FF3292
:10BCA0003100280004F080F8002101917F08D7F1CD
:10BCB00005070097022190FBF1F3D3F140035FF0F9
:10BCC000FF323100280004F0A2F834200090332322
:10BCD000DFF8A02B0C2102A8FFF77BFB250002AEAA
:10BCE000A86904F048FA07005FF0FF32310028002D
:10BCF00004F05AF8002101917F08D7F13707009727
:10BD0000022190FBF1F3D3F140035FF0FF323100E9
:10BD1000280004F07CF861684868496A884705B0E3
:10BD2000F0BD2DE9FE43DFF83C5B03F04FFC2860DB
:10BD3000002003E000212A681154401CB0F5806FF8
:10BD4000F8D3DFF8284B260000217068406872683D
:10BD5000126A9047706126007FF07F4170684068EA
:10BD60007268126A90473061DFF80C1B200004F003
:10BD70008BFA2700DFF8CC6A16F58478B86904F0EE
:10BD8000FAF981465FF0FF324146380004F00CF8C2
:10BD9000002101915FEA5909D9F10509CDF8009018
:10BDA000022190FBF1F3D3F140035FF0FF324146F3
:10BDB000380004F02CF8DFF8C41A200004F064FA0C
:10BDC000270016F1DC08B86904F0D5F981465FF068
:10BDD000FF324146380003F0E7FF002101915FEA9E
:10BDE0005909D9F11209CDF80090022190FBF1F325
:10BDF000D3F140035FF0FF324146380004F007F80A
:10BE0000270016F1C608B86904F0B5F981465FF05D
:10BE1000FF324146380003F0C7FF002101915FEA7D
:10BE20005909D9F11D09CDF80090022190FBF1F3D9
:10BE3000D3F140035FF0FF324146380003F0E7FFE3
:10BE40002700F236B86904F096F980465FF0FF32B9
:10BE50003100380003F0A8FF002101915FEA580883
:10BE6000D8F13508CDF80080022190FBF1F3D3F131
:10BE700040035FF0FF323100380003F0C8FF0220BA
:10BE800001F048FE00280DD028680290DFF8F00984
:10BE9000019000200090152315222B21002003F093
:10BEA000A1FB0EE0012001F035FE29680291DFF8C8
:10BEB000D01901910090152315222B21002003F0A9
:10BEC00091FB022001F026FE29680291DFF8B419E7
:10BED00001910090152315222B21162003F082FBDF
:10BEE00028680290DFF8A009019000200090152337
:10BEF00015222B21552003F075FB28680290DFF8EE
:10BF00008C09019000200090152315222B216B2015
:10BF100003F068FBDFF828693078C0070CD5286883
:10BF20000290DFF86C09019000200090082307229E
:10BF30000221022003F056FB3078800709D500204B
:10BF400001900D20009003230122A3A1200003F003
:10BF50005EFF307840070DD528680290DFF834097D
:10BF6000019000200090092307220221772003F08E
:10BF700039FB0CE03078000709D500200190022041
:10BF800000907723012295A1200003F040FF616813
:10BF90004868496A8847BDE8F7832DE9F84F84B0BF
:10BFA000DFF8C04803F012FB206000200AE0002107
:10BFB0002268115405E0B0F5807FF8D20121226893
:10BFC0001154401CB0F5806F05D28028F3D2FF21B8
:10BFD00022681154F5E7012001F09CFD00281BD1D7
:10BFE000022001F097FD002816D1202001F092FDDB
:10BFF000002802D0DFF8A05810E0402001F08AFDB0
:10C00000002806D000F07BFD002802D1DFF88C5814
:10C0100004E0DFF88C5801E0DFF88858202001F0B8
:10C0200079FD002829D1012001F074FD002824D1D8
:10C03000022001F06FFD00281FD1102001F06AFDE1
:10C04000002807D0082001F065FD002802D0DFF8A5
:10C05000586814E0102001F05DFD002802D0DFF8E0
:10C060004C680CE0082001F055FD002802D0DFF8F4
:10C07000406804E0DFF83C6801E0DFF8286804204D
:10C0800001F048FD002802D0DFF82C7801E0DFF84D
:10C090002C78DFF8D887C2467FF07F494946DAF826
:10C0A00004004068DAF80420126A9047CAF81400C5
:10C0B000C2460021DAF804004068DAF80420126A67
:10C0C0009047CAF81000CDF80880DFF878A7CDF8BF
:10C0D0000CA00298806904F04EF883465FF0FF32AE
:10C0E0000399029803F060FE002101915FEA5B0B67
:10C0F000DBF1030BCDF800B0022190FBF1F3D3F19B
:10C1000040035FF0FF320399029803F080FE20683D
:10C11000029001950020009015231522142105207E
:10C1200003F060FA20680290019600200090152329
:10C1300015221421242003F055FA2068029001975B
:10C1400000200090152315221421452003F04AFAFF
:10C1500020680290DFF86807019000200090152306
:10C1600015221421652003F03DFA44460021606841
:10C1700040686268126A9047606144464946606858
:10C1800040686268126A9047206144461AF1C60509
:10C19000A06903F0F0FF06005FF0FF3229002000E5
:10C1A00003F002FE002101917608D6F134060096D4
:10C1B000022190FBF1F3D3F140035FF0FF3229003D
:10C1C000200003F024FED8F804104868496A884724
:10C1D00005B0BDE8F08F0000540000002A00000008
:10C1E0002DE9FE4300F0FEF9DFF8804626007FF0DF
:10C1F0007F452900706840687268126A90477061D4
:10C2000026000021706840687268126A90473061A9
:10C210002700DFF83066B046B86903F0ACFF81460E
:10C220005FF0FF324146380003F0BEFD002101916E
:10C230005FEA5909D9F10309CDF80090022190FB7A
:10C24000F1F3D3F140035FF0FF324146380003F0D1
:10C25000DEFD27000021786840687A68126A9047FE
:10C26000786127002900786840687A68126A9047E8
:10C270003861002001900D20009008235FF0FF320C
:10C2800016F11601200003F0C2FD002001901720D6
:10C29000009008235FF0FF3216F12C01200003F01C
:10C2A000B6FD002001902120009008235FF0FF32AE
:10C2B00016F14201200003F0AAFD002001902B207E
:10C2C000009008235FF0FF3216F15801200003F0C0
:10C2D0009EFDDFF86C15086800280CD00020019046
:10C2E00009680A204143C91C009101230122B8A119
:10C2F000200003F08CFD61684868496A8847BDE802
:10C30000F7832DE9FC4100F06DF9DFF86045260068
:10C310007FF07F452900706840687268126A904714
:10C32000706126000021706840687268126A904748
:10C3300030612600DFF80C75B06903F01CFF804601
:10C340005FF0FF323900300003F02EFD0021019133
:10C350005FEA5808D8F10308CDF80080022190FB6D
:10C36000F1F3D3F140035FF0FF323900300003F006
:10C370004EFD26000021706840687268126A90477E
:10C38000706126002900706840687268126A9047E0
:10C39000306100F089F961684868496A8847BDE8FA
:10C3A000F3810000005000402DE9F84F84B002A84E
:10C3B000052103F06BFF00F015F9DFF8B04426000B
:10C3C0007FF07F452900706840687268126A904764
:10C3D000706126000021706840687268126A904798
:10C3E00030612600DFF85C74B06903F0C4FE80465B
:10C3F0005FF0FF323900300003F0D6FC00210191DC
:10C400005FEA5808D8F10308CDF80080022190FBBC
:10C41000F1F3D3F140035FF0FF323900300003F055
:10C42000F6FC00264CE0A146DFF89804052101FB4C
:10C4300006F100EB010AD9F8180003F09CFE8346D0
:10C440005FF0FF325146484603F0AEFC01210191F6
:10C45000B8EB5B08CDF80080022190FBF1F03F1AA9
:10C460003B005FF0FF325146484603F0D0FC26E027
:10C47000062E05D0072E03D0082E01D0092ED2D1CA
:10C48000A1460DF1080AD9F8180003F074FE83469E
:10C490005FF0FF325146484603F086FC01210191CE
:10C4A000B8EB5B08CDF80080022190FBF1F03F1A59
:10C4B0003B005FF0FF325146484603F0A8FC761C73
:10C4C000102E7DD216F0030F01D110270CE016F0CC
:10C4D0000300012801D1302706E016F003000228EE
:10C4E00001D1502700E07027042E02D25FF00F0820
:10C4F0000BE0082E02D25FF0190806E00C2E02D2E3
:10C500005FF0230801E05FF02D08CD480068F0409F
:10C51000C00716D5A1462900D9F804004068D9F80B
:10C520000420126A9047C9F81400A1460021D9F8E6
:10C5300004004068D9F80420126A9047C9F8100036
:10C5400015E0A1460021D9F804004068D9F804207C
:10C55000126A9047C9F81400A1462900D9F80400CE
:10C560004068D9F80420126A9047C9F8100000F01A
:10C57000C6FA01287FF47CAFA146D248052101FB11
:10C5800006F100EB010AD9F8180003F0F4FD834628
:10C590005FF0FF325146484603F006FC012101914D
:10C5A000B8EB5B08CDF80080022190FBF1F03F1A58
:10C5B0003B005FF0FF325146484603F028FC7EE71F
:10C5C00061684868496A884705B0BDE8F08F000097
:10C5D0003E00000010110020101200201411002055
:10C5E000F810002070B59F4C02F0F0FF2060002092
:10C5F0000BE0974B1B680B4493F880302568561866
:10C60000AB55491C8029F4D3401C082842D200288D
:10C6100009D1002200218029F6D2FF23256856186F
:10C62000AB55491CF7E701280BD1802202FB00F231
:10C6300000218029E8D2012325685618AB55491CF2
:10C64000F7E7022805D0032803D0042801D00528E5
:10C650000BD1802202FB00F200218029D4D20023DA
:10C6600025685618AB55491CF7E706280DD18022DE
:10C6700002FB00F200218029C6D2754B1B685B5C6F
:10C6800025685618AB55491CF5E7802202FB00F2DD
:10C690000021B7E770BD00000C110020C1D40100DB
:10C6A00018110020405000402DE9F8438AB00122C3
:10C6B0000EE0491C6348162303FB02F31844405C58
:10C6C0000028F6D102A800EB820040F8041C521C9E
:10C6D000092A01D20021EDE702A9029D4868451907
:10C6E00004984519059845190C6948690419089872
:10C6F00004190998041906267543D5F180056D08BB
:10C7000001274BE0DFF86481C1460021D9F804001D
:10C710004068D9F80420126A9047C9F814007FF0E5
:10C720007F41D8F804004068D8F80420126A904786
:10C73000C8F810001BE042480068B842E2D1DFF8B8
:10C740002C81C1467FF07F41D9F804004068D9F8B8
:10C750000420126A9047C9F814000021D8F8040098
:10C760004068D8F80420126A9047C8F810000120E9
:10C770000190142000902B005FF0FF323148162109
:10C7800001FB07F10144394803F041FB02A800EB2B
:10C79000870050F8040C06FB00557F1C052FCAD3F8
:10C7A0007443D4F180046408052543E02F4FB84654
:10C7B0000021D8F804004068D8F80420126A904795
:10C7C000C8F814007FF07F41786840687A68126A80
:10C7D0009047386117E01A480068A842E6D1234F15
:10C7E000B8467FF07F41D8F804004068D8F80420AC
:10C7F000126A9047C8F814000021786840687A6887
:10C80000126A904738610120019020200090230097
:10C810005FF0FF320B48162101FB05F1014413487C
:10C8200003F0F5FA02A800EB850050F8040C06FBB3
:10C8300000446D1C092DCED30BB0BDE8F083000081
:10C84000041100208009002008110020A8DB01004D
:10C8500000110020A8D90100A8DA0100A8D8010021
:10C86000A8D70100FC100020A0D00100540F002028
:10C8700008EB010008E70100D8CF0100A8DC0100A7
:10C8800040E0010080E0010000E10100C0E00100A3
:10C8900010EB010018E7010040E10100C0E30100D6
:10C8A00080E1010080E20100C0E2010000E201003D
:10C8B00040E20100C0E1010040E3010000E30100AB
:10C8C00080E30100F0DF010010B50C000F281CD23E
:10C8D0000C2807D12248036B224A16212000FEF7BC
:10C8E00078FD19E00D2807D11D48436B1E4A16211B
:10C8F0002000FEF76EFD0FE0194951F8203017A215
:10C9000016212000FEF765FD06E01548036813A216
:10C9100016212000FEF75DFD10BD202801D2134A2C
:10C9200011547047202801D3002001E00F49085C12
:10C930007047202905D2082803D20D4B4001184426
:10C9400042547047202906D2082804D2084A4001E0
:10C950001044405C00E00020704700002573200078
:10C960006402002058F0010060F00100681000200F
:10C97000A00C002000202C49086070472B49496C0E
:10C980000840704729494A6C10434864704727495A
:10C990004A6C32EA0000486470470100C9B2442979
:10C9A00002D12248406C09E00100C9B2402902D1FD
:10C9B0001E48006C02E01D49C0B2085C70471B496C
:10C9C000085C7047602801D2184A1154402802D3ED
:10C9D00001201549086070470200D2B20300DBB2A3
:10C9E000602B1CDA0300DBB2402B02D10F4801643C
:10C9F00015E00300DBB2442B02D10C4841640EE089
:10CA00000300DBB2382B02DBC0B2542805D1074843
:10CA10008154521CC943815401E004488154704739
:10CA20000148006870470000B8110020A00E0020E7
:10CA30008B48002101600068C0438A4908600020DB
:10CA400089490870002089490870002088490870C9
:10CA5000002088490870704781480068814909684A
:10CA6000C943884201D1012000E00020704780B511
:10CA7000042801D0062805D179490860202000F05B
:10CA80000BF905E0002076490860202000F00AF943
:10CA900073480068C0437349086001BD724908705B
:10CAA0007047724908707047714908707047714942
:10CAB000087070476A48006870476B480078704794
:10CAC0006A48007870476B4800787047644801688E
:10CAD000042907D164480078202801DA01200DE0FC
:10CAE00000200BE00068062807D15F4800781E2868
:10CAF00001DA012002E0002000E0012070475848E0
:10CB00000068062801D1012000E00020704780B5B0
:10CB100053480068042806D11E20FFF73EFF07286F
:10CB200001D1012000E0002002BD80B54C48006822
:10CB3000042806D11E20FFF730FF082801D101206C
:10CB400000E0002002BD80B545480068042806D1F9
:10CB50001E20FFF722FF092801D1012000E000205C
:10CB600002BD80B53E480068042806D11E20FFF7AC
:10CB700014FF042801D1012000E0002002BD80B58F
:10CB800037480068042806D11E20FFF706FF0A2850
:10CB900001D1012000E0002002BD80B530480168CD
:10CBA000062901D1002014E00068042810D11E20BD
:10CBB000FFF7F3FE042809D0092807D0082805D07C
:10CBC000072803D00A2801D0012002E0002000E05D
:10CBD000012002BD10B50C001100042805D1264A21
:10CBE0002000FEF7F6FB012035E0062805D1234A98
:10CBF0002000FEF7EEFB01202DE0072805D1204A9A
:10CC00002000FEF7E6FB012025E0092805D11D4A9A
:10CC10002000FEF7DEFB01201DE0082805D11A4A9E
:10CC20002000FEF7D6FB012015E0102806D1174B97
:10CC30000AA22000FEF7CDFB01200CE00A2805D156
:10CC4000134A2000FEF7C5FB012004E0114A200032
:10CC5000FEF7BFFB002010BD0000000025730000A0
:10CC6000D0110020D4110020121200201312002035
:10CC7000141200201512002000F0010008F001003D
:10CC800010F0010018F0010020F0010008E8010098
:10CC900028F0010030F0010017490A6832EA00006C
:10CCA0000860704714490A681043086070471249C9
:10CCB00009680840704710480178C90701D5652008
:10CCC00019E00178890701D5662014E00178090789
:10CCD00001D568200FE00178490701D567200AE0F7
:10CCE0000178C90601D5692005E00078800601D5E4
:10CCF0006A2000E0002070472011002010B5BB48DA
:10CD000003F0EAFABA4803F0E7FA03F065FCB94821
:10CD100003F077FC0121B84802F0CEFA0120B749B0
:10CD20000860B748B7490860FF20B749086080210C
:10CD3000B64802F0C1FA8020B5490860B54802F053
:10CD4000E5FAB54802F0E2FA3021B44802F0D0FA30
:10CD500003F060FBB24C60234FF4614201002000FD
:10CD600003F0EAFC10220221200003F0E1FCAD48B0
:10CD7000016831F0100101601021200003F031FD45
:10CD8000200003F008FD0321200003F038FD1620E9
:10CD900003F0AAFC172003F0A7FCC021162003F023
:10CDA0003CFD162003F04AFD0F21162003F02CFC59
:10CDB0009D49162003F03DFC0F21172003F024FCB1
:10CDC0009A49172003F035FC10BD99480068704758
:10CDD000F8B505000127974E02203070002415E0B9
:10CDE000285DC0B20009C0B200F0EBFA06EB4401C6
:10CDF0004870285D10F00F0000F0E3FA06EB4401E4
:10CE00008870002C01D0285D3F18641C2878801C95
:10CE10008442E5D3FF4307F0FF073800000900F024
:10CE2000D0FA06EB4401487017F00F07380000F005
:10CE3000C8FA06EB44018870032006EB4401C87071
:10CE40006000001D00F0BDF8F1BD2DE9F8430500BC
:10CE5000002000E0401CB0F5807F06DA76490A5CCD
:10CE6000032AF7D1040000220A54B0F5807F01DACA
:10CE7000002C01D1002062E0671E00E07F1E002F21
:10CE80005CD46D4EF05D0228F8D10020F055E41B13
:10CE9000641C083CE00701D5022050E06408201F14
:10CEA000792801D302204AE0781C00F0FF00411CE1
:10CEB00001F0FF01715C305C00F0C2F82870287846
:10CEC000844201D002203AE05FF00108F81C00F033
:10CED000FF00411C01F0FF01715C305C00F0B0F814
:10CEE0006870687818EB00085FF0000917E0781D9B
:10CEF00010EB490000F0FF00411C01F0FF01715CE4
:10CF0000305C00F09DF805EB09018870A14504D262
:10CF100005EB0900807858FA80F819F101094C45B1
:10CF2000E5D27FEA080808F0FF0805EB04008078E6
:10CF3000804501D0022002E0012000E00020BDE891
:10CF4000F28310B5364C0121200003F04FFC0100A4
:10CF5000200003F051FC36480068002807D1162055
:10CF600003F0AEFB002808D100F008F805E03348D4
:10CF70000068800601D500F001F810BD80B50020E2
:10CF80002B49086000201D490860002020490860E6
:10CF9000162003F02EFB002003E00021264A115446
:10CFA000401CB0F5807FF8D34FF480700090224B86
:10CFB0001B4A0121162003F048FB162003F011FB49
:10CFC00001BD80B501211A4A11608021104A11600B
:10CFD00001210A4A11600090114B164A01211720C5
:10CFE00003F033FB172003F0FCFA01BD011800F039
:10CFF000000C00F000080020004002400440024005
:10D000004B434F4C20750040247500400070004099
:10D010000072004002100200021402000060004092
:10D0200000D000402CD000400080000C008000C0E8
:10D0300024110020A00B0020A00A00203CD00040BA
:10D0400038B50C00C0B200F0A9F905002D01200090
:10D05000C0B200F0A3F945192800C0B232BDF0B447
:10D060000246106895681318506803EB5004C00717
:10D070001DD54D441BE013F8017B05F8017B491ECB
:10D08000F9D1A0B1B60813F8011B06F00306032E70
:10D0900008BF13F8016B01EB06214942801C2944AB
:10D0A00005D011F8016B05F8016B401EF9D1A342C0
:10D0B0000ED013F8016B16F0030104BF13F8011B27
:10D0C000C91C30090F28DAD113F8010B0F30D6E74D
:10D0D000F0BC02F10C0070471CB59B4C10221021D3
:10D0E000200002F0C6F92078532826D16078442821
:10D0F00023D1A0784B2820D1E07845281DD1207974
:10D1000056281AD160794F2817D1A079002814D158
:10D11000E079002811D1207A00280ED1607A002809
:10D120000BD1A07A002808D1E07A002805D1207B15
:10D13000002802D1607B002803D00820FFF7B2FD51
:10D1400002E00820FFF7A8FD04220A21684602F049
:10D1500090F90420FFF7ABFD00280DD000208DF8DA
:10D16000000000208DF8010004220A21684602F028
:10D1700095F90028F8D114E09DF80000332803D178
:10D180009DF8010034280CD033208DF800003420A5
:10D190008DF8010004220A21684602F07FF9002878
:10D1A000F8D113BD6849085C704710B504005FF002
:10D1B000804003F015FC012803D15FF0804003F0AC
:10D1C00007FC6248444321005FF0804003F00FFCFD
:10D1D0005FF0804003F0F7FB10BD5D4800685D49DB
:10D1E000086070475A48006870475B490A68C0B2D7
:10D1F00010430860704780B503F008FB0F2003F070
:10D2000049FB162003F046FB544803F074F85448D9
:10D2100003F071F8534803F06EF85348534908601F
:10D22000FBE753480068704780B503F0EFFA4FF40E
:10D2300000405049086003F0E9FB4F4803F07AF8DA
:10D24000012003F073F84D4803F046F84C4803F012
:10D2500043F84C4803F040F84B4803F03DF84B4886
:10D2600003F03AF84A4803F037F84A4803F034F834
:10D2700002F0E2F8002803D001203D49086002E0F6
:10D2800000203B490860314803F0D4FB03F0C6FBA3
:10D2900000210F2003F0C1FA0F2003F0CFFA03F0B2
:10D2A000C3FB03F0AFFA5FF0704003F015F85FF0D6
:10D2B000804003F095FB012803D15FF0804003F02C
:10D2C00087FB35495FF0804003F091FB5FF08040C1
:10D2D00003F073FB5FF0804003F091FB5FF0804050
:10D2E00003F06AFB5FF0804003F06DFB01BD80B589
:10D2F00017480068174908601420FFF756FF002000
:10D300001549086001BD80B5134800681F2802D088
:10D310000120FFF7C7FC0E4801680E480068091A93
:10D320000B2902D30120FFF7BDFC002002F0F2FF21
:10D33000000703D50C480D490860FBE701BD044810
:10D340000168491C01607047B81000208038010056
:10D35000F8110020FC11002000120020050400F04C
:10D36000011800F0000C00F00400FA050CED00E0DC
:10D370000412002008ED00E0800300C1000800F066
:10D38000010800F0020800F0030800F0040800F0B3
:10D39000050800F0005800F000B4C40400210100AA
:10D3A000C9B230390A2902D23038C0B208E00100CF
:10D3B000C9B24139062902D23738C0B200E0002094
:10D3C000704710F00F000149085C7047F8E7010052
:10D3D000002801D120207CE0C10701D5002078E0A1
:10D3E000810701D5012074E0410701D5022070E0DA
:10D3F000010701D503206CE0C10601D5042068E0D7
:10D40000810601D5052064E0410601D5062060E0D3
:10D41000010601D507205CE0C10501D5082058E0D0
:10D42000810501D5092054E0410501D50A2050E0CD
:10D43000010501D50B204CE0C10401D50C2048E0CA
:10D44000810401D50D2044E0410401D50E2040E0C7
:10D45000010401D50F203CE0C10301D5102038E0C4
:10D46000810301D5112034E0410301D5122030E0C1
:10D47000010301D513202CE0C10201D5142028E0BE
:10D48000810201D5152024E0410201D5162020E0BB
:10D49000010201D517201CE0C10101D5182018E0B8
:10D4A000810101D5192014E0410101D51A2010E0B5
:10D4B000010101D51B200CE0C10001D51C2008E0B2
:10D4C000810001D51D2004E0400001D51E2000E0B0
:10D4D0001F20704730B400220023994203D19042AC
:10D4E00001D14020FCE10200D20701D50020F7E184
:10D4F0000200920701D50120F2E10200520701D596
:10D500000220EDE10200120701D50320E8E102004C
:10D51000D20601D50420E3E10200920601D50520E0
:10D52000DEE10200520601D50620D9E10200120612
:10D5300001D50720D4E1C20501D50820D0E182053C
:10D5400001D50920CCE1420501D50A20C8E1020538
:10D5500001D50B20C4E1C20401D50C20C0E1820436
:10D5600001D50D20BCE1420401D50E20B8E1020432
:10D5700001D50F20B4E1C20301D51020B0E1820330
:10D5800001D51120ACE1420301D51220A8E102032C
:10D5900001D51320A4E1C20201D51420A0E182022A
:10D5A00001D515209CE1420201D5162098E1020226
:10D5B00001D5172094E1C20101D5182090E1820124
:10D5C00001D519208CE1420101D51A2088E1020120
:10D5D00001D51B2084E1C20001D51C2080E182001E
:10D5E00001D51D207CE1420001D51E2078E10028F4
:10D5F00001D51F2074E110F0000211F00103002496
:10D600000025AB4201D1A24201D0202068E110F0F8
:10D61000000211F0020300240025AB4201D1A24216
:10D6200001D021205CE110F0000211F0040300247D
:10D630000025AB4201D1A24201D0222050E110F0DE
:10D64000000211F0080300240025AB4201D1A242E0
:10D6500001D0232044E110F0000211F01003002457
:10D660000025AB4201D1A24201D0242038E110F0C4
:10D67000000211F0200300240025AB4201D1A24298
:10D6800001D025202CE110F0000211F0400300240D
:10D690000025AB4201D1A24201D0262020E110F0AA
:10D6A000000211F0800300240025AB4201D1A24208
:10D6B00001D0272014E110F0000211F4807300243F
:10D6C0000025AB4201D1A24201D0282008E110F090
:10D6D000000211F4007300240025AB4201D1A242E4
:10D6E00001D02920FCE010F0000211F48063002436
:10D6F0000025AB4201D1A24201D02A20F0E010F077
:10D70000000211F4006300240025AB4201D1A242C3
:10D7100001D02B20E4E010F0000211F4805300242B
:10D720000025AB4201D1A24201D02C20D8E010F05C
:10D73000000211F4005300240025AB4201D1A242A3
:10D7400001D02D20CCE010F0000211F48043002421
:10D750000025AB4201D1A24201D02E20C0E010F042
:10D76000000211F4004300240025AB4201D1A24283
:10D7700001D02F20B4E010F0000211F48033002417
:10D780000025AB4201D1A24201D03020A8E010F028
:10D79000000211F4003300240025AB4201D1A24263
:10D7A00001D031209CE010F0000211F4802300240D
:10D7B0000025AB4201D1A24201D0322090E010F00E
:10D7C000000211F4002300240025AB4201D1A24243
:10D7D00001D0332084E010F0000211F48013002403
:10D7E0000025AB4201D1A24201D0342078E010F0F4
:10D7F000000211F4001300240025AB4201D1A24223
:10D8000001D035206CE010F0000211F480030024F8
:10D810000025AB4201D1A24201D0362060E010F0D9
:10D82000000211F4000300240025AB4201D1A24202
:10D8300001D0372054E010F0000211F08073002472
:10D840000025AB4201D1A24201D0382048E010F0BF
:10D85000000211F0007300240025AB4201D1A24266
:10D8600001D039203CE010F0000211F08063002468
:10D870000025AB4201D1A24201D03A2030E010F0A5
:10D88000000211F0006300240025AB4201D1A24246
:10D8900001D03B2024E010F0000211F0805300245E
:10D8A0000025AB4201D1A24201D03C2018E010F08B
:10D8B000000211F0005300240025AB4201D1A24226
:10D8C00001D03D200CE010F0000011F0804100225A
:10D8D0000023994201D1904201D03E2000E03F2038
:10D8E00030BC7047012111FA00F07047054908600B
:10D8F0007047054908607047024800687047024851
:10D9000000687047BC110020C011002080B562483B
:10D910003021017030214170302181703021C1707F
:10D920005E483021017030214170302181703021FA
:10D93000C17000F06FF800F088F801BDF0B4040089
:10D94000049D0120E4B2002C29D1554C0E0027780B
:10D95000F6B2BE4201D0002013E016006778F6B29E
:10D96000BE4201D000200CE01E00A778F6B2BE42F5
:10D9700001D0002005E02E00E478F6B2A64200D0E7
:10D980000020C9B2332933D1D2B2312A30D1DBB22F
:10D99000302B2DD1EDB2312D2AD1012028E0414C80
:10D9A0000E002778F6B2BE4201D0002013E0160028
:10D9B0006778F6B2BE4201D000200CE01E00A778C6
:10D9C000F6B2BE4201D0002005E02E00E478F6B2A7
:10D9D000A64200D00020C9B2332909D1D2B2312ADF
:10D9E00006D1DBB2302B03D1EDB2312D00D10120B5
:10D9F000F0BC704710B4294C20706170A270E370C5
:10DA000010BC704710B4264C20706170A270E37097
:10DA100010BC7047224821490A7802704A78427047
:10DA20008A788270C978C170704710B41D4C20701C
:10DA30006170A270E37010BC704710B4164C207077
:10DA40006170A270E37010BC7047164812490A78E2
:10DA500002704A7842708A788270C978C1707047C3
:10DA6000042801D3302001E00D49085C70470428E8
:10DA700001D3302001E00949085C7047042801D334
:10DA8000302001E00749085C7047042801D33020AA
:10DA900001E00149085C7047F0110020F4110020FA
:10DAA000EC110020E81100205948002101600068B5
:10DAB000C04358490860704755480068554909688F
:10DAC000C943884201D1012000E0002070470200D4
:10DAD000C943D2B2C9B28A4206D14D49C0B2086028
:10DAE0000868C0434B490860704749490A68C0B29A
:10DAF000104308600868C0434649086070474449BD
:10DB00000A68C0B232EA000008600868C0434149B0
:10DB1000086070473E490968C0B2084070473C48F9
:10DB20000178890701D50A204EE00178C90706D59A
:10DB30000078400701D5092046E0082044E001783C
:10DB4000890606D50078400701D507203CE006206D
:10DB50003AE0017849060BD50178090701D50C2078
:10DB600032E00078C00601D50D202DE00B202BE01F
:10DB7000017811F0180F06D10078400701D5032075
:10DB800022E0002020E0017811F01801182906D1C8
:10DB90000078400701D50F2016E00E2014E0017830
:10DBA000090706D50078400701D504200CE00120C4
:10DBB0000AE00178C90606D50078400701D505209E
:10DBC00002E0022000E00020704738B504000D009C
:10DBD000FFF7A5FF0C2806D10F4B104A29002000A3
:10DBE000FDF7F7FB10E00D2806D10B4B0C4A29007E
:10DBF0002000FDF7EEFB07E00A4951F8203003A2B0
:10DC000029002000FDF7E5FB31BD00002573200051
:10DC1000E0110020E411002080F4030048F001002E
:10DC200050F001002402002080B5FFF73DFFFEF711
:10DC3000FFFE00F0F5F8FFF769FEFEF79BFE01BD61
:10DC400080B5FEF709FF002803D0FFF735FF002855
:10DC500003D10220FFF726F802E00220FFF71CF8AC
:10DC60001020FFF7C2FA01BD5649087070475548A9
:10DC700000787047544908607047544908607047FD
:10DC80005248006870475249086070475048006821
:10DC900070475049086070474E48006870474E49C9
:10DCA000086070474C4800687047010402D44B4933
:10DCB000086005E040F07F4050F47F00474908606D
:10DCC000704746480068704745490A681043086035
:10DCD000704743480068704700204149086070471A
:10DCE00080B50A00374B1978002903D13D49FDF76B
:10DCF00015FA64E01978012903D13B49FDF70EFAC2
:10DD00005DE01978022903D13849FDF707FA56E09A
:10DD10001978032903D13649FDF700FA4FE0197845
:10DD2000042903D13349FDF7F9F948E019780529A9
:10DD300003D13149FDF7F2F941E01978062903D101
:10DD40002E49FDF7EBF93AE01978072903D12C4960
:10DD5000FDF7E4F933E01978082903D12949FDF7E3
:10DD6000DDF92CE01978092903D12749FDF7D6F907
:10DD700025E019780A2903D12449FDF7CFF91EE0DF
:10DD800019780B2903D12249FDF7C8F917E0197852
:10DD90000C2903D11F49FDF7C1F910E019780D29AD
:10DDA00003D11D49FDF7BAF909E01978802903DB91
:10DDB0001A49FDF7B3F902E01749FDF7AFF901BDC4
:10DDC00000000000111200208011002084110020AA
:10DDD000881100208C110020901100209411002047
:10DDE00098110020A0E30300C0E3030080DD0300DE
:10DDF000E0E3030000E4030020E4030040E4030048
:10DE000060E4030080E40300A0E40300C0E4030036
:10DE1000E0E4030020DF030020E5030040E5030009
:10DE2000002006E0FF216B4A115400216A4A115478
:10DE3000401C0E28F6D3704768490860704768494F
:10DE40000860704767490860704780B55720FEF743
:10DE5000A4FD012802D16148006800E0002002BD55
:10DE600080B55720FEF799FD012802D15D48006872
:10DE700000E0002002BD80B55720FEF78EFD01288E
:10DE800002D15748006800E0002002BD56490968E9
:10DE9000884202D15548006800E000207047524A8D
:10DEA000106052480160704780B5012806D15FF0CC
:10DEB000FF304FF6FF7100F061F909E04A49096847
:10DEC000884203D14A48D0E9000101E00020002146
:10DED00004BD454908604648C0E90023704780B545
:10DEE000012802D1FFF708FD07E03F490968884291
:10DEF00002D14048006800E0002002BD3A4A1060AC
:10DF00003C480160704738490968884202D13A4864
:10DF1000006800E000207047334A10603648016016
:10DF2000704710B50C0001280FD1FEF7C6FD002C7C
:10DF300003D10A21B0FBF1F004E00A21B0FBF1F2B9
:10DF400001FB1200FFF73DFA07E027490968884204
:10DF500002D12A48005D00E0002010BD224B18606D
:10DF600026484254704780B5811E0E2904D21A49B2
:10DF7000084410F8020C06E0012803D11E20FEF729
:10DF80000CFD00E0002002BD821E0E2A03D2124AC0
:10DF9000104400F8021C704780B5811E0E2904D27F
:10DFA0000C49084410F8020C0BE0012808D1592054
:10DFB000FEF7F3FC002801D0012002E0002000E081
:10DFC000002002BD821E0E2A03D2024A104400F82D
:10DFD000021C7047A8100020981000209C110020FF
:10DFE000A4110020A0110020A8110020AC110020D5
:10DFF000E0100020B0110020B41100200E1200200B
:10E000002C4AC0B2115470472A49C0B2085C70470C
:10E01000F8B584B004000D000320FFF7F5FF0128D8
:10E0200005D10422244903A8FDF778F82CE0022842
:10E0300005D10422214903A8FDF770F824E0032844
:10E0400005D104221E4903A8FDF768F81CE0042846
:10E0500005D104221B4903A8FDF760F814E0052848
:10E0600005D10422184903A8FDF758F80CE006284A
:10E0700005D10422154903A8FDF750F804E0042255
:10E08000134903A8FDF74AF80520FFF7BDFF060076
:10E090000420FFF7B9FF07000220FFF7B5FF029643
:10E0A0000197009003AB0B4A29002000FDF791F97E
:10E0B00005B0F0BDF010002000EB030020EB0300E2
:10E0C00040EB030060EB030080EB0300A0EB0300D8
:10E0D000C0EB0300E0E60100D2B2203A22BF00FA12
:10E0E00002F1002070475242D041D2F1200291400B
:10E0F0004140D04090404140704730B4002513E08B
:10E1000050F8042BD30744BFA9F101039A18091F43
:10E11000042942F8045BFAD213468C0744BF1580E9
:10E120009B1CC90748BF1D7050F8041B0029E7D18C
:10E1300030BC70474D49086070474D4908607047D2
:10E140004A490968084070474949096808407047CA
:10E1500080B54649086800280AD00868FFF738F9F2
:10E16000202803D2434951F8200002E0002000E0BB
:10E17000002002BD404AC2E9000170473E4AD2E990
:10E1800000231040194070473C49086070473B48E5
:10E190000068704738B504000800FFF719F905005A
:10E1A000374850F825000090324850F82530354A5D
:10E1B00016212000FDF70DF90A2D08D132480090F4
:10E1C0000B23324A16212000FDF703F927E00B2D1F
:10E1D00008D12D4800900C232D4A16212000FDF770
:10E1E000F8F81CE00C2D0CD1FEF789FC012808D1B1
:10E1F000254800900D23274A16212000FDF7E9F855
:10E200000DE00D2D0BD1FEF77AFC012807D11E4839
:10E2100000900E23204A16212000FDF7DAF831BDC8
:10E220001CB504000800FFF7D3F81C4951F8201072
:10E2300000911B4951F82030124A16212000FDF7A9
:10E24000C8F813BD1CB5040010001900FFF742F90F
:10E25000144951F820100091134951F82030094A0F
:10E2600016212000FDF7B5F813BD0000C4110020F1
:10E27000C811002014DE0100E8100020CC1100209D
:10E2800000000020F8EF0100E0DF0300CCEA01000D
:10E29000D8EA0100E4EA0100F0EA010024010020CC
:10E2A00094DE01008000002070DD0100DFF87013B3
:10E2B00008607047DFF86C1308607047DFF8600390
:10E2C00000687047DFF85C030068704780B5130092
:10E2D000B3F11602082A07D30A00DFF84C1351F8ED
:10E2E0002310FCF71BFF07E0DFF83C2352F8233034
:10E2F000DFF83823FDF76DF801BD202801D3002099
:10E3000003E0DFF82C1351F820007047012801D1F9
:10E31000022078E0022801D11E2074E0032801D1F8
:10E32000212070E0042801D109206CE0052801D1EA
:10E330001E2068E0062801D11F2064E0072801D1D3
:10E34000042060E0082801D105205CE0092801D103
:10E35000062058E00A2801D1072054E00B2801D1FB
:10E36000182050E00C2801D108204CE00D2801D1E4
:10E370000E2048E00E2801D11A2044E00F2801D1D8
:10E380000B2040E0102801D10A203CE0112801D1E7
:10E39000152038E0122801D1142034E0132801D1CF
:10E3A000132030E0142801D112202CE0152801D1CF
:10E3B000192028E0162801D1012024E0172801D1D6
:10E3C000032020E0182801D10F201CE0192801D1DA
:10E3D000102018E01A2801D1112014E01B2801D1C7
:10E3E0000D2010E01C2801D116200CE01D2801D1C1
:10E3F0001B2008E01E2801D10C2004E01F2801D1B9
:10E40000172000E000207047022801D1012078E0A9
:10E41000202801D1022074E0212801D1032070E0DE
:10E42000092801D104206CE01E2801D1052068E0F4
:10E430001F2801D1062064E0042801D1072060E0F4
:10E44000052801D108205CE0062801D1092058E008
:10E45000072801D10A2054E0182801D10B2050E0F0
:10E46000082801D10C204CE00E2801D10D2048E0F5
:10E470001A2801D10E2044E00B2801D10F2040E0E2
:10E480000A2801D110203CE0152801D1112038E0E4
:10E49000142801D1122034E0132801D1132030E0D8
:10E4A000122801D114202CE0192801D1152028E0D0
:10E4B000012801D1162024E0032801D1172020E0F3
:10E4C0000F2801D118201CE0102801D1192018E0D4
:10E4D000112801D11A2014E00D2801D11B2010E0D1
:10E4E000162801D11C200CE01B2801D11D2008E0BA
:10E4F0000C2801D11E2004E0172801D11F2000E0C4
:10E500000020C0B2704780B51300DBB2012B04D1EC
:10E510000A004849FCF702FE80E01300DBB2022B40
:10E5200004D10A004449FCF7F9FD77E01300DBB29F
:10E53000032B04D10A004149FCF7F0FD6EE0130003
:10E54000DBB2042B04D10A003D49FCF7E7FD65E08E
:10E550001300DBB2052B04D10A003A49FCF7DEFDBB
:10E560005CE01300DBB2062B04D10A003649FCF74D
:10E57000D5FD53E01300DBB2072B04D10A00334969
:10E58000FCF7CCFD4AE01300DBB2082B04D10A00F3
:10E590002F49FCF7C3FD41E01300DBB2092B04D186
:10E5A0000A002C49FCF7BAFD38E01300DBB20A2B55
:10E5B00004D10A002849FCF7B1FD2FE01300DBB2BB
:10E5C0000B2B04D10A002549FCF7A8FD26E0130017
:10E5D000DBB20C2B04D10A002149FCF79FFD1DE0A2
:10E5E0001300DBB20D2B04D11E4B1F4AFCF7F1FECA
:10E5F00014E01300DBB20E2B04D11A4B1B4AFCF7BC
:10E60000E8FE0BE0D2B20F2A04D10A001849FCF749
:10E6100085FD03E00A001749FCF780FD01BD0000FD
:10E62000D8110020DC110020A4010020FCEA010028
:10E6300014DF0100A0E8030020E50300C0E80300A8
:10E64000E0E8030020DF030020E9030040E90300C5
:10E6500060E9030080E90300A0E9030040E703004C
:10E66000C0D4030008E8010038F0010040F00100C8
:10E6700028EB010080E6030010B54A4C0121200080
:10E6800000F010FE0A2366220121200000F07AFD2E
:10E690000221200000F006FE0A236622022120004B
:10E6A00000F070FD0421200000F0FCFD0A2366222A
:10E6B0000421200000F066FD0821200000F0F2FD9A
:10E6C0000A2366220821200000F05CFD80213648E4
:10E6D00000F0E8FDFEF786FD0A38344908600020A6
:10E6E0003349086010BD10B5FEF77CFD2F4C216842
:10E6F000401A0A2825D3FEF775FD206000202D4919
:10E700000968002901D150F001002B49096800294E
:10E7100001D150F0020029490968002901D150F0C7
:10E72000040027490968002901D150F00800254953
:10E730000968002901D050F0100000F00BF81C49C6
:10E7400008600120FEF751FD10BD19490968C0B2EB
:10E750000840704730B402001000002304E01A495A
:10E7600051F8231008435B1C032BF8D3164DE968BE
:10E7700008401300002403E055F824100B40641CEB
:10E78000032CF9D31843E860022106E005EB81036E
:10E7900053F8043C45F82130491E0029F6D12A607F
:10E7A00030BC704700700040005000404411002011
:10E7B00040110020047000400870004010700040BC
:10E7C00020700040005200408810002010B5FCF777
:10E7D0003DFEDFF8844904222021200000F049FE9C
:10E7E0002068002805D02068012802D0002000F011
:10E7F000A2FC10BD38B5FCF749FEFCF733FEFCF770
:10E800003EFF0500FCF740FF04005FF0FF30FEF71D
:10E810004EFA002808D02800C0B207280CD00321E7
:10E820000720FCF7CAFE07E02800C0B2072803D182
:10E8300003210120FCF7C1FE2800C0B2002804D14A
:10E84000200002F0FFF800F067BC2800C0B20128E9
:10E8500004D1200002F01AF900F05EBC2800C0B21A
:10E86000062804D1200002F0B9FB00F055BC2800B6
:10E87000C0B2082804D1200002F04AFE00F04CBCCF
:10E880002800C0B2072804D1200002F059FD00F092
:10E8900043BC2800C0B2022804D1200003F06FFC62
:10E8A00000F03ABC2800C0B28C2804D1200002F04D
:10E8B000B7FF00F031BC2800C0B2032803D103F039
:10E8C00099FD00F029BC2800C0B2102804D1200016
:10E8D00003F011F800F020BC2800C0B2112804D1C8
:10E8E000200003F0CBF800F017BC2800C0B21228BB
:10E8F00004D1200003F080F900F00EBC2800C0B263
:10E90000132804D1200003F063FA00F005BC2800AE
:10E91000C0B2142803D1200003F042FBFCE328001E
:10E92000C0B2152802D103F0B5FBF5E32800C0B250
:10E930001C2803D1200003F0C5FDEDE32800C0B280
:10E940001D2803D1200003F051FEE5E32800C0B2EA
:10E950001E2803D1200003F0E7FEDDE32800C0B24B
:10E960001F2803D1200004F0B9F8D5E32800C0B275
:10E97000092802D104F0DCF9CEE32800C0B20C284B
:10E9800002D104F0AEFBC7E32800C0B20A2802D1CE
:10E9900004F05AF9C0E32800C0B20B2802D104F0F9
:10E9A0006CFAB9E32800C0B20D2802D104F0FAFADB
:10E9B000B2E32800C0B2162803D1200004F0F0FB17
:10E9C000AAE32800C0B2172802D104F087FCA3E311
:10E9D0002800C0B2182803D1200004F0F3FC9BE308
:10E9E0002800C0B2192803D1200004F097FE93E359
:10E9F0002800C0B21A2803D1200004F034FF8BE3B2
:10EA00002800C0B21B2802D104F0C0FF84E3280014
:10EA1000C0B23A2803D1200005F046F87CE3280074
:10EA2000C0B23B2803D1200005F0CFF874E32800E2
:10EA3000C0B2202803D1200005F09AF96CE3280029
:10EA4000C0B23C2803D1200005F06AFF64E328002F
:10EA5000C0B23D2803D1200006F062F85CE3280034
:10EA6000C0B23E2803D1200006F01AF954E3280072
:10EA7000C0B23F2803D1200006F076FA4CE328000C
:10EA8000C0B2412803D1200006F091F944E32800E8
:10EA9000C0B2402803D1200006F0F3F93CE328007F
:10EAA000C0B2422803D1200006F01EFB34E3280048
:10EAB000C0B2442803D1200006F0A8FF2CE32800B0
:10EAC000C0B2432803D1200006F094FE24E32800BE
:10EAD000C0B2452803D1200007F07EF91CE32800CE
:10EAE000C0B2462803D1200007F0E4F914E328005F
:10EAF000C0B2472803D1200007F03CFB0CE32800FC
:10EB0000C0B2482803D1200007F09CFA04E3280093
:10EB1000C0B2492803D1200007F0DCFBFCE228004A
:10EB2000C0B24A2803D1200007F062FCF4E22800BA
:10EB3000C0B24B2803D1200007F02CFDECE22800E6
:10EB4000C0B24C2803D1200007F090FDE4E2280079
:10EB5000C0B24D2803D1200007F0F8FDDCE2280008
:10EB6000C0B24E2803D1200007F05EFED4E2280098
:10EB7000C0B24F2803D1200007F0D4FECCE2280019
:10EB8000C0B2502803D1200007F054FFC4E228008F
:10EB9000C0B2512803D1200007F0BAFFBCE2280020
:10EBA000C0B2522803D1200008F05AF8B4E228007D
:10EBB000C0B2532803D1200008F021F9ACE22800AC
:10EBC000C0B2542803D1200008F088F9A4E228003C
:10EBD000C0B2552803D1200008F0F3F99CE22800C8
:10EBE000C0B2562803D1200008F05AFA94E2280057
:10EBF000C0B2572803D1200008F0C0FA8CE22800E8
:10EC0000C0B2582803D1200008F030FB84E228006D
:10EC1000C0B2592803D1200008F096FB7CE22800FE
:10EC2000C0B25A2803D1200008F0F9FB74E2280092
:10EC3000C0B25B2803D1200008F062FC6CE228001F
:10EC4000C0B25C2802D108F0FFFC65E22800C0B227
:10EC50005D2802D108F08BFD5EE22800C0B25E287C
:10EC600002D108F0EFFD57E22800C0B25F2802D1C0
:10EC700008F053FE50E22800C0B2252803D120003E
:10EC800005F05CFD48E22800C0B2792803D12000DD
:10EC900008F0C6FE40E22800C0B27A2803D1200066
:10ECA00009F015F838E22800C0B27B2803D1200013
:10ECB00009F09EF830E22800C0B27D2803D1200080
:10ECC00009F044F928E22800C0B27C2803D12000D2
:10ECD00009F0D6F920E22800C0B27E2803D1200036
:10ECE00009F05EFA18E22800C0B27F2803D12000A4
:10ECF00009F0B5FA10E22800C0B2802803D1200044
:10ED000009F004FB08E22800C0B2812803D12000EA
:10ED100009F078FB00E22800C0B2822803D120006D
:10ED200009F0AAFCF8E12800C0B2832803D1200032
:10ED300009F013FFF0E12800C0B2842803D12000BD
:10ED400009F05AFDE8E12800C0B2852803D120006F
:10ED500009F002FEE0E12800C0B2862803D12000BD
:10ED600009F097FED8E12800C0B2872803D120001F
:10ED700009F0DCFFD0E12800C0B2882803D12000D0
:10ED80000AF0BAF8C8E12800C0B2892803D12000EF
:10ED90000AF073F9C0E12800C0B28A2804D1012129
:10EDA00020000AF0FBF9B7E12800C0B28B2804D19B
:10EDB000022120000AF0F2F9AEE12800C0B22628B4
:10EDC00003D120000AF09EFAA6E12800C0B227284D
:10EDD00003D120000AF07DFB9EE12800C0B2282864
:10EDE00003D120000AF08EFC96E12800C0B2292849
:10EDF00003D120000AF00BFC8EE12800C0B22A28C3
:10EE000003D120000AF00AFD86E12800C0B22B28B9
:10EE100003D120000AF09EFD7EE12800C0B22C281C
:10EE200003D120000AF08AFE76E12800C0B22D2826
:10EE300003D120000AF021FF6EE12800C0B22E2885
:10EE400003D120000AF0FAFF66E12800C0B22F28A3
:10EE500003D120000BF078F85EE12800C0B26028F2
:10EE600003D120000BF02AF956E12800C0B2212876
:10EE700003D1200005F080F94EE12800C0B222281D
:10EE800003D1200005F052FA46E12800C0B2232841
:10EE900003D1200005F018FB3EE12800C0B2242871
:10EEA00003D1200005F0A0FB36E12800C0B26128A4
:10EEB00003D120000BF05CFA2EE12800C0B26228DA
:10EEC00003D120000BF055FB26E12800C0B26328D7
:10EED00003D120000BF0C6FA1EE12800C0B264285E
:10EEE00002D10BF0C2FB17E12800C0B2652802D1A5
:10EEF0000BF016FC10E12800C0B2662802D10BF01E
:10EF000087FC09E12800C0B2672802D10BF0C8FCD9
:10EF100002E12800C0B2682803D120000BF000FEF7
:10EF2000FAE02800C0B2692803D120000CF09AF85A
:10EF3000F2E02800C0B2772803D120000CF024FCB6
:10EF4000EAE02800C0B26A2803D120000CF004F9DE
:10EF5000E2E02800C0B26B2803D120000CF075F964
:10EF6000DAE02800C0B26C2803D120000CF0D9F9F7
:10EF7000D2E02800C0B26D2803D120000CF040FA86
:10EF8000CAE02800C0B26E2803D120000CF0B4FA09
:10EF9000C2E02800C0B26F2803D120000CF02AFB89
:10EFA000BAE02800C0B2702803D120000CF068FC41
:10EFB000B2E02800C0B2712803D120000CF0D0FCD0
:10EFC000AAE02800C0B2722803D120000CF0B2FDE4
:10EFD000A2E02800C0B2732803D120000CF046FE46
:10EFE0009AE02800C0B2742803D120000CF0CEFEB5
:10EFF00092E02800C0B2752803D120000CF046FF33
:10F000008AE02800C0B2782803D120000CF01AFD55
:10F0100082E02800C0B2762803D120000CF0B2FFB5
:10F020007AE02800C0B28D2803D120000DF05CF8F2
:10F0300072E02800C0B28E2803D120000DF0CAF87B
:10F040006AE02800C0B28F2803D120000DF033F908
:10F0500062E02800C0B2302803D12000F9F706F999
:10F060005AE02800C0B2312803D12000F9F739FA5C
:10F0700052E02800C0B2322803D12000F9F7BCFAD0
:10F080004AE02800C0B2332803D12000F9F746FC3B
:10F0900042E02800C0B2342803D12000F9F7E0FE96
:10F0A0003AE02800C0B2352803D12000FAF708F86A
:10F0B00032E02800C0B2362803D12000FAF7B0F8B9
:10F0C0002AE02800C0B2372803D12000FAF75EF901
:10F0D00022E02800C0B2382803D12000FAF7FAF95C
:10F0E0001AE02800C0B2392803D12000FAF712FC38
:10F0F00012E02800C0B20E2803D1200002F08FF9E0
:10F100000AE0EDB20F2D03D1200002F0D2F803E0A7
:10F1100003210120FCF751FAFCF7F8FC002803D189
:10F1200003210120FCF749FA0220FEF75EF831BD09
:10F1300009480068704780B5002801D0012806D131
:10F14000054A10602021106800F0F4F902E0012067
:10F15000FDF7A8FD01BD00004C11002038B5CB43E0
:10F1600000F58064D50725684CBF0D431D40256020
:10F1700000F58460920747BF026811430168194097
:10F18000016031BD2DE9F84104464FF0000C04F652
:10F19000C4750326012707FA0CF0014212D04FEA8A
:10F1A0004C00D5F800E006FA00F82EEA080EC5F883
:10F1B00000E0C2F34118D5F800E008FA00F040EA98
:10F1C0000E0028600CF1010CBCF1080FE3DBC84312
:10F1D00004F5A065D6072E684CBF0E4306402E608E
:10F1E00004F2045596072E684CBF0E4306402E606D
:10F1F00004F5A16556072E684CBF0E4306402E60ED
:10F2000004F5A36516072E684CBF0E4306402E601A
:10F2100004F23C55D2062A684CBF0A4302402A60D9
:10F22000DD0704F20C5215684CBF0D430540156014
:10F2300004F5A2629D0715684CBF0D43054015609B
:10F2400004F214525D0715684CBF0D43054015606C
:10F2500004F21C521D0715684CBF0D430540156094
:10F2600004F244529D0515684CBF0D4305401560DE
:10F2700004F5A86213F4407F156814BF0D430540E0
:10F28000156004F5A564002B07BF206808432168BA
:10F2900008402060BDE8F18100EB8100026070470A
:10F2A00001226FE738B500F02DF82946204601B05D
:10F2B000BDE830400823F3E738B504460D4608237F
:10F2C000FFE70122FFF75EFF29462046BDE83840F0
:10F2D000012243E704460D4602223FE738B5FFF717
:10F2E000F9FF2946204601B0BDE830400823D7E7A2
:10F2F00038B5FFF7EFFF2946204601B0BDE83040A2
:10F300000823CDE704460D46002227E710B50D4B34
:10F310000FF234021C68C0F30741CC40E40746BF3B
:10F3200002EBC101496852F8311001F22C51020A76
:10F330000B680F24944000F00F00A3439040184343
:10F34000086010BD6CE00F400040004000800540A8
:10F3500000500040009005400060004000A00540C3
:10F360000070004000B005400040024000C0054071
:10F370000050024000D005400060024000E005401F
:10F380000070024000F0054000D00340000006403D
:10F3900000100640001006400020064000200640F5
:10F3A0000030064000300640004006400040064065
:10F3B00000500640005006400060064000600640D5
:10F3C0000070064000700640008006400080064045
:10F3D000009006400090064038B5044600F029F839
:10F3E000614D0321296000F024F80120E40900FAAE
:10F3F00004F45E48E443046000F01BF80020286039
:10F400000A20BDE8324000F08DBF10B500F011F8C1
:10F41000554C0321216000F00CF85449002008608D
:10F4200000F007F8002020600A20BDE8104000F03E
:10F4300079BF0A2000F076BF10B5022000F072FFFD
:10F440004B4C2168C807FCD4606810F00C0F0CD13D
:10F45000484800F01FFF022000F064FF2068C10749
:10F46000FCD4606810F00C0F01D0022010BD002009
:10F4700010BD10B5404B8C091C60C1F3830192088C
:10F4800059600AD004E0596811B91C68641C1C60FA
:10F49000521E196940F8041BF5D110BD2DE9F84F33
:10F4A00081468A46344D6869C007FCD4DFF8CC80B9
:10F4B000334F344E4FEA9A1028609408CAF3830001
:10F4C000686005D12AE0686810B92968491C29607C
:10F4D00030683840404505D13068010404BF5046CB
:10F4E000FFF77AFFD9F800002861FFF7A2FFD5F8EF
:10F4F00014B05FEACB70FAD45FEACB600AD530680B
:10F500000740474504D13068010408BFFFF77DFF7D
:10F5100058460DE0641E09F10409D4D13068074053
:10F52000474504D13068010408BFFFF76EFF6869E2
:10F53000BDE8F28F38B50D461249104B0A680446F3
:10F540000F4802409A4205D10968080404BF2846C2
:10F55000FFF742FF0848A9090160C5F38301416034
:10F560000461406932BD0000FCD00F40C0E20A4097
:10F5700018F00A40005800F004F00A40000005109E
:10F580000000FF7000E00F4038B5002003E00021CC
:10F590000F4A1154401C40F205418842F7D300F055
:10F5A00038FB0C4C0A4D402380222900200000F03B
:10F5B00075F8280000F004FB074D210028000CF02E
:10F5C0006DFF0649280000F05FFE31BD044870471A
:10F5D000A0020020800F0020540F0020A8DC0100B2
:10F5E000A50200202DE9F0470A9C0D00ED0811F05E
:10F5F0000701802606FB050004EB00051C00E4085B
:10F6000013F0070F00D0641CD2F180030027089884
:10F61000099E01E01D447F1CA7423DD25FF0000C13
:10F620009445F7D2002814D195F800E096F80080B0
:10F6300018FA01F858EA0E0E85F800E015F1800E70
:10F6400096F80080D1F1080958FA09F88EF8008080
:10F650001DE095F800E096F800807FEA080818FAA7
:10F6600001F858EA0E0E85F800E015F1800E9EF8BC
:10F67000008096F800907FEA0909D1F1080A59FA4A
:10F680000AF959EA080818F007088EF800806D1C7E
:10F69000761C1CF1010CC3E7BDE8F08710B42824E8
:10F6A00004604160028143810FF23904C4600FF2AB
:10F6B000610404610FF2192444610FF24D24846146
:10F6C0000FF22934C4610FF2CD4404620FF2F14409
:10F6D000446201200870A1F80120A1F8033010BC99
:10F6E0007047000030B4B0F80140082592FBF5F5F2
:10F6F00004FB05110844401D12F0070201780124A3
:10F700009440A14313FA02F20A43027030BC7047DE
:10F710002DE9F04105000C000698DDF81CC0089E9C
:10F72000099FB5F80110C91D5FF0080E91FBFEFEA0
:10F73000082194FBF1F102FB0E1205EB02014A1DB8
:10F7400014F00704D4F10704BCF1010F00F08C8021
:10F75000BCF1040F04D0BCF1080F00F0B380B5E099
:10F7600013F00103DBB2002B02D0012B2FD081E07C
:10F77000002800F07F803378DBB21B09DBB2032165
:10F780004B43FB5823F07F4315780121A1408D4363
:10F79000C3F3074C44F6CD4EC3F3072849F20A7170
:10F7A00001FB08F80EFB0C8C03F0FF0341F6294126
:10F7B00001FB03C3DB0DA3402B43137021004C1E40
:10F7C000002901D10724521C401E0028D0D03378D4
:10F7D00013F00F0303214B43761CFB5823F07F43A8
:10F7E00015780121A1408D43C3F3074C44F6CD4E5B
:10F7F000C3F3072849F20A7101FB08F80EFB0C8CD1
:10F8000003F0FF0341F6294101FB03C3DB0DA340D5
:10F810002B43137021004C1E002901D10724521CD8
:10F82000401EA5E711785FF0010C1CFA04FC31EAD8
:10F830000C01D3F1070CAE463EFA0CFE1EF0010E91
:10F8400057F82EC01CFA04FC5CEA0101117021007B
:10F850004C1E002901D10724521C5B1C401E082BA2
:10F8600001DA0028DED10023002802D03578761C8A
:10F87000F5E72BE02AE0337803214B43761CFB5855
:10F8800023F07F4315780121A1408D43C3F3074C3A
:10F8900044F6CD4EC3F3072849F20A7101FB08F87C
:10F8A0000EFB0C8C03F0FF0341F6294101FB03C35F
:10F8B000DB0DA3402B43137021004C1E002901D106
:10F8C0000724521C0100481E0029D4D1BDE8F08154
:10F8D00070B4039CB0F80150082693FBF6F605FBC4
:10F8E00006152844451D13F0070309E02E78012072
:10F8F0009840864314FA03F006432E706D1C491C91
:10F900008A42F3DA70BC704770B4039CB0F80150BF
:10F91000082692FBF6F605FB06110844411D002C53
:10F9200000D0FF2412F0070F19D012F00706D6F10D
:10F930000806981A401CB04201DA9E1A761C012073
:10F9400010FA06F6761E12F0070086400878B043DB
:10F95000264006430E702944D21D32F007020800EB
:10F96000C00705D5981A072802DB0C702944083215
:10F970000800800715D5981A0F2812DB0C7001EBD0
:10F980000500047000EB050110320AE00C7001EB79
:10F9900005000470284404702844047000EB05013D
:10F9A000203212F11F008342F0DA12F10F0083427D
:10F9B00006DB0C7001EB0500047000EB0501103252
:10F9C000D01D834202DB0C702944083293420ADBCB
:10F9D000FF209A1A521C10FA02F208781040D24303
:10F9E000224002430A7070BC70470000F0B5B0F8C6
:10F9F0000140B1F90230082593FBF5F5B1F900306B
:10FA000004FB05352844451D002A00D0FF22B1F92A
:10FA1000023013F0070F2DD013F00707D7F10807B6
:10FA2000B1F90600C01A401CB84203DAB1F90670F9
:10FA3000FF1A7F1C012010FA07F77F1E13F0070042
:10FA40008740B1F900C02E000CE096F800E03EEAD5
:10FA5000070E17EA020050EA0E0E86F800E01CF1CD
:10FA6000010C761CB1F904006045EEDA2544DB1D7B
:10FA700033F007032800C00711D5B1F90600C01AFA
:10FA800007280CDBB1F90060280002E00270761C48
:10FA9000401CB1F90470B742F8DA25440833280055
:10FAA00080071FD5B1F90600C01A0F281ADBB1F97B
:10FAB0000060280006E0028020442A806742384423
:10FAC000761C401CB1F90470B742F4DA25441033B7
:10FAD00008E00260761C401CB1F90470B742F8DA05
:10FAE00025440833B1F9060013F11F06B04203DBC9
:10FAF000B1F900602800EFE7B1F9060013F10F0635
:10FB0000B0421BDBB1F90060280002E00280761CE5
:10FB1000401CB1F90470B742F8DA05EB0400083371
:10FB2000B1F90060050002E02A80761C6D1CB1F975
:10FB30000470B742F8DA00EB04050833B1F90600A7
:10FB4000DE1DB0420CDBB1F90060280002E002705B
:10FB5000761C401CB1F90470B742F8DA254408332A
:10FB6000B1F90600984214DBFF20CC88E31A5B1C35
:10FB700010FA03F3B1F9000007E02C781C40DE43D3
:10FB8000164034432C70401C6D1CB1F90440844273
:10FB9000F3DAF0BD10B4C1F3074244F6CD43C1F32C
:10FBA000072449F20A70444303FB024201F0FF01BB
:10FBB00041F6294000FB0121C90D080010BC704727
:10FBC00080B500F076F801BD10B56A4C0022012125
:10FBD0002000FFF761FB012201212000FFF75CFB01
:10FBE000A02000F09FF8C82000F09CF8812000F0D1
:10FBF00099F81F2000F096F82F2000F093F840208D
:10FC000000F090F8A62000F08DF8AF2000F08AF800
:10FC100010BD7CB5584C00F0FDFB2060574800F04B
:10FC20005BFB574800F058FB564800F055FB564820
:10FC300056490860FF2056490860564D28000CF0D0
:10FC400091FC5548FFF762FB5448FFF75FFB494EB4
:10FC500006213000FFF742FB01213000FFF72CFBAB
:10FC60004F4E04213000FFF727FB08213000FFF73B
:10FC700023FB082001904B480090002303222168B9
:10FC800028000CF047FC28000CF066FC042204213C
:10FC90003000FFF701FB082208213000FFF7FCFAD3
:10FCA00020686421B0FBF1F000F03CFBFFF78CFF13
:10FCB00073BD2DE9F041441D002516E0354F380095
:10FCC0000CF071FC0028F9D1217838000CF050FCC0
:10FCD000641C761C802EF1D3092000F023FB042243
:10FCE00004214046FFF7D8FA6D1C082D18D255F0B4
:10FCF000B000C0B200F016F8102000F013F8002099
:10FD000000F010F8DFF89880002204214046FFF749
:10FD1000C3FA082208214046FFF7BEFA0026D9E7B9
:10FD2000BDE8F08170B504001D4D002208212800B7
:10FD3000FFF7B2FA002204212800FFF7ADFA154EB2
:10FD400030000CF030FC0028F9D1E4B22100300082
:10FD50000CF00EFC30000CF026FC0028FAD1042236
:10FD600004212800FFF798FA082208212800FFF74D
:10FD700093FA70BD005002401C110020011C00F0DD
:10FD8000010800F0050800F04B434F4C205502409D
:10FD900024550240009000400204050002080500BE
:10FDA00000500040002D3101FEB504460D461746B7
:10FDB000002657B302AB3A462946204600F08EF89B
:10FDC00018B30146A06901AA00F0EDF9B0B9A06925
:10FDD00001AA2E2100F0E7F980B9A06901AA20212B
:10FDE00000F0E1F950B90DF1060000900DF10703A4
:10FDF000A06901AA0DF1050100F0A8F99DF8040021
:10FE00003618029805443F1AD3E73046FEBD30B598
:10FE100083B0069C079D05B10125EDB200940195C4
:10FE2000C469A04737BD2DE9F041054686B003A857
:10FE300000900F46144698460C9EA8690DF10903E0
:10FE40000DF10A020DF10B0100F080F9B5F90E1069
:10FE5000B142A1BF9DF809003018B5F90A108842D7
:10FE600039DB0D988DF834002CE09DF80A0025E070
:10FE7000B5F90C1088452EDA0146A86902AA00F0EF
:10FE800092F950B9A86902AA2E2100F08CF920B984
:10FE9000A86902AA202100F086F90028E5D00D9972
:10FEA0009DF80B20019102F00102009201463346B9
:10FEB0004246284600F027F89DF808008044049840
:10FEC0000744241A3CB104AB22463946284600F0C8
:10FED00005F80028CCD106B0BDE8F08138B504465D
:10FEE000084611001A4601D1002032BD54F8203FC7
:10FEF0002BB1E47903EBC4035D68A84732BD01214F
:10FF00001160007832BD2DE9FC4F064683B0B6F98A
:10FF10000C00904216DB10464A788018B6F908208B
:10FF200090420FDB4FF00009CB460227D84600E095
:10FF300001990878874280F2E480049AB6F90E00AD
:10FF400042449042C0F2DD800E98C0B900250A7884
:10FF5000974213DAC85D0BF118029040B0FA80FAAC
:10FF6000BAF1080FC8BFCBF1080AD344BBF1080FA0
:10FF7000554404BF4FF0000B7F1CE8D0C4E0CC5DBB
:10FF80002CB1250904F00F047F1C01912BE0C81946
:10FF9000BF1C4078C5000006F7D505F47E740191BA
:10FFA0007AE0B6F908108C45A1BFB6F90C1061458E
:10FFB000B6F90A1088420CDB0F9951B17168736968
:10FFC00001F1040E02466146DEF80000DEF808C0CA
:10FFD000E0476D1ED14601984178894504BF08F17C
:10FFE00001084FF00009002D56D000F0A9F853DBAE
:10FFF000DDF80CC0012DCC4409F1010AD1DD0199D5
:020000040001F9
:1000000049788A45CDDA05EB09029142B4BFA1EBEC
:10001000090AAA46B6F90A10884219DB0F99B9B144
:10002000B6F9082061469445B8BF1146B6F90C20D0
:10003000D444ACF101039A42C8BF1A46D6F804C0B2
:10004000736900930346DCF80400DCF814C0E04751
:10005000A5EB0A05D144BEE7B6F908108C45A1BF4F
:10006000B6F90C106145B6F90A1088420ADB7168CE
:10007000336901F1040E02466146DEF80000DEF845
:1000800008C0E047641EA94601984178894504BF2D
:1000900008F101084FF00009002C3FF449AF00F0CF
:1000A0004FF8FFF645AFDDF80CC0012CCC4409F148
:1000B0000105D1DD01994A789542CDDA04EB0901B9
:1000C0008A42B6F90A10B4BFA2EB090AA2468842D6
:1000D00013DBB6F90810B6F90C2075688C45A8BF7B
:1000E0006146D444ACF101039A42C8BF1A46336951
:1000F0000093034668686D69A847A4EB0A04D144DD
:10010000C2E705B0BDE8F08F0024019101980178A5
:100110008F4214DAC05D0BF118018840C043B0FA79
:1001200080FABAF1080FC8BFCBF1080AD344BBF17B
:10013000080F544404BF4FF0000B7F1CE6D052E779
:100140000498B6F90E1040448142704770B582B0F1
:10015000044625780698AE0605D500906068A46828
:100160002568A84773BD0D7061781170A17819706A
:10017000E178017073BD30B5044683B02078202843
:1001800001D0E0783EBD01A800900DF10503FFE726
:100190006068A46825680DF106020DF10701A84703
:1001A0009DF804003EBDF8B503461878202804D118
:1001B00058689B685C68A047F2BD400618D50020CF
:1001C000DD880C244443A8421C442BD2A668B142CB
:1001D00003D3E768BE19B14224D3401CF0E720697D
:1001E0000344A068091A53F82100D0B1184414E060
:1001F0001878040604D5D8689C681D795B7904E0FA
:10020000D3F8C4001C1D20257E23A94228BF8B42A1
:1002100006D3491B34F81110084441781170F2BD1F
:100220000020F2BDA842DAD1FAE70146087842067A
:1002300001D588887047800603D5486889688A6830
:10024000104700207047F8B50446A069C8B1FFF711
:10025000ECFF04F1260201461378256A002000E035
:10026000401C98420BD235F83060A78CBE4202BFCA
:1002700005EBC00677888F42F2D15070F2BD0020A6
:1002800050704FF0FF30F2BD8161DCE700220CF0CE
:1002900099B9000018B58100DFF88022C0F3072368
:1002A00001F47F71D31841EA431343F084430124DE
:1002B0001C600023009302E0009C641C0094009BDF
:1002C000102BF9D3C0F30720121841EA421141F074
:1002D00084410020086011BDC0F30722DFF84012FE
:1002E00080008A1800F47F7040EA421040F0844099
:1002F000012101607047C0F30722DFF8241280005B
:100300008A1800F47F7040EA421040F084400021D7
:1003100001607047DFF80C1208B188687047086800
:10032000704700000138FDD170477047DFF8F811C1
:100330000860704770B5DFF8EC211469136A014654
:1003400024F4800401F0010544F4006404F0010089
:1003500085F0010543F400631461284213620ED056
:1003600061F0010004404FF48070906014614FF41C
:1003700000201568EE054AD4401EFAD170BD080968
:1003800060F30A14DFF8B00114610340DFF8AC0138
:1003900008400343C80000F0400003431362480BC9
:1003A00060F34D3460F34D3340209060002B47BF25
:1003B0001362146114611362DFF884010440DFF8F2
:1003C000840108400443C80D60F3DC53480008D59D
:1003D000DFF8740123F48003084044F480040343ED
:1003E00001E023F0804308050BD44FF40040574947
:1003F0000D68EE0701D4401EFAD124F4006423F402
:100400000063146113621020BDE870408AE7002881
:10041000B5D170BDF0B54E490A6D0B6E002B4CBFC7
:1004200003F0700002F0300040B1102847D02028BF
:1004300047D0302847D0702848D04AE00FF22C101F
:10044000C2F3841450F82450424C04EA0306B6F177
:10045000004F4FF0FF3003D0002B41D416053FD49E
:10046000334E376876680968C6F3042C06F01F0619
:100470000CF1010C761C16FB0CF67600B5FBF6F5BC
:10048000C7F30906C7F389276F4301F47041BF0A18
:10049000B1F5005F06FB057542F480020DD0B1F5A1
:1004A000405F18D0B1F5804F17D0B1F5E04F16D0AE
:1004B000B1F5104F08BF284812E0284810E01B4D46
:1004C000C2E7274DC0E747F23055BDE74FF400457E
:1004D000BAE70020F0BD234802E0234800E01548B9
:1004E000510217D5002B10D559000BD51C40B4F183
:1004F000004F03D0002B05D4110503D46D00C3F3C6
:10050000865104E0C3F3C55101E0C2F3C351491C55
:10051000B5FBF1F5A84288BF2846F0BD00E50F40C5
:1005200000E60F4050E00F407CE00F400024F40054
:1005300060E10F4040787D018FFFFF7F3000008039
:10054000FEFF3FF80100C0070000404068E10F4097
:1005500010E00F4000080080002D310100B4C404F9
:1005600000093D0080F0FA02005A620240420F008A
:1005700000201C0080841E0000802500999E36000B
:100580000040380000093D0000803E0000004B00A4
:10059000404B4C0000204E00808D5B0000C05D0091
:1005A0000080700000127A0000007D0080969800A4
:1005B000001BB7000080BB00C0E8CE00647ADA0000
:1005C0000024F4000000FA0080A81201002D31017F
:1005D00000366E0140787D014D49FFE7012008603B
:1005E0007047012100F01F0001FA00F0494908603E
:1005F0007047012100F01F0001FA00F04649086031
:10060000704746490860704700F01F00012202FA57
:1006100000F081B0424ACB0748BF10608B0748BF4B
:1006200090614B0748BF1062090748BF906001B056
:1006300070473A4A126800F03F0002EB0012394856
:1006400093680340194391607047F0B5334C2568B7
:10065000354C00F03F0005EB0016B76827408406D4
:1006600004D5042914BF062941F00101DDF814C0A6
:10067000ACF1010E41EA0E14274307F04064B4F1D7
:10068000406F04D0A40E0CFA04F4A218521E32607B
:1006900007F04042B2F1404F0FD0042918BF06299D
:1006A00006D140F0200005EB001000F10C0304E03F
:1006B000920F0CFA02F003445B1E7360B760F0BD4A
:1006C0001649096800F03F0001EB0010806800F057
:1006D00007004108490004291EBF42085200062AAB
:1006E00004BF40084000704700F0FF0110B5CB0880
:1006F0000E4A02EB8302890001F01C0113680F24EB
:100700008C40000CA34388401843106010BD0000CB
:1007100004F00F4028F00F402CF00F4008F00F407D
:100720001CF00F40F73FFC0008C0FFFF10F50F4022
:10073000114340F8341F7047F8B504460E4617467B
:100740001D4600F035F8B6EB071F04F1300005D266
:10075000016841F0200101607F0803E0026822F097
:1007600020020260F600B6FBF7F0401C400804F1DE
:1007700024028109116000F03F0004F128010860A3
:1007800004F12C0004F118010560002008602046E7
:10079000BDE8F240FFE700F12C010A6842F01002C8
:1007A0000A6040F2013150F8303F0B43036070475C
:1007B00081B000F118010A681307FCD400F12C0184
:1007C0000A6822F010020A6050F8303F02490B40DC
:1007D000036001B070470000FEFCFFFF11430160A1
:1007E000704750F8302F22F01002F7E7002914BFAD
:1007F00040303C300068704740F8441F704750F864
:10080000482FEBE780B50BF011FF02E080B50BF04D
:1008100009FF00B10120C0B202BD10B50FF2D40231
:10082000830852F823201368C00000F01800FF244A
:100830008440A34381401943116010BD04282B4913
:1008400003D1086840F480300BE0052804D10A6821
:1008500042F400320A607047062804D1086840F468
:100860008020086070470F2805D12148016841F0B9
:100870000201016070470CD90FF21413A0F11001AE
:100880001038400953F82000012201F01F018A406E
:10089000026070470428154903D1086820F48030AD
:1008A0000BE0052804D10A6822F400320A60704780
:1008B000062804D1086820F48020086070470F28BB
:1008C00005D10B48016821F00201016070470CD985
:1008D0000FF2D003A0F110011038400953F82000A6
:1008E000012201F01F018A400260704724ED00E000
:1008F00010E000E00000000018ED00E01CED00E05A
:1009000020ED00E000E400E004E400E008E400E0A2
:100910000CE400E010E400E014E400E018E400E07F
:100920001CE400E020E400E024E400E028E400E02F
:100930002CE400E030E400E034E400E038E400E0DF
:100940003CE400E040E400E044E400E048E400E08F
:100950004CE400E050E400E054E400E058E400E03F
:100960005CE400E060E400E064E400E068E400E0EF
:100970006CE400E070E400E074E400E078E400E09F
:100980007CE400E080E400E084E400E088E400E04F
:1009900000E100E004E100E008E100E00CE100E03B
:1009A00010E100E080E100E084E100E088E100E0A7
:1009B0008CE100E090E100E01BE050F8081F41F0FE
:1009C00002010160704700F540600121016070473D
:1009D00000F54060014901607047000051E5CC1A04
:1009E00000F540600068012818BF002070470160D2
:1009F000704750F8081F41F001010160704700F591
:100A00008360016841F480710160704702480168A9
:100A100041F040410160704734EF00E00748016851
:100A200041F00501016070470448016841F002018E
:100A3000016070470249401E0860704710E000E006
:100A400014E000E010B504000020FBF768F8FCF7A4
:100A5000C9FBA169401A40F6B931884214D3FCF7AA
:100A600029F8002810D0002060615FF0FF30FCF70B
:100A70001EF9002804D003210720FAF79EFD03E0A9
:100A800003210120FAF799FD10BD000030B59BB09D
:100A9000040040F25A200021F9F769FAFCF716F831
:100AA000002804D15FF480100021F9F760FAFCF708
:100AB00001F8062805D1162209A90620FCF78AF8B4
:100AC00025E0FBF7F7FF04281BD11E20FBF765FF8D
:100AD000162215A9FCF77EF84FF40070FBF74EFFC5
:100AE000002807D015ABDFF8CC29162109A8FAF7A2
:100AF00070FC0CE015AB95A2162109A8FAF769FC69
:100B000005E0DFF8B429162109A8FAF762FCFCF722
:100B100069FBDFF8A8592968401A40F2F5118842AC
:100B20000CD3FCF75FFB2860DFF89409016801290A
:100B300002D10021016001E0012101605FF4800029
:100B40000021FDF71BFB00220023994201D19042B6
:100B500012D0DFF86C090068002805D17CA21621AC
:100B600001A8FAF736FC99E0DFF8583977A2162188
:100B700001A8FAF72EFC91E0FDF7EAFA002816D05A
:100B8000DFF83C090068002805D171A2162101A8F0
:100B9000FAF71FFC82E0FDF7DBFA0090DFF8283956
:100BA000DFF82829162101A8FAF713FC76E0FDF7F3
:100BB00057F9002818D0DFF808090068002805D187
:100BC00063A2162101A8FAF704FC67E0FDF748F9D3
:100BD000FCF7FEFB0090DFF8F038DFF8F428162170
:100BE00001A8FAF7F6FB59E04FF480400021FDF729
:100BF000C5FA00220023994201D1904211D0DFF8BA
:100C0000C0080068002805D151A2162101A8FAF7F2
:100C1000E0FB43E01622DFF8BC1801A8FAF77EFAE1
:100C20003CE008200021FDF7A9FA002200239942A8
:100C300001D1904211D0DFF888080068002805D162
:100C400043A2162101A8FAF7C4FB27E01622DFF819
:100C5000881801A8FAF762FA20E05FF4003000215A
:100C6000FDF78CFA00220023994201D1904211D065
:100C7000DFF84C080068002805D135A2162101A82C
:100C8000FAF7A7FB0AE01622DFF8501801A8FAF7D6
:100C900045FA03E0162101A8FDF7BAF9FCF7E7FFD2
:100CA000802806DBDFF8382816210FA8FAF791FB19
:100CB00003E016210FA8FCF788FF0020FDF7A4F938
:100CC00005000120FDF7A0F903000095DFF81428C6
:100CD000062107A8FAF77DFB0025FBF710FF002887
:100CE0000DD1DFF804080021FDF748FA00220023A7
:100CF000994201D1904202D055F0010510E0FBF776
:100D0000FEFE01280CD1DFF8E0070021FDF736FADE
:100D100000220023994201D1904201D055F00105F3
:100D20005FF080500021FDF729FA0022002399424C
:100D300001D1904201D055F002056068012802D02F
:100D4000E068012806D155F0040508E0257300008D
:100D500000000000A068012801D155F0080501201D
:100D6000FAF7DDFE09A90C20FAF70EFF01A90A2007
:100D7000FAF70AFF0FA90920FAF706FF07A90B20C7
:100D8000FAF702FF2800FAF7CEFE5620FBF705FE21
:100D9000800712D4FBF744FE01280ED14020FCF757
:100DA000B9FE002809D02020FCF7A9FE4020FCF75E
:100DB000A6FE00200121F9F7DAF86068002840F06B
:100DC0000B810120FAF7AEFD00282AD00820FAF79F
:100DD000A9FD002825D00420FAF7A4FD002820D181
:100DE0000220FAF79FFD00281BD1FCF7FBF9E06118
:100DF000FCF7F8F9A169401A41F289318842C0F044
:100E0000EB80FCF7EFF9A0610120DFF8E016086045
:100E1000E068012802D10020E060DDE00120E06010
:100E2000DAE00420FAF77EFD002825D00220FAF748
:100E300079FD002820D00120FAF774FD00281BD18D
:100E40000820FAF76FFD002816D1FCF7CBF9A06156
:100E5000FCF7C8F9E169401A40F6B9318842C0F0A0
:100E6000BB80FCF7BFF9E0610120FCF72DFF0020FB
:100E70008021F9F77CF8AFE0FCF7B4F9A061FCF74A
:100E8000B1F9E061E068002840F098800420FAF7AA
:100E900053FD00281FD0FBF732FE002808D1FBF7D6
:100EA00015FE012804D101210E20FAF786FB85E00A
:100EB000A068012806D103210820FAF77EFB002054
:100EC00020617BE001210820FAF777FB0121022055
:100ED000FAF773FB72E00820FAF72EFD00280ED017
:100EE000DFF808060068002809D10220FCF712FE8E
:100EF000002804D101210620FAF75FFB5EE0012003
:100F0000FAF71AFD00282FD0DFF8E0050068002866
:100F10002AD10220FCF7FEFD00284FD1A06801284D
:100F200008D0FBF7ECFD002804D00120FCF7F2FD0F
:100F3000002810D00120FCF7EDFD002803D001208F
:100F4000FCF7DDFD02E00120FCF7CFFD00200121D0
:100F5000F9F70DF832E003210420FAF72EFB012106
:100F60000220FAF72AFB29E00220FAF7E5FC002824
:100F700024D0A068012808D0FBF7C1FD002804D0C8
:100F80000220FCF7C7FD002810D00220FCF7C2FDAC
:100F9000002803D00220FCF7B2FD02E00220FCF79B
:100FA000A4FD00200121F8F7E2FF07E0032105205E
:100FB000FAF703FB01210220FAF7FFFA0820FAF7FB
:100FC000B1FC002808D10120FAF7ACFC002803D1BD
:100FD0000020DFF8181508601BB030BD10B586B0D2
:100FE00042200021F8F7C3FF1622DFF804156846F7
:100FF000FAF794F869460020FAF7C6FD162168460C
:10100000FCF7E3FD0220FAF78AFD69460920FAF7AA
:10101000BBFD5620FBF7C1FC800712D4FBF700FD97
:1010200001280ED14020FCF775FD002809D02020B2
:10103000FCF765FD4020FCF762FD00200121F8F778
:1010400096FF0120FAF778FC00284BD00120FCF72E
:1010500061FD002840F02B81FBF751FD012810D1E4
:101060002020FCF757FD002803D02020FCF747FD87
:1010700002E02020FCF739FD00200121F8F777FF7E
:1010800026E04020FCF746FD002815D1DFF8640477
:10109000006801281CD02020FCF73CFD002803D06C
:1010A0002020FCF72CFD02E02020FCF71EFD002094
:1010B0000121F8F75CFF0BE0DFF838040068012835
:1010C00006D04020FCF71BFD00200121F8F74FFF60
:1010D000FCF788F8DFF8201408600020DFF814140B
:1010E0000860E4E00120FAF71DFC00284ED05620ED
:1010F000FBF753FC80073FD5FBF792FC01283BD15F
:101100005720FBF74AFC012836D1DFF8E843206876
:10111000002840F0CC80FCF765F8DFF8DC130968A4
:10112000401A40F6B9318842C0F0C18001202060E9
:101130004020FCF7EFFC002813D14020FCF7D5FC41
:101140000820FCF7E7FC00280ED01020FCF7E2FC9A
:10115000002809D00820FCF7D2FC1020FCF7CFFCB7
:1011600002E04020FCF7CBFC2020FCF7C8FC00206C
:101170000121F8F7FCFE9AE00020DFF87813086000
:10118000FCF730F8DFF87013086090E00220FAF7FF
:10119000D3FB002864D00120FCF7BCFC002840F001
:1011A00086802020FCF7B6FC002840F08080FBF70A
:1011B000A6FC01280FD10820FCF7ACFC002803D1C5
:1011C0000820FCF792FC02E00820FCF798FC1020B5
:1011D000FCF795FC3FE00820FCF79CFC00280BD1B5
:1011E0001020FCF797FC002806D10820FCF77DFCB6
:1011F0001020FCF784FC2EE00820FCF78BFC002874
:101200000BD01020FCF786FC002806D01020FCF73D
:1012100076FC0820FCF773FC1DE00820FCF77AFC44
:10122000002806D01020FCF760FC0820FCF767FCC3
:1012300011E04020FCF76EFC002806D11020FCF7DE
:1012400054FC0820FCF751FC05E01020FCF757FC8B
:101250000820FCF754FC00200121F8F788FE26E066
:101260000420FAF769FB002810D00420FCF752FC98
:10127000002803D00420FCF742FC02E00420FCF725
:1012800034FC00200121F8F772FE10E00820FAF784
:1012900053FB002807D003210120FAF78EF9002024
:1012A0009449086003E0FBF79DFF9349086006B08E
:1012B00010BD10B586B078200021F8F758FE162230
:1012C00069460620FBF786FC69460020FAF75CFCBD
:1012D0000420FAF724FC0120FAF779FC162287494A
:1012E0006846F9F71BFF69460120FAF74DFC70A428
:1012F00021000220FAF748FC21000320FAF744FC01
:1013000021000420FAF740FC21000520FAF73CFCFC
:1013100021000620FAF738FC21000720FAF734FCF8
:1013200021000820FAF730FC0020FAF7FCFB082027
:10133000FAF702FB002801D0FAF797F906B010BDC2
:1013400030B587B0040002200021F8F710FE162205
:101350006B4901A8F9F7E2FE01A90020FAF714FC95
:10136000FBF7A9FC0090584B664A162101A8FAF732
:1013700030F80420FAF7D3FB0020FAF728FC01A983
:101380000120FAF701FC0020FAF7CDFB48A529005F
:101390000220FAF7F9FB29000320FAF7F5FB2900F0
:1013A0000420FAF7F1FB29000520FAF7EDFB2900EC
:1013B0000620FAF7E9FB29000720FAF7E5FB2900E8
:1013C0000820FAF7E1FB0420FAF7ACFA002810D065
:1013D0000220FAF7A7FA00280BD00120FAF7A2FAA8
:1013E000002806D10820FAF79DFA002801D1FBF762
:1013F00002FFFBF7F7FEA169401A41F289318842EA
:101400000BD31020FBF753FC002806D12020FBF75C
:101410004EFC002801D1FBF7EEFE07B030BD10B541
:1014200092B0162238490CA8F9F778FE1622254901
:1014300006A8F9F773FE354A16216846F9F7C9FF81
:101440000420FAF76CFB0120FAF7C1FB0CA900207D
:10145000FAF79AFB06A90120FAF796FB69460520E0
:10146000FAF792FB12A421000220FAF78DFB21006B
:101470000320FAF789FB21000420FAF785FB2100FD
:101480000620FAF781FB21000720FAF77DFB2100F7
:101490000820FAF779FB0020FAF745FB0820FAF755
:1014A0004BFA002801D0FAF7E0F812B010BD0000A6
:1014B00000000000B0EC0100B8EC01005811002061
:1014C0005411002040F7030020E50300C8E80100A4
:1014D000D4E8010020E30300A0E1030060F0030072
:1014E000C0EC0100E0E80100299E3F6C5C11002087
:1014F00020EC0300601100206411002080F0030044
:1015000000D00300C8EC0100C0D90300D0EC0100FA
:10151000F0B5BDB0040058200021F8F728FD1622D0
:10152000AA496846F9F7FAFD69460020FAF72CFB4C
:101530000320FAF7F4FA0420FAF749FBA44BA54A72
:10154000162106A8F9F745FFA34BA44A16210DF171
:101550002E00F9F73EFFA24BA24A162111A8F9F777
:1015600038FFA14BA14A16210DF15A00F9F731FFBE
:101570005720FBF712FA012828D19D4B9D4A1621CE
:101580001CA8F9F726FF9C4B9C4A16210DF18600FA
:10159000F9F71FFF9A4B9B4A162127A8F9F719FF65
:1015A000994B9A4A16210DF1B200F9F712FF984BA8
:1015B000984A162132A8F9F70CFF974B974A162143
:1015C0000DF1DE00F9F705FF0A2526E08A4B894A6E
:1015D00016211CA8F9F7FDFE894B884A16210DF14A
:1015E0008600F9F7F6FE884B864A162127A8F9F7F8
:1015F000F0FE874B854A16210DF1B200F9F7E9FE9E
:10160000854B844A162132A8F9F7E3FE6EA2162113
:101610000DF1DE00F9F7DDFE09252800F9F764FF7A
:101620000020F9F790FF401CFAF77DFA0220F9F745
:101630008AFF0600162706A807FB06F101440120D1
:10164000FAF7A2FA06A807FB06F1084410F1160102
:101650000220FAF799FA06A807FB06F1084410F1F0
:101660002C010320FAF790FA06A87E43304410F1CB
:1016700042010420FAF788FA0820FAF75DF90028F9
:1016800000F092800120F9F75EFF002809D10121C6
:101690003A20F9F792FF0BF07BF82063206BE063B0
:1016A0008FE0012813D1A068012802D0206900280A
:1016B00008D101212020F9F780FF01210220F9F74C
:1016C0007CFF7EE001212020F9F777FF79E00228F6
:1016D00018D1FBF714FA012804D101210A20F9F7E7
:1016E0006CFF6EE04FF40070FBF748F9002804D05F
:1016F00001210A20F9F761FF63E001210920F9F7D0
:101700005CFF5EE0032804D101210D20F9F755FFAD
:1017100057E004280BD10A2D04D001211620F9F737
:101720004CFF4EE001218120F9F747FF49E00528F1
:101730000BD10A2D04D001211C20F9F73EFF40E017
:1017400001211620F9F739FF3BE006280BD10A2DBD
:1017500004D001213020F9F730FF32E001211C20B4
:10176000F9F72BFF2DE007280BD10A2D04D001211A
:101770008C20F9F722FF24E001213020F9F71DFF2A
:101780001FE008280BD10A2D04D001218D20F9F784
:1017900014FF16E001218C20F9F70FFF11E0012161
:1017A0008D20F9F70AFF0CE00120FAF7C5F80028B0
:1017B00004D003210120F9F700FF02E02800F9F727
:1017C0006CFF3DB0F0BD00BF00000000C0D90300B9
:1017D00020D2030060EC010040D2030068EC01005D
:1017E00060D2030070EC010080D2030078EC0100AD
:1017F00020F1030080EC0100A0D2030088EC01007E
:10180000C0D2030090EC0100E0D2030098EC01008C
:1018100000D30300A0EC010020D30300A8EC0100DA
:1018200030B591B0040002200021F8F7A0FB02209F
:10183000F9F75AFE1622DFF8581C6846F9F76EFCD5
:1018400069460020FAF7A0F90320FAF768F90420A6
:10185000FAF7BDF9DFF83C3CDFF83C2C162106A86E
:10186000F9F7B7FDDFF8343CDFF8342C16210DF121
:101870002E00F9F7AEFD06A90120FAF785F90DF162
:101880002E010220FAF780F97BA529000320FAF740
:101890007BF929000420FAF777F90020F9F753FEC5
:1018A000401CFAF740F90820FAF746F8002815D04E
:1018B0000120F9F748FE00280BD101211020F9F78B
:1018C0007CFE2069002814D101210220F9F775FE61
:1018D0000FE001211120F9F770FE0AE00120FAF76C
:1018E0002BF8002802D0F9F7C0FE02E00220F9F739
:1018F000D4FE11B030BD30B587B005000220002104
:10190000F8F735FB1622DFF89C1B01A8F9F706FC57
:1019100001A90020FAF738F90420FAF700F90420A9
:10192000FAF755F9B3A421000120FAF72DF92100A7
:101930000220FAF729F921000320FAF725F92100FE
:101940000420FAF721F94CA421000520FAF71CF92C
:1019500021000620FAF718F921000720FAF714F9F8
:1019600021000820FAF710F90020FAF7DCF8E86AFD
:10197000284490F820008DF8000000208DF8010028
:10198000E86A012804D169460120FAF7FDF816E05B
:10199000E86A022804D169460220FAF7F5F80EE059
:1019A000E86A032804D169460320FAF7EDF806E057
:1019B000E86A042803D169460420FAF7E5F8EC6ADE
:1019C0000220F9F7B4FF00281BD0002C03D1E86AED
:1019D000401CE8624DE005EB040090F82000392837
:1019E00009DA05EB040090F82000401C05EB040127
:1019F00081F820003DE0302005EB040181F8200053
:101A000037E00420F9F793FF00281BD0002C03D106
:101A1000E86A401CE8622CE005EB040090F8200026
:101A2000312809DB05EB040090F82000401E05EB8F
:101A3000040181F820001CE0392005EB040181F845
:101A4000200016E00820F9F777FF00280AD0042CC0
:101A500004D102211220F9F7B0FD0AE0E86A401C27
:101A6000E86206E00120F9F767FF002801D0F9F7E6
:101A7000FCFD07B030BD00000000000030B587B0AD
:101A8000050002200021F8F772FA1622DFF81C1A6E
:101A900001A8F9F743FB01A90020FAF775F8042023
:101AA000FAF73DF80420FAF792F852A42100012039
:101AB000FAF76AF821000220FAF766F821000320FD
:101AC000FAF762F821000420FAF75EF8BEA42100BC
:101AD0000520FAF759F821000620FAF755F82100F9
:101AE0000720FAF751F821000820FAF74DF80020F6
:101AF000FAF719F8EC6A05EB040090F820008DF86D
:101B0000000000208DF80100012C04D1694601205D
:101B1000FAF73AF813E0022C04D169460220FAF7EA
:101B200033F80CE0032C04D169460320FAF72CF8B3
:101B300005E0042C03D169460420FAF725F80220B9
:101B4000F9F7F5FE00281BD0002C03D1E86A401CF1
:101B5000E8624DE005EB040090F82000392809DA2E
:101B600005EB040090F82000401C05EB040181F80F
:101B700020003DE0302005EB040181F8200037E033
:101B80000420F9F7D4FE00281BD0002C03D1E86A0A
:101B9000401CE8622CE005EB040090F8200031289E
:101BA00009DB05EB040090F82000401E05EB040162
:101BB00081F820001CE0392005EB040181F82000A9
:101BC00016E00820F9F7B8FE00280AD0042C04D14A
:101BD00002211320F9F7F1FC0AE0E86A401CE862F0
:101BE00006E00120F9F7A8FE002801D0F9F73DFD35
:101BF00007B030BD2A00000030B587B005000220D4
:101C00000021F8F7B4F91622DFF8A41801A8F9F7B3
:101C100085FA01A90020F9F7B7FF0420F9F77FFF43
:101C20000420F9F7D4FF69A421000120F9F7ACFFE3
:101C300021000220F9F7A8FF21000320F9F7A4FFF3
:101C400021000420F9F7A0FF5FA421000520F9F787
:101C50009BFF21000620F9F797FF21000720F9F7E5
:101C600093FF21000820F9F78FFF0020F9F75BFFB1
:101C7000EC6A05EB040090F825008DF800000020C8
:101C80008DF80100012C04D169460120F9F77CFF91
:101C900013E0022C04D169460220F9F775FF0CE02D
:101CA000032C04D169460320F9F76EFF05E0042CEC
:101CB00003D169460420F9F767FF0220F9F737FEE0
:101CC00000281BD0002C03D1E86A401CE86279E0B0
:101CD00005EB040090F82500392809DA05EB04002B
:101CE00090F82500401C05EB040181F8250069E00F
:101CF000302005EB040181F8250063E00420F9F7AA
:101D000016FE00281BD0002C03D1E86A401CE862B4
:101D100058E005EB040090F82500312809DB05EBBD
:101D2000040090F82500401E05EB040181F8250011
:101D300048E0392005EB040181F8250042E0082045
:101D4000F9F7FAFD002836D0042C30D195F826009A
:101D500095F82110884225D195F8270095F8221092
:101D600088421FD195F8280095F82310884219D190
:101D700095F8290095F82410884213D102211420E7
:101D8000F9F71BFC95F8293095F8282095F82710CD
:101D900095F82600FBF72EFE00204FF48071F8F72F
:101DA000E6F80FE002211220F9F707FC0AE0E86AE2
:101DB000401CE86206E00120F9F7BEFD002801D0D2
:101DC000F9F753FC07B030BD000000002A00000006
:101DD00030B587B0050002200021F8F7C8F81622B8
:101DE000DFF8D01601A8F9F799F901A90020F9F751
:101DF000CBFE0420F9F793FE0420F9F7E8FEA3A434
:101E000021000120F9F7C0FE21000220F9F7BCFEF5
:101E100021000320F9F7B8FE21000420F9F7B4FEF1
:101E20009BA421000520F9F7AFFE21000620F9F759
:101E3000ABFE21000720F9F7A7FE21000820F9F7E3
:101E4000A3FE0020F9F76FFEEC6A05EB040090F8A2
:101E500025008DF8000000208DF80100012C04D130
:101E600069460120F9F790FE13E0022C04D169467F
:101E70000220F9F789FE0CE0032C04D16946032007
:101E8000F9F782FE05E0042C03D169460420F9F736
:101E90007BFE0220F9F74BFD00281BD0002C03D15C
:101EA000E86A401CE86279E005EB040090F8250040
:101EB000392809DA05EB040090F82500401C05EBF1
:101EC000040181F8250069E0302005EB040181F868
:101ED000250063E00420F9F72AFD00281BD0002C20
:101EE00003D1E86A401CE86258E005EB040090F872
:101EF0002500312809DB05EB040090F82500401E81
:101F000005EB040181F8250048E0392005EB0401C8
:101F100081F8250042E00820F9F70EFD002836D0B0
:101F2000042C30D195F8260095F82110884225D14F
:101F300095F8270095F8221088421FD195F82800BF
:101F400095F82310884219D195F8290095F82410A6
:101F5000884213D102211520F9F72FFB95F829307B
:101F600095F8282095F8271095F82600FBF765FDD1
:101F700000204FF40071F7F7FAFF0FE00221132061
:101F8000F9F71BFB0AE0E86A401CE86206E0012062
:101F9000F9F7D2FC002801D0F9F767FB07B030BD94
:101FA00010B586B002200021F7F7E1FF0420F9F711
:101FB000B6FD1622DFF8EC146846F9F7AFF869466B
:101FC0000020F9F7E1FD0020FBF751FD040000209F
:101FD000FBF746FDE4B2844224D10120FBF747FD24
:101FE00004000120FBF73CFDE4B284421AD1022038
:101FF000FBF73DFD04000220FBF732FDE4B2844212
:1020000010D10320FBF733FD04000320FBF728FD6C
:10201000E4B2844206D11622DFF89C146846F9F730
:102020007DF805E01622DFF894146846F9F776F893
:1020300069460120F9F7A8FD15A421000220F9F74F
:10204000A3FD21000320F9F79FFD21000420F9F7EB
:102050009BFD21000520F9F797FD21000620F9F7E7
:1020600093FD21000720F9F78FFD21000820F9F7E3
:102070008BFD0120F9F7ABFD0820F9F75DFC002886
:1020800001D0F9F7F2FA06B010BD00002A000000F6
:102090000000000010B586B002200021F7F767FFAE
:1020A0000420F9F73CFD1622DFF800146846F9F722
:1020B00035F869460020F9F767FD0020FBF7D7FCEB
:1020C00004000020FBF7CCFCE4B2844224D10120C0
:1020D000FBF7CDFC04000120FBF7C2FCE4B2844214
:1020E0001AD10220FBF7C3FC04000220FBF7B8FC66
:1020F000E4B2844210D10320FBF7B9FC04000320B2
:10210000FBF7AEFCE4B2844206D11622DFF8A81336
:102110006846F9F703F805E01622DFF8A0136846D1
:10212000F8F7FCFF69460120F9F72EFDB0A4210065
:102130000220F9F729FD21000320F9F725FD2100F0
:102140000420F9F721FD21000520F9F71DFD2100EC
:102150000620F9F719FD21000720F9F715FD2100E8
:102160000820F9F711FD0120F9F731FD0820F9F7F2
:10217000E3FB002801D0F9F778FA06B010BD78B576
:1021800087B00600F9F782FA050002200021F7F770
:10219000EEFE0420F9F7C3FC042D03D0052D01D079
:1021A000082D05D11622C64901A8F8F7B7FF04E0AB
:1021B0001622B84901A8F8F7B1FF01A90020F9F7E4
:1021C000E3FC0420F9F703FDB0A421000120F9F796
:1021D000DBFC21000220F9F7D7FC21000320F9F7EE
:1021E000D3FC21000420F9F7CFFC81A421000520B5
:1021F000F9F7CAFC21000620F9F7C6FC21000720E8
:10220000F9F7C2FC21000820F9F7BEFC0020F9F71D
:102210008AFCF46A06EB040090F820008DF80400B4
:1022200000208DF80500012C04D101A90120F9F747
:10223000ABFC13E0022C04D101A90220F9F7A4FCA5
:102240000CE0032C04D101A90320F9F79DFC05E063
:10225000042C03D101A90420F9F796FC0220F9F718
:1022600066FB00281ED0002C07D1F06A401CF062EB
:10227000F16A0020F9F783F914E006EB040090F806
:102280002000392809DA06EB040090F82000401CF1
:1022900006EB040181F8200004E0302006EB040185
:1022A00081F820000420F9F742FB00281ED0002C02
:1022B00007D1F06A401CF062F16A0020F9F75FF97B
:1022C00014E006EB040090F82000312809DB06EB4F
:1022D000040090F82000401E06EB040181F8200065
:1022E00004E0392006EB040181F820000820F9F70A
:1022F00023FB002871D0042C67D196F824000090AD
:1023000096F8233096F8222096F821100120FBF74A
:1023100015FB040096F82400009096F8233096F8F8
:10232000222096F821100020FBF708FB082D14D17D
:10233000002C04D1012802D10121316101E00021EA
:102340003161012C01D0012802D1F9F78EF94DE05D
:1023500002210320F9F731F948E0042D14D1012CB2
:1023600001D001280BD10120FBF7BFFB0020012188
:10237000F7F7FDFD03210120F9F71FF936E00221EF
:102380000320F9F71AF931E0052D14D1012C01D001
:1023900001280BD10220FBF7A8FB00200121F7F751
:1023A000E6FD03210120F9F708F91FE002210320CF
:1023B000F9F703F91AE0012802D1F9F756F915E007
:1023C00002210320F9F7F9F810E0F06A401CF062EE
:1023D000F16A0020F9F7D3F808E00120F9F7ACFA28
:1023E000002803D0F9F741F9F9F73FF908B070BDBB
:1023F0000000000010B586B002200021F7F7B7FDFD
:10240000162223496846F8F789FE69460020F9F745
:10241000BBFB0420F9F783FB0120F9F7D8FB162258
:1024200026496846F8F77AFE69460120F9F7ACFBC1
:102430001DA421000220F9F7A7FB21000320F9F7D2
:10244000A3FB21000420F9F79FFB21000520F9F7E9
:102450009BFB21000620F9F797FB21000720F9F7E5
:1024600093FB21000820F9F78FFB0120F9F764FAAC
:10247000002804D10820F9F75FFA002803D0F9F703
:10248000F4F8F9F7F2F806B010BD00002A000000D9
:1024900000D3030040EE030060EE010060EE030095
:1024A00068EE010080EE030000000000C0EE0300B3
:1024B000A0EE0300E0EE030000EF030040EC030099
:1024C00060EC030018B597B0040040200021F7F736
:1024D0004EFDDFF8143791A216216846F8F779FF10
:1024E00069460020F9F750FB0320F9F718FB042098
:1024F000F9F76DFB0020F9F726F8401CF9F713FBFC
:10250000DFF8E836DFF8E826162106A8F8F761FFBD
:10251000DFF8E036DFF8E02616210DF12E00F8F79F
:1025200058FFDFF8D836DFF8D826162111A8F8F7BB
:1025300050FF06A90120F9F727FB0DF12E0102201B
:10254000F9F722FB11A90320F9F71EFB74A104205F
:10255000F9F71AFB0120F9F7EFF9002802D0F9F793
:1025600084F841E00820F9F7E7F9002839D0012084
:10257000F8F7E9FF002810D101211E20F9F71DF816
:102580000220FBF741FD20630420FBF73DFD606363
:102590000520FBF739FDA0631EE001280CD10121C5
:1025A0001D20F9F70AF80120FBF72EFD206300201B
:1025B000FBF72AFD60630FE002280DD101211F20E7
:1025C000F8F7FBFF0120FAF7D9F9002802D0012023
:1025D000206301E0002020630020DFF82816086057
:1025E00002E00320F9F759F818B010BD38B588B0EB
:1025F00004001622DFF8FC1502A8F8F78FFD02A9E7
:102600000020F9F7C1FA0420F9F789FA0420F9F754
:10261000DEFADFF8F455236B2A00032102A8F8F74D
:10262000D8FE02A90120F9F7AFFA3EA10220F9F77E
:10263000ABFA636B2A00032102A8F8F7CAFE02A9CD
:102640000320F9F7A1FA36A529000420F9F79CFA2E
:1026500029000520F9F798FA29000620F9F794FADD
:1026600029000720F9F790FA29000720F9F78CFADA
:10267000DFF890552868F9F756FA0120F9F75CF968
:10268000002802D0F8F7F1FF45E00820F9F754F9E7
:10269000002815D0286803280ED1216B0120FBF7F4
:1026A000AFFC616B0020FBF7ABFC00202021F7F7AB
:1026B0005EFCF8F7DAFF2EE02868401C28602AE06C
:1026C0002868002803D12868401C286023E0286877
:1026D00001280BD10120019001200090012300224C
:1026E0001721206BF9F74CF8206314E028680228C2
:1026F00003D12868401C28600DE0286803280AD10F
:102700000120019001200090012300223B21606BF9
:10271000F9F736F8606309B030BD0000257300009A
:10272000000000003A000000F8B596B0040008A8C8
:10273000DFF8D81438220AF041F81622DFF8AC147A
:1027400002A8F8F7EBFC02A90020F9F71DFA042013
:10275000F9F7E5F90420F9F73AFADFF8A854286800
:1027600000281BD1A06B0190606B0090236BDFF8F9
:10277000A024092102A8F8F72CFE02A90120F9F7EC
:1027800003FA7BA631000220F9F7FEF9310003209D
:10279000F9F7FAF931000420F9F7F6F92868012869
:1027A00021D1236BDFF86024032102A8F8F711FE82
:1027B00002A90120F9F7E8F9A06B0090636BDFF83C
:1027C0005424072102A8F8F704FE02A90220F9F711
:1027D000DBF967A631000320F9F7D6F931000420B0
:1027E000F9F7D2F948E02868022825D1236BDFF8F1
:1027F0002824042102A8F8F7ECFD02A90120F9F72A
:10280000C3F9636BDFF80024032102A8F8F7E1FDA8
:1028100002A90220F9F7B8F9A36BDFF8002404211C
:1028200002A8F8F7D6FD02A90320F9F7ADF950A1E7
:102830000420F9F7A9F91FE0606B0090236BDFF823
:10284000E023062102A8F8F7C4FD02A90120F9F748
:102850009BF9A1A10220F9F797F9A36BDFF8A82350
:10286000032102A8F8F7B5FD02A90320F9F78CF9B6
:102870003FA10420F9F788F9216B0722B1FBF2F0A0
:1028800002FB101094F8381011F0030F0BD1616B9C
:10289000012902D0616B022905D108A9226B01EB45
:1028A0008201C96A05E008A9626B01EB820151F857
:1028B000041CA36B1C26A76B5FF01C0CB3FBF6F289
:1028C00006FB1232B7FBFCF30CFB137712EB9702FB
:1028D00008181018801D0721B0FBF1F201FB12004F
:1028E000012806D10422DFF83C1302A8F8F716FCF1
:1028F0002DE0022806D10422DFF82C1302A8F8F7F5
:102900000DFC24E0032805D10422C84902A8F8F7E9
:1029100005FC1CE0042805D10422C54902A8F8F7EB
:10292000FDFB14E0052805D10422C24902A8F8F7EE
:10293000F5FB0CE0062805D10422BF4902A8F8F7F0
:10294000EDFB04E00422BD4902A8F8F7E7FB0020F4
:102950008DF80B00206B00280CD0606B002809D08C
:10296000A06B002806D002A90520F9F70DF905E0B3
:10297000000000009AA10520F9F706F998A6310099
:102980000620F9F701F931000720F9F7FDF83100C9
:102990000820F9F7F9F82868F9F7C5F80120F8F7E1
:1029A000CBFF002802D0F8F760FE93E00820F8F78C
:1029B000C3FF00285BD02868032830D1206B1D2876
:1029C00008D1606B022805D194F8380010F0030F8D
:1029D00040F080800220FBF717FB216B81420BD176
:1029E0000420FBF711FB616B814205D10520FBF749
:1029F0000BFBA16B81420FD0216B0220FBF700FB88
:102A0000616B0420FBF7FCFAA16B0520FBF7F8FAD9
:102A100000202021F7F7ABFAF8F727FE5AE02868E4
:102A2000022820D1606B022806D1206B1E2851D2CB
:102A30002868401C28604DE0606B042808D0606B5B
:102A4000062805D0606B092802D0606B0B2806D1E0
:102A5000206B1F283ED22868401C28603AE0286876
:102A6000401C286036E02868401C286032E0286856
:102A7000002803D12868401C28602BE02868012822
:102A80000BD10120019001200090012301221F2180
:102A9000206BF8F775FE20631CE0286802280BD134
:102AA0000120019001200090012301220C21606B84
:102AB000F8F766FE60630DE0286803280AD101205C
:102AC000019001200090012300226321A06BF8F700
:102AD00057FEA06317B0F0BD2F00000038B588B0D6
:102AE000040040200021F7F742FA444B3DA2162192
:102AF00002A8F8F76EFC02A90020F9F745F80420B7
:102B0000F9F70DF80420F9F762F8206B002805D1D9
:102B100016224B4902A8F8F701FB04E016224949A6
:102B200002A8F8F7FBFA02A90120F9F72DF82CA565
:102B300029000220F9F728F829000320F9F724F8E2
:102B400029000420F9F720F829000520F9F71CF8DE
:102B500029000620F9F718F829000720F9F714F8DA
:102B600029000820F9F710F80820F8F7E5FE0028FA
:102B700020D0206B002804D00120F9F7FFFE0028A8
:102B800007D0206B002812D10120F9F7F7FE0028AA
:102B90000DD0206B002803D10120F9F7F8FE02E0E8
:102BA0000120F9F7EFFE00200821F7F7E0F9F8F728
:102BB0005CFD12E00120F8F7BFFE002802D0F8F714
:102BC00054FD0AE000200190002000900123002223
:102BD0000121206BF8F7D4FD206309B030BD00005F
:102BE0000000000025730000C0D2030080ED030048
:102BF00010EC0100A0ED030018EC010060ED0300F3
:102C000020EC01005011002028EC010000E401003C
:102C100068E70100A4E8010030EC010038EC010095
:102C2000B0E8010000EB030020EB030040EB0300E1
:102C300060EB030080EB0300A0EB0300C0EB03009C
:102C400080E60300E0D9030030B591B04FF4006096
:102C50000021F7F78CF9DFF8284516222100684695
:102C6000F8F75CFA2300DFF81C25162106A8F8F710
:102C7000B0FBF9F744FF012808D12300DFF808254D
:102C800016210DF12E00F8F7A4FB07E02300DFF872
:102C9000FC2416210DF12E00F8F79BFB0220F8F71B
:102CA00023FC0320F8F73BFF0420F8F790FF694668
:102CB0000020F8F769FF0020F8F745FC401CF8F702
:102CC00032FF0220F8F73FFC040006A90120F8F7C4
:102CD0005BFF0DF12E010220F8F756FFB0A5290089
:102CE0000320F8F751FF29000420F8F74DFF0120D9
:102CF000F8F722FE002802D0F8F7B7FC16E008200B
:102D0000F8F71AFE00280ED00120F8F71CFC012865
:102D100004D101210B20F8F750FC07E00121092024
:102D2000F8F74BFC02E02000F8F7B7FC11B030BD1B
:102D300070B5B2B01622DFF848146846F8F7EEF91D
:102D400069460020F8F720FF0320F8F7E8FE04208A
:102D5000F8F73DFF00200AE0002206AB162404FB32
:102D600000F423445A54491C1629F5D3401C082862
:102D700001D20021F8E7012400265FF0FF30FBF7C5
:102D8000DFF905000EE025420BD0F9F7B8FE02008E
:102D9000210006A8162303FB06F31844FBF7FAF9F3
:102DA000761C6400082E01D2002CECD13000F8F71C
:102DB0009BFB002D03D10020F8F7B5FE05E00020B5
:102DC000F8F7C1FB401CF8F7AEFE0220F8F7BBFB9A
:102DD0000500162406A804FB05F101440120F8F7BC
:102DE000D3FE06A804FB05F1084410F116010220E9
:102DF000F8F7CAFE06A804FB05F1084410F12C01FF
:102E00000320F8F7C1FE06A86543284410F14201EB
:102E10000420F8F7B9FE0120F8F78EFD002802D053
:102E2000F8F723FC27E00820F8F786FD00281FD0DC
:102E30000120F8F788FB0500F9F761FE0200102178
:102E40006846FBF7A7F91222694606A8654328449D
:102E5000F8F7C6FA002808D1FBF799F9002804D042
:102E600002210C20F8F7A9FB05E0F8F7FEFB02E0D1
:102E70003000F8F712FC32B070BD70B5B2B04FF44C
:102E800000600021F7F773F8F9F739FE012806D141
:102E9000BB4BBF4A16216846F8F79BFA05E0B84BD2
:102EA000BC4A16216846F8F794FA69460020F8F7FC
:102EB0006BFE0320F8F733FE0420F8F788FE0020AD
:102EC0000AE0002206AB162404FB00F423445A5403
:102ED000491C1629F5D3401C082801D20021F8E727
:102EE000012400265FF0FF30FBF72EF905000BE010
:102EF000254208D0210006A8162202FB06F2104443
:102F0000FBF78EF9761C6400082E01D2002CEFD15D
:102F10003000F8F7E9FA002D03D10020F8F703FE9E
:102F200005E00020F8F70FFB401CF8F7FCFD02203D
:102F3000F8F709FB0400162506A805FB04F1014477
:102F40000120F8F721FE06A805FB04F1084410F162
:102F500016010220F8F718FE06A805FB04F1084444
:102F600010F12C010320F8F70FFE06A86C43204453
:102F700010F142010420F8F707FE0820F8F7DCFC06
:102F8000002804D10120F8F7D7FC002802D0F8F778
:102F90006CFB02E03000F8F780FB32B070BD00003F
:102FA000000000002DE97043C8B048200021F6F76A
:102FB000DEFF162278496846F8F7B0F800200AE0EC
:102FC000002206AB162404FB00F423445A54491C87
:102FD0001629F5D3401C0C2801D20021F8E7012462
:102FE000002500265FF0FF304FF6FF71FBF7C6F8B3
:102FF0008046894617E018EA040019EA0501002214
:103000000023994201D1904209D022002B0006A84A
:10301000162101FB06F10844FBF714F9761C6D003C
:1030200045EAD47564000C2E05D2002000218D42A3
:10303000E1D18442DFD13000F8F756FA0320F8F7E7
:103040006EFD0420F8F7C3FD69460020F8F79CFDEB
:1030500000200021894505D1804503D10020F8F7E3
:1030600062FD05E00020F8F76EFA401CF8F75BFD02
:103070000220F8F768FA0400162506A805FB04F1FB
:1030800001440120F8F780FD06A805FB04F108447F
:1030900010F116010220F8F777FD06A805FB04F1F0
:1030A000084410F12C010320F8F76EFD06A86C43CC
:1030B000204410F142010420F8F766FD0820F8F7DB
:1030C0003BFC002804D10120F8F736FC002802D090
:1030D000F8F7CBFA02E03000F8F7DFFA48B0BDE8C5
:1030E000708310B58CB0FBF752F804002B4B21A273
:1030F000162106A8F8F76DF923001FA216216846CD
:10310000F8F767F90420F8F70AFD0120F8F75FFDEA
:1031100006A90020F8F738FD69460120F8F734FDCC
:1031200016A421000220F8F72FFD21000320F8F754
:103130002BFD21000420F8F727FD21000520F8F7DA
:1031400023FD21000620F8F71FFD21000720F8F7D6
:103150001BFD21000820F8F717FD0020F8F7E3FC1D
:103160000820F8F7E9FB002801D0F8F77EFA0CB048
:1031700010BD000025730000256400000000000061
:1031800060D2030040EC0100BCE8010048EC010003
:1031900050EC010058EC010080D20300E0DD030098
:1031A00018B597B0040049200021F6F7E0FE03208F
:1031B000F8F79AF91622DFF888186846F7F7AEFF95
:1031C00069460020F8F7E0FC0320F8F7A8FC04208B
:1031D000F8F7FDFCDFF86C38DFF86C28162106A83C
:1031E000F8F7F7F8DFF86438DFF8642816210DF1F6
:1031F0002E00F8F7EEF8DFF85C38DFF85C281621CF
:1032000011A8F8F7E6F80020F8F79DF9401CF8F748
:103210008AFC06A90120F8F7B7FC0DF12E01022067
:10322000F8F7B2FC11A90320F8F7AEFC64A1042062
:10323000F8F7AAFC0820F8F77FFB002841D001200E
:10324000F8F781F9002804D101211720F8F7B5F922
:1032500042E001281FD1A068012802D0206900287F
:1032600008D101211920F8F7A8F901210220F8F767
:10327000A4F903E001211920F8F79FF90820F9F7D4
:103280007DFB002802D00120206301E000202063A4
:10329000206BE06320E002281ED1A068012802D044
:1032A0002069002808D101211B20F8F786F90121A7
:1032B0000220F8F782F90FE001211B20F8F77DF9D1
:1032C0000AE00120F8F738FB002802D0F8F7CDF922
:1032D00002E00320F8F7E1F918B010BD30B58DB069
:1032E00049200021F6F743FE1622DFF8581701A8FF
:1032F000F7F714FF01A90020F8F746FC0420F8F7BF
:103300000EFC0120F8F763FC0A23152207A9DFF859
:103310004C07F8F7D7FAFAF7F2FADFF84447A04279
:1033200001D3DFF84007FAF7EAFADFF83C570090DC
:1033300007AB2A00162101A8F8F74BF801A90120D4
:10334000F8F722FC0A23152207A9DFF82007F8F76F
:10335000B9FAFAF7D1FAA04201D3DFF808070090D2
:1033600007AB2A00162101A8F8F733F801A90520B8
:10337000F8F70AFC12A421000220F8F705FC21004E
:103380000320F8F701FC21000420F8F7FDFB2100E1
:103390000620F8F7F9FB21000720F8F7F5FB2100DC
:1033A0000820F8F7F1FB0020F8F7BDFB0820F8F73C
:1033B000C3FA002801D0F8F758F90DB030BD00006D
:1033C00000000000F8B588B0050040200021F6F7A5
:1033D000CEFD286B002805D0686B002802D0A86BB2
:1033E000002801D1012600E000261622DFF8801611
:1033F00002A8F7F793FE02A90020F8F7C5FB042006
:10340000F8F78DFB0420F8F7E2FB0020F8F79BF8B3
:1034100004002000F8F787FB002C1CD1A86B01905A
:10342000686B00902B6BDFF84C26092102A8F7F798
:10343000D0FF02A90120F8F7A7FBB6A739000220A8
:10344000F8F7A2FB39000320F8F79EFB39000420AF
:10345000F8F79AFB6BE0012C21D12B6BDFF81826D3
:10346000032102A8F7F7B5FF02A90120F8F78CFBAA
:10347000A86B00906B6BDFF80426072102A8F7F712
:10348000A8FF02A90220F8F77FFBA2A739000320BA
:10349000F8F77AFB39000420F8F776FB47E0022CB6
:1034A00025D12B6BDFF8D825042102A8F7F791FF6F
:1034B00002A90120F8F768FB6B6BDFF8BC2503213C
:1034C00002A8F7F786FF02A90220F8F75DFBAB6BB5
:1034D000DFF8B025042102A8F7F77BFF02A903203B
:1034E000F8F752FB8BA10420F8F74EFB1FE0686B46
:1034F00000902B6BDFF89025062102A8F7F769FFF3
:1035000002A90120F8F740FB83A10220F8F73CFB59
:10351000AB6BDFF86425032102A8F7F75AFF02A975
:103520000320F8F731FB7BA10420F8F72DFB012ED7
:103530000AD11622DFF8541502A8F7F7EFFD02A909
:103540000520F8F721FB03E072A10520F8F71CFB2A
:1035500070A631000620F8F717FB31000720F8F7B6
:1035600013FB31000820F8F70FFB0120F8F7E4F90E
:10357000002802D0F8F779F8CAE00820F8F7DCF95B
:10358000002800F09C80032C30D1286B1D2808D126
:10359000686B022805D195F8380010F0030F40F051
:1035A000B7805020F9F7F9F9296B81420BD15120EE
:1035B000F9F7F3F9696B814205D15220F9F7EDF97A
:1035C000A96B81420FD000200821F6F7D0FC296BAF
:1035D0005020F9F701FA696B5120F9F7FDF9A96B51
:1035E0005220F9F7F9F9F8F740F891E0022C41D1AF
:1035F000686B002817D15120F9F7CFF900280FD0B8
:1036000000215020F9F7E8F900215120F9F7E4F9F9
:1036100000215220F9F7E0F900200821F6F7A7FC75
:10362000F8F723F874E0686B022808D1286B1E288D
:103630006ED2641C21000020F7F7A1FF68E0686BE0
:10364000042808D0686B062805D0686B092802D0CA
:10365000686B0B2808D1286B1F2859D2641C2100E5
:103660000020F7F78CFF53E0641C21000020F7F7DF
:1036700086FF4DE0012C1FD1286B002817D1502068
:10368000F9F78BF900280FD000215020F9F7A4F9A1
:1036900000215120F9F7A0F900215220F9F79CF9F7
:1036A00000200821F6F763FCF7F7DFFF30E0022186
:1036B0000020F7F764FF2BE0F7F7D7FF28E0012C95
:1036C0000BD10120019001200090012300221F2135
:1036D000286BF8F755F828631AE0022C0BD101206B
:1036E000019001200090012300220C21686BF8F763
:1036F00047F868630CE0032C0AD1012001900120F7
:103700000090012300226321A86BF8F739F8A86321
:1037100009B0F0BD000000002F00000038B588B0EF
:10372000040040200021F6F722FC1622D84902A806
:10373000F7F7F4FC02A90020F8F726FA0420F8F7BE
:10374000EEF9F9F7DCF9002803D10420F8F73FFA85
:1037500002E00320F8F73BFA206B002806D0CD4B9F
:1037600089A2162102A8F7F734FE05E0C74B86A20E
:10377000162102A8F7F72DFE02A90120F8F704FA96
:10378000ACA529000220F8F7FFF929000320F8F77B
:10379000FBF929000420F8F7F7F929000520F8F7CC
:1037A000F3F929000620F8F7EFF929000720F8F7C8
:1037B000EBF929000820F8F7E7F90020F8F7B3F94A
:1037C0000120F8F7B9F8002802D0F7F74EFF48E0DB
:1037D0000820F8F7B1F8002832D0206BE16B88425E
:1037E0001DD0206B002803D00820F9F7CBF802E0A9
:1037F0000820F9F7CCF8A8494020F9F7EDF80021A6
:103800005020F9F7E9F800215120F9F7E5F80021F7
:103810005220F9F7E1F800200821F6F7A8FB206B09
:10382000002802D1F7F721FF1BE002211A20F7F749
:10383000C4FE4020F9F7B1F82063206BE06310E08C
:103840000020019001200090012300220121206B23
:10385000F7F796FF2063F9F752F9012801D101200B
:10386000206309B030BD38B588B004004020002185
:10387000F6F77DFB1622894902A8F7F74FFC02A94B
:103880000020F8F781F90420F8F749F90420F8F747
:103890009EF9236B68A2082102A8F7F79AFD02A9F6
:1038A0000120F8F771F963A529000220F8F76CF9F7
:1038B00029000320F8F768F929000420F8F764F9D3
:1038C00029000520F8F760F929000620F8F75CF9CF
:1038D00029000720F8F758F929000820F8F754F9CB
:1038E0000020F8F720F90120F8F726F8002802D088
:1038F000F7F7BBFE46E00820F8F71EF800282FD0A7
:10390000206BE16B884207D0216B4020F9F764F807
:1039100000200821F6F72BFB02211820F7F74DFEB7
:103920005020F9F73AF820635120F9F736F8606330
:103930005220F9F732F8A06301210020F7F71FFEAB
:10394000206B002805D0606B002802D0A06B0028F7
:1039500018D100202063002060630020206311E064
:10396000F9F7CDF8012801D14B4900E04C4942F26A
:10397000107201200190012000901300206BF7F7D6
:10398000FFFE206309B030BD2573000010B586B07E
:10399000162230496846F7F7C1FB69460020F8F760
:1039A000F3F80420F8F7BBF80320F8F710F93D4BC3
:1039B00022A216216846F7F70CFD69460120F8F7A8
:1039C000E3F80020F8F7AFF81AA421000220F8F776
:1039D000DBF821000320F8F7D7F821000420F8F7DE
:1039E000D3F821000520F8F7CFF821000620F8F7DA
:1039F000CBF821000720F8F7C7F821000720F8F7D7
:103A0000C3F80120F7F798FF002802D0F7F72DFE42
:103A10000EE00820F7F790FF002809D05FF0007053
:103A2000FAF752F900208021F6F7A1FAF7F71DFE08
:103A300006B010BD000000002564000025730000E2
:103A4000A0D2030000ED0300D8EB010020ED03003D
:103A5000E0EB010040ED0300E8EB0100C0EC0300E7
:103A600000CA9A3BFFC99A3BF0EB0100E0EC03006F
:103A700080EC030058E70100F8EB01008CE801003E
:103A800000EC010008EC010098E8010080E603006A
:103A900060F00300E0D9030040420F00A0DD030006
:103AA00080841E00E0DA030078B5ADB00400072082
:103AB000F7F71AFD16229C496846F7F72FFB9B4B38
:103AC0009B4A162106A8F7F784FC9A4B9A4A1621BE
:103AD0000DF12E00F7F77DFC984B994A162111A89D
:103AE000F7F777FC974B984A16210DF15A00F7F734
:103AF00070FC964B964A16211CA8F7F76AFC954B6A
:103B0000954A16210DF18600F7F763FC934B944A12
:103B1000162127A8F7F75DFC0320F8F700F804202A
:103B2000F8F755F869460020F8F72EF80220F7F765
:103B30000AFD0500162606A806FB05F10144012032
:103B4000F8F722F806A806FB05F1084410F1160163
:103B50000220F8F719F806A806FB05F1084410F151
:103B60002C010320F8F710F806A87543284410F13B
:103B700042010420F8F708F80020F7F7E4FC401CA5
:103B8000F7F7D1FF0820F7F7D7FE00280BD0206BFE
:103B9000E16B884204D001213B20F7F70EFD12E0D3
:103BA000F7F763FD0FE00120F7F7C6FE002802D00B
:103BB000F7F75BFD07E00720F7F76FFD0120F7F748
:103BC000C2FC401C20632EB070BD38B58CB0040020
:103BD0001622554906A8F7F7A1FA206B012806D14D
:103BE000524B4FA216216846F7F7F3FB55E0206BC6
:103BF000022806D14F4B4AA216216846F7F7E9FB87
:103C00004BE0206B032806D14C4B45A21621684699
:103C1000F7F7DFFB41E0206B042806D1494B40A2B7
:103C200016216846F7F7D5FB37E0206B052806D14B
:103C3000464B3BA216216846F7F7CBFB2DE0206BE5
:103C4000062806D1434B36A216216846F7F7C1FB7A
:103C500023E0206B072806D1404B31A2162168468D
:103C6000F7F7B7FB19E0206B082806D13D4B2CA2D3
:103C700016216846F7F7ADFB0FE0206B092806D147
:103C8000394B27A216216846F7F7A3FB05E0374B0F
:103C900023A216216846F7F79CFB0420F7F73FFFA5
:103CA0000320F7F794FF06A90020F7F76DFF694698
:103CB0000120F7F769FF1BA529000220F7F764FF31
:103CC00029000320F7F760FF29000420F7F75CFFC5
:103CD00029000520F7F758FF29000620F7F754FFC1
:103CE00029000720F7F750FF29000820F7F74CFFBD
:103CF0000020F7F718FF0120F7F71EFE002802D07A
:103D0000F7F7B3FC09E00820F7F716FE002804D007
:103D1000206B08F0EBFCF7F7A8FC0DB030BD0000FD
:103D200025733F000000000020D2030020D00300D4
:103D300048ED010040D0030050ED010060D00300C9
:103D400058ED010080D0030060ED0100A0D0030019
:103D500068ED0100C0D0030070ED0100E0D0030069
:103D600078ED010000D1030020D1030040D1030011
:103D7000F0B5BDB0050070200021F6F7F8F8F8F7AF
:103D8000BEFE012801D1092400E00A242000F7F733
:103D9000ABFB1622DFF8A01A6846F7F7BFF9F8F771
:103DA000AEFE012854D1DFF8943ADFF8942A1621A8
:103DB00006A8F7F70EFBDFF88C3ADFF88C2A1621FD
:103DC0000DF12E00F7F705FBDFF8843ADFF8842ABF
:103DD000162111A8F7F7FDFADFF87C3ADFF87C2A04
:103DE00016210DF15A00F7F7F4FADFF8743ADFF80C
:103DF000742A16211CA8F7F7ECFADFF86C3ADFF802
:103E00006C2A16210DF18600F7F7E3FADFF8603A25
:103E1000DFF8602A162127A8F7F7DBFADFF8583A0F
:103E2000DFF8582A16210DF1B200F7F7D2FADFF8C1
:103E3000503ADFF8502A162132A8F7F7CAFA03A23F
:103E400016210DF1DE00F7F7C4FA56E0000000007D
:103E5000DFF8343ADFF8E829162106A8F7F7B9FAAF
:103E6000DFF8D839DFF8E02916210DF12E00F7F739
:103E7000B0FADFF8D039DFF8DC29162111A8F7F7FE
:103E8000A8FADFF8CC39DFF8D42916210DF15A0051
:103E9000F7F79FFADFF8C039DFF8C82916211CA808
:103EA000F7F797FADFF8B839DFF8C02916210DF1D6
:103EB0008600F7F78EFADFF8B039DFF8B829162157
:103EC00027A8F7F786FADFF8A839DFF8B029162116
:103ED0000DF1B200F7F77DFADFF89C39DFF8A4297D
:103EE000162132A8F7F775FADFF89439DFF89C2924
:103EF00016210DF1DE00F7F76CFA0320F7F70FFE3D
:103F00000420F7F764FE69460020F7F73DFE002025
:103F1000F7F719FB401CF7F706FE0220F7F713FB33
:103F20000600162706A807FB06F101440120F7F753
:103F30002BFE06A807FB06F1084410F1160102202B
:103F4000F7F722FE06A807FB06F1084410F12C0142
:103F50000320F7F719FE06A87E43304410F1420112
:103F60000420F7F711FE0120F7F7E6FC002802D045
:103F7000F7F77BFBFEE00820F7F7DEFC002800F0F7
:103F8000F6800120F7F7DFFA0400F8F7B8FD012802
:103F900052D1002C04D101213C20F7F70EFBE3E0C5
:103FA000012C04D101214920F7F707FBDCE0022CAA
:103FB00004D101215C20F7F700FBD5E0032C0ED1E2
:103FC00001212520F7F7F9FA1020F8F7D7FC00288F
:103FD00002D001202863C7E000202863C4E0042C3D
:103FE00004D101212620F7F7E8FABDE0052C04D121
:103FF00001212B20F7F7E1FAB6E0062C04D10121CC
:104000006020F7F7DAFAAFE0072C0DD1F8F755FD8D
:104010001E2804D201210F20F7F7CFFAA4E00121D6
:104020007920F7F7CAFA9FE0082C40F09D80012123
:104030006820F7F7C2FA97E0002C29D1012121204E
:10404000F7F7BBFAF8F763FD012802D104202863D3
:104050008AE0F8F76AFD012802D10320286383E093
:10406000F8F771FD012802D1012028637CE0F8F700
:1040700078FD012802D10220286375E0F8F77FFD62
:10408000012802D1052028636EE0002028636BE040
:10409000012C08D1F8F781FD002804D101213C2032
:1040A000F7F78BFA60E0022C08D1F8F776FD0028CC
:1040B00004D101214920F7F780FA55E0032C08D1FB
:1040C000F8F76BFD002804D101215C20F7F775FAA1
:1040D0004AE0042C12D1F8F760FD00280ED101212E
:1040E0002520F7F76AFA1020F8F748FC002802D0DC
:1040F0000120286338E00020286335E0052C08D132
:10410000F8F74BFD002804D101212620F7F755FAD6
:104110002AE0062C08D1F8F740FD002804D101213F
:104120002B20F7F74AFA1FE0072C08D1F8F735FDE6
:10413000002804D101216020F7F73FFA14E0082C91
:1041400008D1F8F72AFD002804D101217920F7F7DA
:1041500034FA09E0092C07D1F8F71FFD002803D134
:1041600001216820F7F729FA286BE86302E02000B4
:10417000F7F793FA3DB0F0BD38B594B00400502085
:104180000021F5F7F4FE1622DFF8FC160EA8F6F76C
:10419000C5FF206B01280AD1162208A90920F8F7CB
:1041A00019FD61A2162102A8F7F713F941E0206B6F
:1041B00002280AD1162208A90420F8F70BFDBCA298
:1041C000162102A8F7F705F933E0206B03280AD17E
:1041D000162208A90820F8F7FDFCB6A2162102A8AD
:1041E000F7F7F7F825E0206B04280AD1162208A972
:1041F0000720F8F7EFFCB0A2162102A8F7F7E9F8BC
:1042000017E0206B05280AD1162208A90A20F8F722
:10421000E1FCAAA2162102A8F7F7DBF809E0A8A2A0
:10422000162108A8F7F7D5F8A6A2162102A8F7F7D5
:10423000D0F80420F7F773FC0420F7F7C8FC0EA9A8
:104240000020F7F7A1FC08A90120F7F79DFC02A9BF
:104250000520F7F799FC9BA529000220F7F794FCAD
:1042600029000320F7F790FC29000420F7F78CFCC5
:1042700029000620F7F788FC29000720F7F784FCBF
:1042800029000820F7F780FC0020F7F74CFC0820F5
:10429000F7F752FB002822D0206B002841D0206B7A
:1042A000E16B884204D001212220F7F786F938E03B
:1042B000206B042810D101212320F7F77EF902207A
:1042C000F8F75CFB002802D10020206301E0012008
:1042D0002063206BE06324E0F7F7C7F921E00120B9
:1042E000F7F72AFB002802D0F7F7BFF919E0206B97
:1042F00000280BD000200190012000900123012212
:104300000521206BF7F73CFA20630AE000200190BA
:1043100001200090012300220521206BF7F730FADD
:10432000206315B030BD00002831290038B592B0A7
:10433000040078200021F5F71AFE1622DFF8481550
:104340006846F6F7EBFE69460020F7F71DFCDFF83C
:104350004035A4A2162106A8F7F73BF8206B0428E5
:1043600005D1162269460720F8F734FC1FE0206BC0
:10437000022805D1162269460420F8F72BFC16E026
:10438000206B032805D1162269460820F8F722FC85
:104390000DE0206B052805D1162269460A20F8F7A2
:1043A00019FC04E0162269460920F8F713FC6B4655
:1043B000DFF8E02416210CA8F7F70BF80420F7F734
:1043C000AEFB0320F7F703FC0020F7F7ACFB06A9D0
:1043D0000120F7F7D9FB3BA529000220F7F7D4FB12
:1043E00029000320F7F7D0FB29000420F7F7CCFBC6
:1043F00029000520F7F7C8FB29000620F7F7C4FBC2
:1044000029000720F7F7C0FB29000820F7F7BCFBBD
:104410000820F7F791FA002840D0206B042804D137
:1044200007211E20F8F7D8FA1BE0206B022804D1E0
:1044300004211E20F8F7D0FA13E0206B032804D1E2
:1044400008211E20F8F7C8FA0BE0206B052804D1DC
:104450000A211E20F8F7C0FA03E009211E20F8F710
:10446000BBFA00200221F5F782FD206B042810D151
:1044700002212320F7F7A1F80220F8F77FFA00289D
:1044800002D10020206301E001202063206BE06363
:104490000CE0F7F7EAF8F7F7E8F807E00120F7F79C
:1044A0004BFA002802D0200000F00EFA13B030BD05
:1044B00028322900283329002834290028352900EA
:1044C0004E4F00000000000038B58EB00400782088
:1044D0000021F5F74CFD1622DFF8BC1308A8F6F70B
:1044E0001DFE206B002806D11622DFF8B01302A8AB
:1044F000F6F714FE05E01622DFF8A41302A8F6F77B
:104500000DFE0420F7F70BFB0420F7F760FB0020FB
:10451000F7F709FB08A90020F7F736FB02A90120ED
:10452000F7F732FB84A529000220F7F72DFB2900BD
:104530000320F7F729FB29000420F7F725FB2900C2
:104540000520F7F721FB29000620F7F71DFB2900BE
:104550000720F7F719FB29000820F7F715FB0820BB
:10456000F7F7EAF9002826D0E06B216B88420DD0DE
:10457000206B002803D00220F8F704FA02E00220A2
:10458000F8F705FA00200821F5F7F1FC1E20F8F7EE
:1045900004FA07280AD15E20F8F7FFF92063206BA0
:1045A000E06302212420F7F708F818E0F7F75DF838
:1045B000F7F75BF813E00120F7F7BEF9002803D006
:1045C000200000F081F90AE0002001900120009015
:1045D000012300220121206BF7F7D2F820630FB0EE
:1045E00030BD00002573000038B58EB004004820AF
:1045F0000021F5F7BCFC0420F7F791FA1622A9492F
:1046000002A8F6F78BFD02A90020F7F7BDFA0220F9
:10461000F8F7B4F9216B002912D1002805D1A24A7C
:10462000162102A8F6F7D5FE04E0A04A162102A83A
:10463000F6F7CFFE7DA2162108A8F6F7CAFE27E0FE
:10464000216B012912D1002805D1994A162102A80F
:10465000F6F7BFFE04E0974A162102A8F6F7B9FE66
:1046600073A2162108A8F6F7B4FE11E0002805D1C0
:10467000914A162102A8F6F7ACFE04E08F4A1621F3
:1046800002A8F6F7A6FE6BA2162108A8F6F7A1FE6F
:104690000020F7F748FA02A90120F7F775FA26A5D6
:1046A00029000220F7F770FA29000320F7F76CFAC7
:1046B00029000420F7F768FA08A90520F7F764FA3B
:1046C00029000620F7F760FA29000720F7F75CFABF
:1046D00029000820F7F758FA0420F7F778FA08209D
:1046E000F7F72AF9002810D0E06B216B884207D039
:1046F000216B5E20F8F770F900200821F5F737FCF0
:10470000F6F7B3FFF6F7B1FF13E00120F7F714F95E
:10471000002803D0200000F0D7F80AE00020019024
:1047200001200090012300220221206BF7F728F8D6
:1047300020630FB030BD00000000000038B58EB01F
:10474000040070200021F5F712FC1622424908A847
:10475000F6F7E4FC206B002805D11622584902A880
:10476000F6F7DCFC04E01622564902A8F6F7D6FC60
:104770000420F7F7D4F90420F7F729FA0020F7F717
:10478000D2F908A90020F7F7FFF902A90120F7F7ED
:10479000FBF92EA529000220F7F7F6F929000320DE
:1047A000F7F7F2F929000420F7F7EEF929000520C0
:1047B000F7F7EAF929000620F7F7E6F929000720BC
:1047C000F7F7E2F929000820F7F7DEF90820F7F7F4
:1047D000B3F8002814D0206BE16B88420DD0206B19
:1047E000002803D11020F8F7D2F802E01020F8F7E3
:1047F000C9F800200821F5F7BAFBF6F736FF12E0FA
:104800000120F7F799F8002802D0F6F72EFF0AE00A
:104810000020019001200090012300220121206B43
:10482000F6F7AEFF20630FB030BD0000283129003D
:10483000283229002833290040D2030040D3030046
:1048400070EE010060D3030078EE0100000000006C
:1048500080F1030080EE010080D3030088EE0100A8
:10486000A0D3030090EE0100C0D3030098EE010036
:10487000E0D30300A0EE010020F10300A8EE010048
:1048800020D40300B0EE010060F40300B8EE010094
:10489000E0DA0300D8E7010000DA0300C0DA030021
:1048A000A0DA030000F60300E8E90100F4E90100E2
:1048B000CCE60100E8E7010000EA01000CEA010093
:1048C00080E60300E0D9030010B50400F8F71FF9F3
:1048D000012802D1042020631DE0F8F726F9012801
:1048E00002D10320206316E0F8F72DF9012802D148
:1048F000012020630FE0F8F734F9012802D10220EB
:10490000206308E0F8F73BF9012802D10520206375
:1049100001E000202063206BE063F6F7A6FE10BDE7
:1049200078B5A7B0040070200021F5F720FB062021
:10493000F6F7DAFDF8F7E3F8012801D1062500E0E3
:1049400005251622C5496846F6F7E8FBF8F7D7F8BB
:10495000012828D1C24E3300C24A162106A8F6F714
:1049600038FDC14BC14A16210DF12E00F6F731FD7D
:104970003300BF4A162111A8F6F72BFD3300BD4ABC
:1049800016210DF15A00F6F724FD3300BA4A16211C
:104990001CA8F6F71EFDB94BB94A16210DF1860089
:1049A000F6F717FD26E0AE4E3300AE4A162106A8F4
:1049B000F6F70FFDAC4BAD4A16210DF12E00F6F7C0
:1049C00008FD3300AF4A162111A8F6F702FD3300A7
:1049D000AD4A16210DF15A00F6F7FBFCA74BAB4A86
:1049E00016211CA8F6F7F5FC9BA216210DF18600F6
:1049F000F6F7EFFC0320F7F792F80420F7F7E7F853
:104A00000020F6F7A0FD401CF7F78DF8694600205E
:104A1000F7F7BAF80220F6F796FD162606A97043B6
:104A200001440120F7F7B0F80220F6F78CFD06A943
:104A30007043084410F116010220F7F7A5F8022090
:104A4000F6F781FD06A97043084410F12C010320FC
:104A5000F7F79AF80220F6F776FD06A906FB00F6AE
:104A600001EB060010F142010420F7F78DF8012058
:104A7000F6F762FF002802D0F6F7F7FD4EE00820B7
:104A8000F6F75AFF002846D00120F6F75CFD002813
:104A900004D101213E20F6F790FD3FE0012804D12A
:104AA00001214520F6F789FD38E0022804D10121D3
:104AB0003F20F6F782FD31E003280DD1F8F71FF80B
:104AC000012804D101214020F6F777FD26E00121DD
:104AD0004120F6F772FD21E0042811D1F8F70FF814
:104AE000012804D101214120F6F767FD16E00121DC
:104AF0003D20F6F762FD3B20F7F74FFF20630DE006
:104B000005280BD101213D20F6F757FD3B20F7F793
:104B100044FF206302E02800F6F7BFFD28B070BD17
:104B200038B58CB0040070200021F5F720FA534B03
:104B3000574A162106A8F6F74CFC206B012805D130
:104B4000162254496846F6F7E9FA0FE0206B03286D
:104B500005D1162250496846F6F7E0FA06E016221B
:104B60004E496846F6F7DAFA002020630420F6F78B
:104B7000D6FF0420F7F72BF806A90020F7F704F872
:104B800069460120F7F700F833A529000220F6F75F
:104B9000FBFF29000320F6F7F7FF29000420F6F7B2
:104BA000F3FF29000520F6F7EFFF29000620F6F7AE
:104BB000EBFF29000720F6F7E7FF29000820F6F7AA
:104BC000E3FF0020F6F7AFFF0120F6F7B5FE00285F
:104BD00002D0F6F74AFD3CE00820F6F7ADFE0028CB
:104BE00010D03B20F7F7D9FE216B814207D0216B13
:104BF0003B20F7F7F1FE00200421F5F7B8F9F6F7AE
:104C000034FD26E00220F6F792FE00280ED0206B3D
:104C1000012802D1032020631BE0206B032802D16E
:104C20000020206315E00120206312E00420F6F745
:104C30007EFE00280DD0206B032802D101202063C6
:104C400007E0206B012802D10020206301E003204F
:104C500020630DB030BD00000000000040D3030011
:104C600080D403001CE90100A0D4030028E901005E
:104C700034E9010040E901004CE9010020D50300BE
:104C800058E9010064E9010070E901007CE90100D4
:104C9000E8EC010080D90300A0D9030080E60300FE
:104CA00010B59CB0040070200021F5F760F90420D5
:104CB000F6F71AFCDFF8303BDFF8302B1621684698
:104CC000F6F787FB1622A4A106A8F6F727FA162204
:104CD000A2A10DF12E00F6F721FA1622A0A111A82B
:104CE000F6F71CFA16229FA10DF15A00F6F716FAF4
:104CF0000320F6F714FF0420F6F769FF0020F6F70B
:104D000022FC401CF6F70FFF69460020F6F73CFF37
:104D100006A90120F6F738FF0DF12E010220F6F763
:104D200033FF11A90320F6F72FFF0DF15A010420DC
:104D3000F6F72AFF0120F6F7FFFD002802D0F6F76C
:104D400094FC32E00820F6F7F7FD00282AD0012075
:104D5000F6F7F9FB002806D1012001F033F82063B3
:104D60000120606417E0012806D1022001F02AF832
:104D70002063022060640EE0022806D103206064F4
:104D8000032001F01FF8206305E004206064042084
:104D900001F018F8206301214220F6F70EFC206B89
:104DA000E06302E00420F6F778FC1CB010BD30B5DB
:104DB00091B0040070200021F5F7D9F80220F6F731
:104DC00093FBDFF8243ADFF8282A16216846F6F725
:104DD00000FB69460020F6F7D7FE0320F6F79FFE9A
:104DE0000420F6F7F4FE1622B6A106A8F6F796F907
:104DF0001622B5A10DF12E00F6F790F90020F6F776
:104E0000A2FB401CF6F78FFE06A90120F6F7BCFEB8
:104E10000DF12E010220F6F7B7FEACA52900032004
:104E2000F6F7B2FE29000420F6F7AEFE0820F6F7EA
:104E300083FD002818D00120F6F785FB002806D155
:104E400009206064092000F0BDFF206305E00A200E
:104E500060640A2000F0B6FF206301214220F6F7CB
:104E6000ACFB206BE0630AE00120F6F765FD00284B
:104E700002D0F6F7FAFB02E00220F6F70EFC11B0C2
:104E800030BD30B591B0040070200021F5F76FF807
:104E90000220F6F729FBDFF85039DFF8642B1621E2
:104EA0006846F6F796FA69460020F6F76DFE03208D
:104EB000F6F735FE0420F6F78AFE0020F6F743FBEE
:104EC000401CF6F730FE82A2162106A8F6F781FAFA
:104ED00080A216210DF12E00F6F77BFA06A901201B
:104EE000F6F752FE0DF12E010220F6F74DFE77A5E2
:104EF00029000320F6F748FE29000420F6F744FEB7
:104F00000820F6F719FD002818D00120F6F71BFB42
:104F1000002806D10B2060640B2000F053FF2063B3
:104F200005E00C2060640C2000F04CFF20630121A0
:104F30004220F6F742FB206BE0630AE00120F6F71F
:104F4000FBFC002802D0F6F790FB02E00220F6F707
:104F5000A4FB11B030BD000049310000493200000F
:104F6000493300004934000070B59CB00400F7F7E5
:104F7000C6FD012801D1042500E002257020002192
:104F8000F4F7F5FF0420F6F7AFFADFF85C38DFF846
:104F9000742A162116A8F6F71CFA4FA216216846A5
:104FA000F6F717FA4DA216210DF11600F6F711FAD1
:104FB000F7F7A5FD01280BD149A216210BA8F6F79A
:104FC00008FA48A216210DF14200F6F702FA0BE0AA
:104FD0003EA6320016210BA8F6F7FBF93200162187
:104FE0000DF14200F6F7F5F90320F6F798FD0420DD
:104FF000F6F7EDFD0020F6F7A6FA401CF6F793FD54
:1050000016A90020F6F7C0FD69460120F6F7BCFDA1
:105010000DF116010220F6F7B7FD0BA90320F6F7F4
:10502000B3FD0DF142010420F6F7AEFD0120F6F7C5
:1050300083FC002802D0F6F718FB41E00820F6F7C1
:105040007BFC002839D00120F6F77DFA002806D134
:10505000052000F0B7FE20630520606426E00128EB
:1050600011D1F7F74CFD012806D1062000F0AAFE69
:1050700020630620606419E0082000F0A3FE20638E
:105080000820606412E002280AD1F7F738FD0128F1
:1050900006D1072000F096FE20630720606405E03B
:1050A000082000F08FFE2063082060640121422068
:1050B000F6F783FA206BE06302E02800F6F7EDFADA
:1050C0001CB070BD453100004532000000000000FA
:1050D00020490000204500005331000053320000F9
:1050E000533300005334000070B58EB00400042028
:1050F000F6F715FD70200021F4F739FF02A9606C66
:1051000000F030FDDFF8540A009002ABDFF8502ABF
:10511000162108A8F6F75DF908A90020F6F734FD76
:10512000226B162102A8F9F7D1F802A90120F6F79F
:105130002BFD0CA631000220F6F726FD31000320DE
:10514000F6F722FD31000420F6F71EFD206B002843
:1051500002D0206B202807D33200162102A8F6F7D0
:1051600038F90CE000000000206BF9F7C6F80500E4
:105170002B00DFF8D42A162102A8F6F72AF902A993
:105180000520F6F701FD31000620F6F7FDFC3100A1
:105190000720F6F7F9FC31000820F6F7F5FC0020AF
:1051A000F6F7C1FC0420F6F712FD0820F6F7C4FB61
:1051B000002800F02581206BE16B884229D0606CCB
:1051C00000F06CFD050015F0C005206BF9F79EF8A6
:1051D0000543206B0C2807D0206B0D2804D0206BD2
:1051E0000E2801D035F04005206B00280BD0206B35
:1051F000022808D0206B032805D0206B052802D098
:10520000206B062801D135F080052900606C00F084
:1052100090FDF7F774FC012840F0C880002060631F
:10522000206B192808D0206B1A2805D0206B0F2876
:1052300002D0206B10283CD1606C012806D12900D7
:10524000022000F076FD01206063AFE0606C03286F
:1052500006D12900042000F06CFD01206063A5E068
:10526000606C052806D12900062000F062FD0120AF
:1052700060639BE0606C072806D12900082000F0DD
:1052800058FD0120606391E0606C092806D1290077
:105290000A2000F04EFD0120606387E0606C0B285F
:1052A00040F0848029000C2000F043FD0120606361
:1052B0007CE0606C012811D1022000F0EFFC30F09E
:1052C000C000102805D0112803D00B2801D00A28CF
:1052D0006CD100212A20F7F77FFB67E0606C032880
:1052E00011D1042000F0DAFC30F0C000102805D005
:1052F000112803D00B2801D00A2857D100212E20D5
:10530000F7F76AFB52E0606C092811D10A2000F01F
:10531000C5FC30F0C000102805D0112803D00B28A0
:1053200001D00A2842D100213220F7F755FB3DE099
:10533000606C052811D1062000F0B0FC30F0C000F0
:10534000102805D0112803D00B2801D00A282DD110
:1053500000212220F7F740FB28E0606C072811D1DC
:10536000082000F09BFC30F0C000102805D0112868
:1053700003D00B2801D00A2818D100212620F7F7E6
:105380002BFB13E0606C0B2810D10C2000F086FC86
:1053900030F0C000102805D0112803D00B2801D010
:1053A0000A2803D100213620F7F716FB002004213C
:1053B000F4F7DDFD206B00281FD0206B02281CD0E5
:1053C000206B032819D0206B052816D0206B0628E7
:1053D00013D0606C00F062FC10F08000002802D056
:1053E0000120206301E00020206302214320F6F722
:1053F000E4F8206BE0630EB070BDF6F736F9FAE71B
:105400000120F6F799FA002802D0F6F72EF9F2E714
:10541000F7F775FB01285BD1606C02280ED0606C39
:1054200004280BD0606C062808D0606C082805D0D2
:10543000606C0A2802D0606C0C2849D1606C02288C
:1054400004D1012000F0BEFC050026E0606C0428B9
:1054500004D1032000F0B6FC05001EE0606C0A28B1
:1054600004D1092000F0AEFC050016E0606C0628AF
:1054700004D1052000F0A6FC05000EE0606C0828B1
:1054800004D1072000F09EFC050006E0606C0C28AB
:1054900003D10B2000F096FC0500192D05D01A2D24
:1054A00003D00F2D01D0102D04D125630120F6F774
:1054B0008EFBA0E7206B192808D0206B1A2805D096
:1054C000206B0F2802D0206B102801D10020206310
:1054D0000020019001200090012300221F21206B59
:1054E000F6F74EF92063F7F70AFB012840F01E811A
:1054F000606C0B2836D1206B18281BD0206B11282C
:1055000018D0206B122815D0206B132812D0206BD6
:1055100014280FD0206B15280CD0206B0E2809D032
:10552000206B1D2806D0206B1C2803D0206B182868
:105530007FF461AF00200190012000900123002240
:105540001F21206BF6F71CF920630220F6F7EFF914
:105550000028D0D10420F6F7E5F90028CBD10020AF
:105560002063C8E7606C0C2842D1206B182827D034
:10557000206B112824D0206B122821D0206B1328F7
:105580001ED0206B14281BD0206B0F2818D0206B46
:10559000102815D0206B152812D0206B0E280FD0A4
:1055A000206B1D280CD0206B192809D0206B1A28DD
:1055B00006D0206B1C2803D0206B18287FF41BAF6B
:1055C0000020019001200090012300221F21206B68
:1055D000F6F7D6F820630220F6F7A9F90028C4D11F
:1055E0000420F6F79FF90028BFD100202063BCE714
:1055F000606C02280BD0606C042808D0606C062810
:1056000005D0606C082802D0606C0A284ED1206B4F
:10561000112833D0206B122830D0206B13282DD0C6
:10562000206B14282AD0206B0F2827D0206B10283D
:1056300024D0206B152821D0206B0E281ED0206B83
:105640001D281BD0206B192818D0206B1A2815D0C4
:10565000206B1C2812D0206B18280FD0206B032839
:105660000CD0206B022809D0206B062806D0206BB6
:10567000052803D0206B18287FF4BDAE00200190D0
:1056800001200090012300221F21206BF6F778F8FB
:1056900020630220F6F74BF90028B8D10420F6F772
:1056A00041F90028B3D100202063B0E7206B112816
:1056B00024D0206B122821D0206B13281ED0206B01
:1056C00014281BD0206B152818D0206B0E2815D05D
:1056D000206B1D2812D0206B1C280FD0206B18289F
:1056E0000CD0206B032809D0206B022806D0206B39
:1056F000062803D0206B05287FF47DAE00200190A2
:1057000001200090012300221F21206BF6F738F8BA
:1057100020630220F6F70BF90028C7D10420F6F722
:1057200001F90028C2D100202063BFE7F7F7EFF9A5
:10573000012803D0F7F723FA012837D1206B02287C
:1057400015D0206B032812D0206B05280FD0206BBA
:1057500006280CD0206B092809D0206B0D2806D014
:10576000206B0B2803D0206B1B287FF444AE002055
:10577000019001200090012300221F21206BF5F7EA
:10578000FFFF20630220F6F7D2F80028D6D10420CC
:10579000F6F7C8F80028D1D100202063CEE7042016
:1057A000F6F7C0F8002801D100202063206B022802
:1057B00009D0206B032806D0206B052803D0206B6E
:1057C00006287FF418AE00200190012000900123EC
:1057D00000221F21206BF5F7D3FF20630220F6F78C
:1057E000A6F80028E2D1DAE780D4030088E90100B6
:1057F00094E9010038B58EB0040070200021F4F760
:10580000B6FB02A9606C00F0ADF902ABDFF87424BE
:10581000162108A8F5F7DDFD206B002806D1162219
:10582000DFF8641402A8F5F779FC05E01622DFF82A
:105830005C1402A8F5F772FC0420F6F770F9042056
:10584000F6F7C5F908A90020F6F79EF902A901208C
:10585000F6F79AF96CA529000220F6F795F92900C8
:105860000320F6F791F929000420F6F78DF92900B5
:105870000520F6F789F929000620F6F785F92900B1
:105880000720F6F781F929000820F6F77DF90020B6
:10589000F6F749F90820F6F74FF800286CD0606C4D
:1058A00000F0FCF90500206BE16B884207D0206B0B
:1058B000002802D135F0800501E055F0800529006F
:1058C000606C00F036FAF7F71AF9012831D1606BF5
:1058D00000282ED0606C012804D12900022000F09D
:1058E00028FA26E0606C032804D12900042000F087
:1058F00020FA1EE0606C052804D12900062000F083
:1059000018FA16E0606C072804D12900082000F07E
:1059100010FA0EE0606C092804D129000A2000F07A
:1059200008FA06E0606C0B2803D129000C2000F077
:1059300000FA00200421F4F71AFB606C00F042FA30
:105940000C2803D00D2801D00E2812D1606C00F075
:10595000A5F910F04000002802D00120206301E0EA
:1059600000202063206BE06302214420F5F725FE30
:1059700043E0F5F77AFE40E00120F5F7DDFF00286F
:1059800002D0F5F772FE38E0F7F7B9F8012820D118
:10599000606C00F017FA616C02290ED0616C04296A
:1059A0000BD0616C062908D0616C082905D0616CA8
:1059B0000A2902D0616C0C290BD1192805D01A28AC
:1059C00003D00F2801D0102803D10120F6F7FFF8EB
:1059D00013E000200190012000900123002201210A
:1059E000206BF5F7CDFE2063606C00F057F930F0C6
:1059F000C000172801D1002020630FB030BD000087
:105A0000F0EC0100A0E901000000000038B58EB004
:105A1000040070200021F4F7AAFA02A9606C00F0DB
:105A2000A1F802AB9A4A162108A8F5F7D2FC206B20
:105A3000002805D11622974902A8F5F76FFB04E06C
:105A40001622954902A8F5F769FB0420F6F767F8D6
:105A50000420F6F7BCF808A90020F6F795F802A98B
:105A60000120F6F791F879A529000220F6F78CF8C5
:105A700029000320F6F788F829000420F6F784F8B7
:105A800029000520F6F780F829000620F6F77CF8B3
:105A900029000720F6F778F829000820F6F774F8AF
:105AA0000020F6F740F80820F5F746FF002819D047
:105AB000606C00F0F3F80100206BE26B904207D0BD
:105AC000206B002802D131F0400101E051F040018B
:105AD000606C00F02EF900200421F4F748FAF5F785
:105AE000C4FD38E00120F5F727FF002802D0F5F7C4
:105AF000BCFD30E0F7F703F8012821D1606C0228E3
:105B00000ED0606C04280BD0606C062808D0606C46
:105B1000082805D0606C0A2802D0606C0C280FD1D0
:105B2000206B192808D0206B1A2805D0206B0F286D
:105B300002D0206B102803D10120F6F748F80AE0C4
:105B40000020019001200090012300220121206B00
:105B5000F5F716FE20630FB030BD000040D80300FB
:105B6000F8EC010010B50C00012805D138A2042181
:105B70002000F5F72EFC66E0022805D135A20421AD
:105B80002000F5F726FC5EE0032805D132A20421AF
:105B90002000F5F71EFC56E0042805D12FA20421B1
:105BA0002000F5F716FC4EE0092805D12CA20421AF
:105BB0002000F5F70EFC46E00A2805D129A20421B1
:105BC0002000F5F706FC3EE0052805D126A20421B9
:105BD0002000F5F7FEFB36E0062805D123A20421BC
:105BE0002000F5F7F6FB2EE0072805D120A20421BE
:105BF0002000F5F7EEFB26E008280FD1F6F77FFF2F
:105C0000012805D11BA204212000F5F7E2FB1AE0D0
:105C100016A204212000F5F7DCFB14E00B2805D1C7
:105C200015A204212000F5F7D4FB0CE00C2805D1C7
:105C300012A204212000F5F7CCFB04E010A20421FD
:105C40002000F5F7C6FB10BD00ED010000000000CC
:105C50004931000049320000493300004934000056
:105C6000453100004532000053310000533200003E
:105C70005333000053340000490000004500000089
:105C800045720000ACE9010040D9030060D903006F
:105C900008ED010080E60300E0D9030080B501288B
:105CA00003D12820F6F779FE42E0022803D12A200A
:105CB000F6F773FE3CE0032803D12C20F6F76DFEC7
:105CC00036E0042803D12E20F6F767FE30E00528E1
:105CD00003D12020F6F761FE2AE0062803D1222016
:105CE000F6F75BFE24E0072803D12420F6F755FEE3
:105CF0001EE0082803D12620F6F74FFE18E00928F9
:105D000003D13020F6F749FE12E00A2803D13220F1
:105D1000F6F743FE0CE00B2803D13420F6F73DFEE6
:105D200006E00C2803D13620F6F737FE00E000200D
:105D300002BD80B5012803D12820F6F74DFE40E0D2
:105D4000022803D12A20F6F747FE3AE0032803D1C0
:105D50002C20F6F741FE34E0042803D12E20F6F77C
:105D60003BFE2EE0052803D12020F6F735FE28E083
:105D7000062803D12220F6F72FFE22E0072803D1C0
:105D80002420F6F729FE1CE0082803D12620F6F788
:105D900023FE16E00B2803D13420F6F71DFE10E099
:105DA0000C2803D13620F6F717FE0AE0092803D1A4
:105DB0003020F6F711FE04E00A2802D13220F6F76F
:105DC0000BFE01BD80B5FFF769FF30F0C000F8F7AA
:105DD0001BFBC0B202BD000030B591B004007020C2
:105DE0000021F4F7C4F80220F5F77EFBDFF8B434A5
:105DF000DFF8B42416216846F5F7EBFA8FA21621D6
:105E000006A8F5F7E6FA8EA216210DF12E00F5F799
:105E1000E0FA0320F5F783FE0420F5F7D8FE002012
:105E2000F5F791FB401CF5F77EFE69460020F5F77B
:105E3000ABFE06A90120F5F7A7FE0DF12E01022009
:105E4000F5F7A2FECAA529000320F5F79DFE29005B
:105E50000420F5F799FE0120F5F76EFD002802D029
:105E6000F5F703FC24E00820F5F766FD00281CD0B8
:105E70000120F5F768FB002808D10D206064482058
:105E8000F6F78BFD30F0C000206307E00E20606461
:105E90004920F6F782FD30F0C00020630121462042
:105EA000F5F78BFB206BE06302E00220F5F7F5FBD2
:105EB00011B030BD38B58EB0040070200021F4F769
:105EC00056F80420F5F72BFE606C0D2808D1DFF89A
:105ED000DC33DFF8DC23162108A8F5F77AFA07E0AF
:105EE000DFF8C833DFF8CC23162108A8F5F771FADC
:105EF00008A90020F5F748FE226BD2B2162102A8AD
:105F0000F8F701FB02A90120F5F73EFE98A529004C
:105F10000220F5F739FE29000320F5F735FE2900A8
:105F20000420F5F731FE226BDFF88C1302A8F5F799
:105F300045FA02A90520F5F727FE29000620F5F706
:105F400023FE29000720F5F71FFE29000820F5F79A
:105F50001BFE0020F5F7E7FD0420F5F738FE0820CA
:105F6000F5F7EAFC002853D0206BE16B88421FD084
:105F7000606C0D2806D14820F6F70FFD010011F0E6
:105F8000800105E04920F6F708FD010011F08001CD
:105F9000206B0143606C0D2803D14820F6F71CFDEF
:105FA00002E04920F6F718FD00200821F3F7DFFF93
:105FB000206B092810D102214820F5F7FEFA606C09
:105FC0000D2804D14A20F6F7E8FC206333E04B208B
:105FD000F6F7E3FC20632EE002214720F5F7EDFA07
:105FE000606C0D2805D14820F6F7D7FC10F0800032
:105FF00004E04920F6F7D1FC10F08000002802D020
:106000000120206301E000202063206BE06312E0A8
:106010000120F5F791FC002802D0F5F726FB0AE0F5
:106020000020019001200090012300220F21206B0D
:10603000F5F7A6FB20630FB030BD00004F31000024
:106040004F32000038B58EB0040070200021F3F705
:106050008EFF606C0D2806D1984B954A162108A832
:10606000F5F7B7F905E0954B924A162108A8F5F720
:10607000B0F9236B924A162102A8F5F7AAF9042079
:10608000F5F74DFD0420F5F7A2FD0020F5F74BFDD7
:1060900008A90020F5F778FD02A90120F5F774FDA5
:1060A00033A529000220F5F76FFD29000320F5F73D
:1060B0006BFD29000420F5F767FD29000520F5F7A1
:1060C00063FD29000620F5F75FFD29000720F5F79D
:1060D0005BFD29000820F5F757FD0820F5F72CFC9B
:1060E00000282FD0206BE16B88420FD0606C0D2808
:1060F00004D1216B4A20F6F76FFC03E0216B4B20A3
:10610000F6F76AFC00200821F3F731FF022147204F
:10611000F5F753FA606C0D2805D14820F6F73DFCE1
:1061200010F0800004E04920F6F737FC10F0800002
:10613000002802D00120206301E000202063206BB2
:10614000E06312E00120F5F7F7FB002802D0F5F735
:106150008CFA0AE001200190002000900123012226
:10616000F021206BF5F70CFB20630FB030BD000071
:106170000000000038B58EB0040070200021F3F755
:10618000F6FE606C0D2805D14E4A162108A8F5F7D9
:1061900020F904E04C4A162108A8F5F71AF9206BFB
:1061A000002805D11622494902A8F4F7B7FF04E0F8
:1061B0001622474902A8F4F7B1FF0420F5F7AFFC17
:1061C0000420F5F704FD0020F5F7ADFC08A9002038
:1061D000F5F7DAFC02A90120F5F7D6FC30A5290075
:1061E0000220F5F7D1FC29000320F5F7CDFC2900AA
:1061F0000420F5F7C9FC29000520F5F7C5FC2900A6
:106200000620F5F7C1FC29000720F5F7BDFC2900A1
:106210000820F5F7B9FC0120F5F78EFB002802D025
:10622000F5F723FA39E00820F5F786FB002829D096
:10623000206BE16B884222D0606C0D2806D148208B
:10624000F6F7ABFB010031F0800105E04920F6F7DD
:10625000A4FB010031F08001206B002801D051F037
:106260008001606C0D2803D14820F6F7B5FB02E0F1
:106270004920F6F7B1FB00200821F3F778FEF5F787
:10628000F4F90AE00020019001200090012300228F
:106290000121206BF5F774FA20630FB030BD0000C8
:1062A00000000000A0D40300C4E9010040D80300AE
:1062B00040EE010048EE010050EE010020D903003D
:1062C00058EE0100D0E90100DCE9010040D90300EB
:1062D00060D9030010B59CB0040070200021F3F7D2
:1062E00046FE0420F5F700F9DFF80C39A8A21621C4
:1062F0006846F5F76EF8DFF80439DFF8042916214F
:1063000006A8F5F766F8DFF8FC38DFF8FC28162158
:106310000DF12E00F5F75DF8DFF8F038DFF8F02822
:10632000162111A8F5F755F8DFF8E838DFF8E82866
:1063300016210DF15A00F5F74CF80320F5F7EFFBA5
:106340000420F5F744FC0020F5F7FDF8401CF5F7B4
:10635000EAFB69460020F5F717FC06A90120F5F7CE
:1063600013FC0DF12E010220F5F70EFC11A90320FC
:10637000F5F70AFC0DF15A010420F5F705FC082099
:10638000F5F7DAFA002826D00120F5F7DCF8002826
:1063900004D101214A20F5F710F919E0012804D1B0
:1063A00001215220F5F709F912E0022808D1012154
:1063B0005A20F5F702F95420F6F7EFFA206307E0C8
:1063C00001215B20F5F7F9F85C20F6F7E6FA206387
:1063D000206BE0630AE00120F5F7AEFA002802D056
:1063E000F5F743F902E00420F5F757F91CB010BDAA
:1063F00078B5A7B0040070200021F3F7B8FD06209F
:10640000F5F772F8DFF8F43761A216216846F4F761
:10641000E0FFDFF80838DFF8E827162106A8F4F7D0
:10642000D8FFDFF8FC37DFF8E02716210DF12E004A
:10643000F4F7CFFFDFF8EC37DFF8D427162111A8E7
:10644000F4F7C7FFDFF8E037DFF8CC2716210DF1AE
:106450005A00F4F7BEFFDFF8D437DFF8D42716214F
:106460001CA8F4F7B6FFDFF8CC37DFF8CC271621ED
:106470000DF18600F4F7ADFF0320F5F750FB042083
:10648000F5F7A5FB0020F5F75EF8401CF5F74BFB90
:1064900069460020F5F778FB0220F5F754F805006F
:1064A000162606A806FB05F101440120F5F76CFB52
:1064B00006A806FB05F1084410F116010220F5F7C5
:1064C00063FB06A806FB05F1084410F12C0103202C
:1064D000F5F75AFB06A87543284410F14201042041
:1064E000F5F752FB0820F5F727FA002842D00120E3
:1064F000F5F729F8002808D101214B20F5F75DF8C0
:106500001620F6F74AFA20633FE0012808D101215E
:106510004C20F5F752F81020F6F73FFA206334E0EC
:10652000022808D101214E20F5F747F80E20F6F792
:1065300034FA206329E0032808D101214F20F5F720
:106540003CF81C20F6F729FA20631EE0042808D145
:1065500001215020F5F731F80420F6F71EFA2063E8
:1065600013E001215120F5F728F80620F6F715FA77
:1065700020630AE00120F5F7DFF9002802D0F5F7E3
:1065800074F802E00620F5F788F828B070BD000026
:106590002573000038B58EB0040070200021F3F799
:1065A000E6FC1622DFF8941608A8F4F7B7FD236B73
:1065B0009CA2162102A8F4F70CFF0420F5F7AFFA0D
:1065C0000420F5F704FB0020F5F7ADFA08A9002038
:1065D000F5F7DAFA02A90120F5F7D6FAD0A52900D5
:1065E0000220F5F7D1FA29000320F5F7CDFA2900AA
:1065F0000420F5F7C9FA29000520F5F7C5FA2900A6
:106600000620F5F7C1FA29000720F5F7BDFA2900A1
:106610000820F5F7B9FA0820F5F78EF9002810D010
:106620001620F6F7BAF9216B814207D0216B1620AC
:10663000F6F7D2F900200221F3F799FCF5F715F8E7
:1066400012E00120F5F778F9002802D0F5F70DF8EF
:106650000AE00020019001200090012301220A217C
:10666000206BF5F78DF820630FB030BD38B58EB0D4
:10667000040070200021F3F77AFC1622DFF8C01521
:1066800008A8F4F74BFD236BDFF8B825162102A804
:10669000F4F79FFE0420F5F742FA08A90020F5F769
:1066A00073FA02A90120F5F76FFA9DA529000220CF
:1066B000F5F76AFA29000320F5F766FA29000420A5
:1066C000F5F762FA29000520F5F75EFA29000620A1
:1066D000F5F75AFA29000720F5F756FA290008209D
:1066E000F5F752FA0020F5F71EFA0820F5F724F91D
:1066F000002816D01020F6F750F9216B814207D000
:10670000216B1020F6F768F900200221F3F72FFC27
:1067100002214D20F4F751FF0020F6F73EF92063E7
:1067200012E00120F5F708F9002802D0F4F79DFFE8
:106730000AE0012001900020009001230022C821DE
:10674000206BF5F71DF820630FB030BD38B58EB063
:10675000040070200021F3F70AFC1622DFF8E81489
:1067600008A8F4F7DBFC236BB1A2162102A8F4F70A
:1067700030FE0420F5F7D3F90420F5F728FA08A92C
:106780000020F5F701FA02A90120F5F7FDF964A54B
:1067900029000220F5F7F8F929000320F5F7F4F9AC
:1067A00029000420F5F7F0F929000520F5F7ECF9A8
:1067B00029000620F5F7E8F929000720F5F7E4F9A4
:1067C00029000820F5F7E0F90020F5F7ACF90820DA
:1067D000F5F7B2F8002810D00020F6F7DEF8216BAC
:1067E000814207D0216B0020F6F7F6F80020022145
:1067F000F3F7BDFBF4F739FF12E00120F5F79CF841
:10680000002802D0F4F731FF0AE0002001900020B8
:106810000090012301220321206BF4F7B1FF2063D4
:106820000FB030BD2532640038B58EB00400702042
:106830000021F3F79CFB1622DFF8101408A8F4F7E8
:106840006DFC236BB1A2162102A8F4F7C2FD04204F
:10685000F5F765F9F6F753F9012803D10120F5F7AB
:10686000B6F902E00420F5F7B2F908A90020F5F71F
:106870008BF902A90120F5F787F929A52900022043
:10688000F5F782F929000320F5F77EF929000420A5
:10689000F5F77AF929000520F5F776F929000620A1
:1068A000F5F772F929000720F5F76EF9290008209D
:1068B000F5F76AF90020F5F736F90820F5F73CF806
:1068C000002810D00E20F6F768F8216B814207D01F
:1068D000216B0E20F6F780F800200221F3F747FB2A
:1068E000F4F7C3FE1AE00120F5F726F8002806D0D9
:1068F000F6F705F9012811D0F4F7B7FE0EE0F6F728
:10690000FEF801280AD00020019000200090012309
:1069100001220A21206BF4F733FF20630FB030BD52
:106920000000000030B58FB0040070200021F3F7A4
:106930001EFB1622C64909A8F4F7F0FB236BC54AD3
:10694000032102A8F4F745FD9DF808008DF80C001E
:1069500003A82E2141709DF8091081700021C1709B
:106960000420F5F7DCF8F6F7CAF8012803D1012076
:10697000F5F72DF902E00420F5F729F909A900201F
:10698000F5F702F903A90120F5F7FEF896A1022018
:10699000F5F7FAF895A529000320F5F7F5F8290091
:1069A0000420F5F7F1F829000520F5F7EDF82900A6
:1069B0000620F5F7E9F829000720F5F7E5F82900A2
:1069C0000820F5F7E1F80020F5F7ADF80820F4F716
:1069D000B3FF00280FD01C20F5F7DFFF216B8142A9
:1069E00007D0216B1C20F5F7F7FF00200221F3F7F9
:1069F000BEFAF4F73AFE0120F4F79EFF002806D015
:106A0000F6F77DF8012811D0F4F72FFE0EE0F6F727
:106A100076F801280AD0012001900020009001237F
:106A200001221E21206BF4F7ABFE20630FB030BDB6
:106A30002564000038B58EB0040070200021F3F703
:106A400096FA1622844908A8F4F768FB236B68A21B
:106A5000162102A8F4F7BDFC0420F5F760F8042025
:106A6000F5F7B5F80020F5F75EF808A90020F5F76E
:106A70008BF802A90120F5F787F85CA52900022010
:106A8000F5F782F829000320F5F77EF829000420A5
:106A9000F5F77AF829000520F5F776F829000620A1
:106AA000F5F772F829000720F5F76EF8290008209D
:106AB000F5F76AF80820F4F73FFF002810D004200B
:106AC000F5F76BFF216B814207D0216B0420F5F7AE
:106AD00083FF00200221F3F74AFAF4F7C6FD12E023
:106AE0000120F4F729FF002802D0F4F7BEFD0AE0E8
:106AF0000020019000200090012301220A21206B38
:106B0000F4F73EFE20630FB030BD00002532640074
:106B100038B58EB0040070200021F3F728FA162251
:106B20004E4908A8F4F7FAFA236B32A2162102A8FC
:106B3000F4F74FFC0420F4F7F2FF0420F5F747F8D0
:106B40000020F4F7F0FF08A90020F5F71DF802A9CE
:106B50000120F5F719F825A529000220F5F714F80A
:106B600029000320F5F710F829000420F5F70CF8A8
:106B700029000520F5F708F829000620F5F704F8A4
:106B800029000720F5F700F829000820F4F7FCFF9A
:106B90000820F4F7D1FE002810D00620F5F7FDFEFE
:106BA000216B814207D0216B0620F5F715FF0020ED
:106BB0000221F3F7DCF9F4F758FD12E00120F4F7B5
:106BC000BBFE002802D0F4F750FD0AE0002001903F
:106BD00000200090012301220A21206BF4F7D0FD50
:106BE00020630FB030BD00002073000000000000E3
:106BF000256400002532640060D3030080D50300C3
:106C0000C0ED0100A0D50300C8ED0100C0F50300F0
:106C1000D0ED010020F70300D8ED0100C0D503003E
:106C2000E0D5030000D6030020D6030040D60300C1
:106C3000E0ED010060D60300E8ED010080D603001E
:106C4000A0D60300F0ED0100C0D60300E0D603009B
:106C500000D70300F8ED010020D7030040D7030060
:106C600078B5A7B0040070200021F3F780F9062062
:106C7000F4F73AFCDFF8703997A216216846F4F76A
:106C8000A8FBDFF86839DFF86829162106A8F4F7B1
:106C9000A0FBDFF86039DFF8602916210DF12E0026
:106CA000F4F797FBDFF85439DFF85429162111A8BF
:106CB000F4F78FFBDFF84C39DFF84C2916210DF182
:106CC0005A00F4F786FBDFF84439DFF8442916212F
:106CD0001CA8F4F77EFBDFF83C39DFF83C291621CD
:106CE0000DF18600F4F775FB0320F4F718FF04207C
:106CF000F4F76DFF0020F4F726FC401CF4F713FFB7
:106D000069460020F4F740FF0220F4F71CFC050060
:106D1000162606A806FB05F101440120F4F734FF0E
:106D200006A806FB05F1084410F116010220F4F74D
:106D30002BFF06A806FB05F1084410F12C010320E7
:106D4000F4F722FF06A87543284410F142010420FD
:106D5000F4F71AFF0820F4F7EFFD002842D00120D5
:106D6000F4F7F1FB002808D101215320F4F725FCAA
:106D70001820F5F712FE20633FE0012808D1012119
:106D80005420F4F71AFC1220F5F707FE206334E0D4
:106D9000022808D101215620F4F70FFC0C20F5F74A
:106DA000FCFD206329E0032808D101215720F4F7D6
:106DB00004FC1A20F5F7F1FD20631EE0042808D139
:106DC00001215820F4F7F9FB0820F5F7E6FD2063D0
:106DD00013E001215920F4F7F0FB0A20F5F7DDFD5F
:106DE00020630AE00120F4F7A7FD002802D0F4F7A1
:106DF0003CFC02E00620F4F750FC28B070BD38B52A
:106E00008EB0040070200021F3F7B1F81622DFF8ED
:106E10000C1808A8F4F782F9236BA0A2162102A887
:106E2000F4F7D7FA0420F4F77AFE0420F4F7CFFE43
:106E30000020F4F778FE08A90020F4F7A5FE02A9C7
:106E40000120F4F7A1FECCA529000220F4F79CFE56
:106E500029000320F4F798FE29000420F4F794FE9B
:106E600029000520F4F790FE29000620F4F78CFE97
:106E700029000720F4F788FE29000820F4F784FE93
:106E80000820F4F759FD002810D01820F5F785FDEB
:106E9000216B814207D0216B1820F5F79DFD002062
:106EA0000221F3F764F8F4F7E0FB12E00120F4F7B5
:106EB00043FD002802D0F4F7D8FB0AE0002001903F
:106EC00000200090012301220A21206BF4F758FCD6
:106ED00020630FB030BD00002573000038B58EB0C0
:106EE000040070200021F3F742F81622DFF8301773
:106EF00008A8F4F713F9236BDFF82827162102A856
:106F0000F4F767FA0420F4F70AFE0420F4F75FFEB2
:106F100008A90020F4F738FE02A90120F4F734FE96
:106F200095A529000220F4F72FFE29000320F4F78D
:106F30002BFE29000420F4F727FE29000520F4F792
:106F400023FE29000620F4F71FFE29000720F4F78E
:106F50001BFE29000820F4F717FE0020F4F7E3FDDC
:106F60000820F4F7E9FC002816D01220F5F715FDEB
:106F7000216B814207D0216B1220F5F72DFD0020F7
:106F80000221F2F7F4FF02215520F4F716FB02204C
:106F9000F5F703FD206312E00120F4F7CDFC002893
:106FA00002D0F4F762FB0AE001200190002000907B
:106FB00001230022C821206BF4F7E2FB20630FB00D
:106FC00030BD38B58EB0040070200021F2F7CFFF3D
:106FD0001622DFF8541608A8F4F7A0F8236B2FA2A6
:106FE000162102A8F4F7F5F90420F4F798FD04201F
:106FF000F4F7EDFD08A90020F4F7C6FD02A9012071
:10700000F4F7C2FD5CA529000220F4F7BDFD2900BC
:107010000320F4F7B9FD29000420F4F7B5FD290099
:107020000520F4F7B1FD29000620F4F7ADFD290095
:107030000720F4F7A9FD29000820F4F7A5FD00209A
:10704000F4F771FD0820F4F777FC002810D0022037
:10705000F5F7A3FC216B814207D0216B0220F5F7E5
:10706000BBFC00200221F2F782FFF4F7FEFA12E0E7
:107070000120F4F761FC002802D0F4F7F6FA0AE0E8
:107080000020019000200090012301220321206BA9
:10709000F4F776FB20630FB030BD000025640000DC
:1070A00038B58EB0040070200021F2F760FF162280
:1070B000DFF8781508A8F4F731F8236BA1A21621A0
:1070C00002A8F4F786F90420F4F729FD0420F4F768
:1070D0007EFD08A90020F4F757FD02A90120F4F76E
:1070E00053FD25A529000220F4F74EFD29000320B9
:1070F000F4F74AFD29000420F4F746FD2900052095
:10710000F4F742FD29000620F4F73EFD2900072090
:10711000F4F73AFD29000820F4F736FD0020F4F7D3
:1071200002FD0820F4F708FC002810D00C20F5F729
:1071300034FC216B814207D0216B0C20F5F74CFC0D
:1071400000200221F2F713FFF4F78FFA12E001207A
:10715000F4F7F2FB002802D0F4F787FA0AE00020E7
:10716000019000200090012301220A21206BF4F7F6
:1071700007FB20630FB030BD0000000030B58FB0BA
:10718000040070200021F2F7F2FE1622DFF8A014AE
:1071900009A8F3F7C3FF236BDFF89824032102A8A3
:1071A000F4F717F99DF808008DF80C0003A82E21BC
:1071B00041709DF8091081700021C1700420F4F71E
:1071C000AEFC0420F4F703FD09A90020F4F7DCFC71
:1071D00003A90120F4F7D8FCC6A10220F4F7D4FCDF
:1071E000C5A529000320F4F7CFFC29000420F4F7FB
:1071F000CBFC29000520F4F7C7FC29000620F4F792
:10720000C3FC29000720F4F7BFFC29000820F4F78D
:10721000BBFC0020F4F787FC0820F4F78DFB002866
:107220000FD01A20F5F7B9FB216B814207D0216BF3
:107230001A20F5F7D1FB00200221F2F798FEF4F7AF
:1072400014FA0120F4F778FB002802D0F4F70DFAC5
:107250000AE00120019000200090012301221E215C
:10726000206BF4F78DFA20630FB030BD38B58EB0C7
:10727000040070200021F2F77AFE1622DFF8B8131E
:1072800008A8F3F74BFF236B9CA2162102A8F4F782
:10729000A0F80420F4F743FC0420F4F798FC002045
:1072A000F4F741FC08A90020F4F76EFC02A90120C4
:1072B000F4F76AFC90A529000220F4F765FC290088
:1072C0000320F4F761FC29000420F4F75DFC290099
:1072D0000520F4F759FC29000620F4F755FC290095
:1072E0000720F4F751FC29000820F4F74DFC082092
:1072F000F4F722FB002810D00820F5F74EFB216B95
:10730000814207D0216B0820F5F766FB002002219F
:10731000F2F72DFEF4F7A9F912E00120F4F70CFBC7
:10732000002802D0F4F7A1F90AE000200190002023
:107330000090012301220A21206BF4F721FA206337
:107340000FB030BD2532640038B58EB00400702017
:107350000021F2F70CFE1622B84908A8F3F7DEFE6A
:10736000236B66A2162102A8F4F733F80420F4F781
:10737000D6FB0420F4F72BFC0020F4F7D4FB08A97B
:107380000020F4F701FC02A90120F4F7FDFB5AA547
:1073900029000220F4F7F8FB29000320F4F7F4FB9E
:1073A00029000420F4F7F0FB29000520F4F7ECFB9A
:1073B00029000620F4F7E8FB29000720F4F7E4FB96
:1073C00029000820F4F7E0FB0820F4F7B5FA0028BC
:1073D00010D00A20F5F7E1FA216B814207D0216B2A
:1073E0000A20F5F7F9FA00200221F2F7C0FDF4F7C0
:1073F0003CF912E00120F4F79FFA002802D0F4F7DC
:1074000034F90AE0002001900020009001230122BD
:107410000A21206BF4F7B4F920630FB030BD38B502
:107420008EB0040070200021F2F7A1FD16228449DD
:1074300008A8F3F773FE236B30A2162102A8F3F716
:10744000C8FF0420F4F76BFB0420F4F7C0FB002016
:10745000F4F769FB08A90020F4F796FB02A90120C4
:10746000F4F792FB24A529000220F4F78DFB2900F4
:107470000320F4F789FB29000420F4F785FB290099
:107480000520F4F781FB29000620F4F77DFB290095
:107490000720F4F779FB29000820F4F775FB082092
:1074A000F4F74AFA002810D05420F5F776FA216B49
:1074B000814207D0216B5420F5F78EFA0020082175
:1074C000F2F755FDF4F7D1F812E00120F4F734FAA1
:1074D000002802D0F4F7C9F80AE00020019000204B
:1074E0000090012301220521206BF4F749F9206364
:1074F0000FB030BD207300000000000025640000C4
:1075000038B58EB0040070200021F2F730FD4D4BED
:1075100032A2162108A8F3F75CFF236B30A21621D4
:1075200002A8F3F756FF0420F4F7F9FA08A900209F
:10753000F4F72AFB02A90120F4F726FB29A529006C
:107540000220F4F721FB29000320F4F71DFB29009A
:107550000420F4F719FB29000520F4F715FB290096
:107560000620F4F711FB29000720F4F70DFB290092
:107570000820F4F709FB0020F4F7D5FA0820F4F707
:10758000DBF900280ED0206BE16B884207D0216B1D
:107590005C20F5F721FA00200821F2F7E8FCF4F767
:1075A00064F819E00120F4F7C7F9002802D0F4F7D5
:1075B0005CF811E0F5F7A3FA012802D1002020635E
:1075C0000AE00020019001200090012300220A21FE
:1075D000206BF4F7D5F820630FB030BD25730000A1
:1075E0002532640000000000A0D50300C0D50300D0
:1075F00000EE0100E0D5030008EE010000D6030014
:1076000010EE010020D6030018EE010040D6030062
:1076100020EE010060D6030028EE010060D70300D1
:1076200080D7030030EE0100A0D70300C0D70300CD
:10763000E0D7030038EE010000D8030020D8030093
:10764000C0F5030020F7030030B597B0702000218B
:10765000F2F78DFC0320F3F747FF1622DFF89C13A7
:107660006846F3F75BFDDFF89833DFF898231621BF
:1076700006A8F3F7AEFEDFF89033DFF8902316216B
:107680000DF12E00F3F7A5FEE14BE24A162111A8F9
:10769000F3F79FFE0320F4F742FA0420F4F797FA79
:1076A0000020F3F750FF401CF4F73DFA0220F3F7F7
:1076B0004AFF040069460020F4F766FA162506A87A
:1076C00005FB04F101440120F4F75EFA06A805FB6E
:1076D00004F1084410F116010220F4F755FA06A847
:1076E00005FB04F1084410F12C010320F4F74CFAD7
:1076F00006A86C43204410F142010420F4F744FA38
:107700000120F4F719F9002802D0F3F7AEFF2CE0BE
:107710000820F4F711F9002824D00120F3F713FF13
:10772000002809D101215D20F3F747FF3820F5F744
:1077300034F9B949086018E0012809D101215E2017
:10774000F3F73BFF3920F5F728F9B34908600CE05F
:1077500001215F20F3F731FF3A20F5F71EF9AE491A
:10776000086002E00320F3F798FF17B030BD38B58A
:1077700088B070200021F2F7FAFB1622A04902A877
:10778000F3F7CCFC02A90020F4F7FEF90420F4F78B
:10779000C6F9A14C2368A14A162102A8F3F719FEE5
:1077A00002A90120F4F7F0F90420F4F710FA91A5EA
:1077B00029000220F4F7E8F929000320F4F7E4F99E
:1077C00029000420F4F7E0F929000520F4F7DCF99A
:1077D00029000620F4F7D8F929000720F4F7D4F996
:1077E00029000820F4F7D0F90020F4F79CF90820CC
:1077F000F4F7A2F8002810D03820F5F7CEF8216869
:10780000814207D021683820F5F7E6F800200421EE
:10781000F2F7ADFBF3F729FF12E00120F4F78CF843
:10782000002802D0F3F721FF0AE001200190002098
:107830000090012300221E212068F3F7A1FF2060A1
:1078400009B030BD38B58EB070200021F2F78FFB43
:107850000420F4F764F90420F4F7B9F916226A4910
:1078600008A8F3F75BFC08A90020F4F78DF96A4C2F
:1078700023686A4A162102A8F3F7ABFD02A901208A
:10788000F4F782F95BA529000220F4F77DF92900BD
:107890000320F4F779F929000420F4F775F9290099
:1078A0000520F4F771F929000620F4F76DF9290095
:1078B0000720F4F769F929000820F4F765F900209A
:1078C000F4F731F90820F4F737F8002810D0392000
:1078D000F5F763F82168814207D021683920F5F770
:1078E0007BF800200421F2F742FBF3F7BEFE12E022
:1078F0000120F4F721F8002802D0F3F7B6FE0AE0E1
:10790000012001900020009001230022F021206836
:10791000F3F736FF20600FB030BD38B58EB0702061
:107920000021F2F724FB3A4B33A2162108A8F3F703
:1079300050FD394C2368394A162102A8F3F749FD56
:107940000420F4F7ECF80420F4F741F90020F4F7F0
:10795000EAF808A90020F4F717F902A90120F4F7C2
:1079600013F924A529000220F4F70EF929000320B9
:10797000F4F70AF929000420F4F706F92900052094
:10798000F4F702F929000620F4F7FEF82900072091
:10799000F4F7FAF829000820F4F7F6F80120F3F7D5
:1079A000CBFF002802D0F3F760FE20E00820F3F7B9
:1079B000C3FF002810D03A20F4F7EFFF216881427E
:1079C00007D021683A20F5F707F800200421F2F7E4
:1079D000CEFAF3F74AFE0AE0012001900020009061
:1079E00001230022F0212068F3F7CAFE20600FB0C7
:1079F00030BD0000000000002573000080F103008E
:107A000040D40300C0EE010060D40300C8EE0100C2
:107A100060D50300D0EE010078110020D8EE0100FF
:107A20002DE9F841A7B0050048200021F2F79FFAA0
:107A30001622DFF8681921A8F3F770FB21A90020AE
:107A4000F4F7A2F85720F4F7A8FF0400002C06D1A1
:107A5000DFF84C2916216846F3F7BBFC06E023004B
:107A6000DFF8402916216846F3F7B3FC002C0CD050
:107A70005620F4F792FF800707D5DFF82C2916214E
:107A80000DF11600F3F7A5FC06E0DFF8202916211A
:107A90000DF11600F3F79DFC002C0BD05620F4F7E7
:107AA0007CFF400706D5DFF8082916210BA8F3F75D
:107AB00090FC05E0DFF8FC2816210BA8F3F789FC01
:107AC000002C0CD05620F4F768FF000707D5DFF82C
:107AD000E82816210DF14200F3F77BFC06E0DFF801
:107AE000DC2816210DF14200F3F773FC012C12D1B2
:107AF0000626DFF8CC38DFF8CC28162116A8F3F7D5
:107B000068FCDFF8C438DFF8C42816210DF16E00D8
:107B1000F3F75FFC0CE0B5A63200162116A8F3F7C8
:107B200058FC320016210DF16E00F3F752FC0426CA
:107B30003000F3F7D9FC0320F3F7F1FF0420F4F74A
:107B400046F80020F3F7FFFC401CF3F7ECFF02209F
:107B5000F3F7F9FC07005FF01608684608FB07F129
:107B600001440120F4F710F8684608FB07F10844C7
:107B700010F116010220F4F707F8684608FB07F138
:107B8000084410F12C010320F3F7FEFF684608FBC0
:107B900007F7384410F142010420F3F7F5FF012004
:107BA000F3F7CAFE002802D0F3F75FFD8CE008204F
:107BB000F3F7C2FE002800F084800120F3F7C3FC35
:107BC000002808D101217A20F3F7F7FC5720F4F7B9
:107BD000E4FE286372E0012828D1F4F790FF012821
:107BE00004D101210F20F3F7E8FC67E0012C01D05C
:107BF000032C16D101217B20F3F7DFFC5620F4F78C
:107C0000CCFE800702D40020286357E05820F4F708
:107C1000C4FE022802D1022028634FE0012028631D
:107C20004CE001218020F3F7C8FC47E0022820D176
:107C3000F4F765FF012804D101210F20F3F7BDFC03
:107C40003CE0002C10D0092C0ED201217D20F3F74E
:107C5000B4FC5620F4F7A1FE400702D400202863AC
:107C60002CE00120286329E001218020F3F7A5FC06
:107C700024E0032817D1002C10D0082C0ED20121AB
:107C80007C20F3F79AFC5620F4F787FE000702D415
:107C90000020286312E0012028630FE001218020EA
:107CA000F3F78BFC0AE0042804D101217E20F3F7CE
:107CB00084FC03E001218120F3F77FFC286BE8635B
:107CC00002E03000F3F7E9FC28B0BDE8F08138B5F8
:107CD0008EB0040048200021F2F749F9DFF8BC36E5
:107CE000DFF8EC26162108A8F3F773FB206B0028B9
:107CF00007D1DFF8E03694A2162102A8F3F769FB5A
:107D000006E0236BDFF8D026162102A8F3F761FB0B
:107D10000420F3F704FF0420F3F759FF08A900201B
:107D2000F3F732FF02A90120F3F72EFFD3A52900B4
:107D30000220F3F729FF29000320F3F725FF29008C
:107D40000420F3F721FF29000520F3F71DFF290088
:107D50000620F3F719FF29000720F3F715FF290084
:107D60000820F3F711FF0020F3F7DDFE0820F3F7FA
:107D7000E3FD002824D0206BE16B88421DD0216BED
:107D80005720F4F729FE00215620F4F725FE206B3A
:107D900002280ED30020F4F7C5FD0100C80708D55E
:107DA000490849000020F4F7B8FD00204021F2F70F
:107DB000DEF800200821F2F7DAF8F3F756FC12E0BB
:107DC0000120F3F7B9FD002802D0F3F74EFC0AE0DA
:107DD0000020019001200090012300220F21206B40
:107DE000F3F7CEFC20630FB030BD000000000000B0
:107DF00038B58EB0040048200021F2F7B8F804200E
:107E0000F3F78DFE1622DFF8D41508A8F3F786F9EC
:107E100008A90020F3F7B8FE206B002806D116222F
:107E2000DFF8B01502A8F3F779F90FE0206B01280D
:107E300006D11622DFF8A81502A8F3F76FF905E0BE
:107E40001622DFF8A01502A8F3F768F902A90120AD
:107E5000F3F79AFE89A529000220F3F795FE290081
:107E60000320F3F791FE29000420F3F78DFE206B29
:107E7000002804D129000520F3F786FE11E05720E1
:107E8000F4F78BFD012801D1032300E00123DFF883
:107E90005825162102A8F3F79CFA02A90520F3F74A
:107EA00073FE29000620F3F76FFE29000720F3F781
:107EB0006BFE29000820F3F767FE0020F3F733FE7E
:107EC0000420F3F784FE0820F3F736FD002826D0BF
:107ED000206BE16B88421FD05620F4F75EFD010055
:107EE00031F00201206B002801D1012409E0206B50
:107EF000012803D151F00201012402E051F00201F6
:107F000002245620F4F768FD21005820F4F764FDA0
:107F100000200821F2F72BF8F3F7A7FB12E001206D
:107F2000F3F70AFD002802D0F3F79FFB0AE00020D8
:107F3000019001200090012300220221206BF3F721
:107F40001FFC20630FB030BD2573000070B58EB0EC
:107F5000040048200021F2F70AF80420F3F7DFFDBF
:107F60001622DFF8881408A8F3F7D8F808A900202B
:107F7000F3F70AFE5720F4F710FD0500E80701D4D7
:107F80006D1E00E06D1C206B012806D11622DFF863
:107F9000601402A8F3F7C2F805E01622DFF83414E3
:107FA00002A8F3F7BBF802A90120F3F7EDFD33A611
:107FB00031000220F3F7E8FD31000320F3F7E4FD80
:107FC00031000420F3F7E0FD206B002804D13100DC
:107FD0000520F3F7D9FD0AE02B00DFF80C24162169
:107FE00002A8F3F7F6F902A90520F3F7CDFD310059
:107FF0000620F3F7C9FD31000720F3F7C5FD310076
:108000000820F3F7C1FD0020F3F78DFD0420F3F7FE
:10801000DEFD0820F3F790FC002819D05620F4F775
:10802000BCFC0100206BE26B90420ED0206B01285B
:1080300002D151F0040101E031F004015620F4F7BF
:10804000CBFC00200821F1F792FFF3F70EFB12E0C2
:108050000120F3F771FC002802D0F3F706FB0AE0D9
:108060000020019001200090012300220121206BBB
:10807000F3F786FB20630EB070BD00000000000027
:1080800070B58EB0040048200021F1F770FF042085
:10809000F3F745FDD74B9CA2162108A8F3F799F9F1
:1080A00008A90020F3F770FD5720F4F776FC0500CF
:1080B0000835206B012805D11622CD4902A8F3F717
:1080C0002DF804E01622C34902A8F3F727F802A905
:1080D0000120F3F759FDAFA631000220F3F754FD5C
:1080E00031000320F3F750FD31000420F3F74CFD7D
:1080F000206B002804D131000520F3F745FD09E08D
:108100002B00B94A162102A8F3F763F902A905204A
:10811000F3F73AFD31000620F3F736FD3100072072
:10812000F3F732FD31000820F3F72EFD0020F3F7BE
:10813000FAFC0420F3F74BFD0820F3F7FDFB0028C1
:1081400019D05620F4F729FC0100206BE26B904215
:108150000ED0206B012802D151F0080101E031F06E
:1081600008015620F4F738FC00200821F1F7FFFE43
:10817000F3F77BFA12E00120F3F7DEFB002802D0D0
:10818000F3F773FA0AE00020019001200090012328
:1081900000220121206BF3F7F3FA20630EB070BDCB
:1081A00038B58CB0040048200021F1F7E0FE56A558
:1081B000834B2A00162106A8F3F70BF98E4B2A00F1
:1081C00016216846F3F705F90420F3F7A8FC03200D
:1081D000F3F7FDFC0020F3F7A6FC06A90020F3F757
:1081E000D3FC69460120F3F7CFFC6AA529000220E1
:1081F000F3F7CAFC29000320F3F7C6FC290004208A
:10820000F3F7C2FC29000520F3F7BEFC2900062085
:10821000F3F7BAFC29000720F3F7B6FC2900082081
:10822000F3F7B2FC0820F3F787FB00280ED04020BC
:10823000F5F74AFD00208021F1F799FE02217F2009
:10824000F3F7BBF9F4F7CEFF206306E00120F3F764
:1082500073FB002801D0F3F708FA0DB030BD38B534
:108260008CB004001622564906A8F2F757FF634A5D
:1082700016216846F3F7ADF80420F3F750FC002010
:10828000F3F7A5FC06A90020F3F77EFC6946012060
:10829000F3F77AFC3FA529000220F3F775FC2900CB
:1082A0000320F3F771FC29000420F3F76DFC29008B
:1082B0000520F3F769FC29000620F3F765FC290087
:1082C0000720F3F761FC29000820F3F75DFC00208C
:1082D000F3F729FCF4F786FF216B401A40F2D171C5
:1082E00088420ED35FF080700021F5F747FF00222F
:1082F0000023994205D1904203D102218120F3F756
:108300005CF90DB030BD00002573000010B58CB0D5
:1083100021A2162106A8F3F75CF8394A162168460F
:10832000F3F757F80420F3F7FAFB0120F3F74FFCBB
:1083300006A90020F3F728FC69460120F3F724FC86
:1083400014A421000220F3F71FFC21000320F3F7FF
:108350001BFC21000420F3F717FC21000520F3F794
:1083600013FC21000620F3F70FFC21000720F3F790
:108370000BFC21000820F3F707FC0020F3F7D3FBE8
:108380000820F3F7D9FA002801D0F3F76EF90CB002
:1083900010BD0000000000002049440020F103004F
:1083A00018E50100F0E5010004E6010030E50100F8
:1083B00018E6010048E501002CE6010060E5010037
:1083C00080E0030050EB010020F6030058EB0100B1
:1083D00060EB010080E6030068EB010080F403001D
:1083E00040F6030060F6030020E80100A0F403005B
:1083F000E0D9030008E80100E0DA03002CE80100FE
:1084000070EB01002DE9F043E9B00400DFF8680AE1
:108410000021F1F7ACFD00250DE095A216210EA874
:10842000162303FB05F31844F2F7D3FF00205BA9E2
:1084300041F825006D1C0E2DEFD3012601205B9025
:10844000F5F719FD8046F5F700FD0500F5F708FD85
:1084500007005FF0FF30F5F773FE002801D057F0FA
:1084600001075FF002090BE04846F5F73BFA18EA0E
:10847000000F03D05BA840F82690761C19F1010983
:10848000B9F1100FF0D35FF000082AE002A80190C4
:1084900008A8009059F82830DFF8E02916210EA826
:1084A0005FF0160C0CFB08FC6044F2F792FF16E03C
:1084B00070A2162102A8F2F78CFF59F828001028A4
:1084C000E4D302A8009008ABDFF8B42916210EA867
:1084D0005FF0160C0CFB08FC6044F2F77AFF18F111
:1084E0000108B04546D20DF5B67959F82800F5F7E0
:1084F0003AFD162208A9F4F76DFB59F82800F5F7A4
:10850000F1F9054203D159F828100129D0D10742C9
:1085100018D059F82800F5F73FFD00280CD059F87D
:108520002800F5F739FDFF2806D0DFF85829162175
:1085300002A8F2F74EFFC0E74EA2162102A8F2F7FA
:1085400048FFBAE759F82800F5F726FD00280BD0B8
:1085500059F82800F5F720FDFF2805D0A5A216211F
:1085600002A8F2F736FFA8E741A2162102A8F2F707
:1085700030FFA2E73000F2F7B7FF0320F3F7CFFA9E
:108580000420F3F724FB1622DFF8FC1802A8F2F708
:10859000C5FD02A90020F3F7F7FA0020F2F7D3FF98
:1085A000401CF3F7C0FA0220F2F7CDFF07005FF09E
:1085B00016080EA808FB07F101440120F3F7E4FABE
:1085C0000EA808FB07F1084410F116010220F3F78A
:1085D000DBFA0EA808FB07F1084410F12C01032078
:1085E000F3F7D2FA0EA808FB07F7384410F142015E
:1085F0000420F3F7C9FA0120F3F79EF9002802D00E
:10860000F3F733F830E00820F3F796F9002828D084
:108610000120F2F798FF5BA951F820002064206C3C
:10862000F5F7A1FC0600206CF5F75CF9054206D0D1
:10863000162202A93000F4F7CDFA012802D0206CEE
:10864000012811D1206CF5F78EFC102804D10121EE
:108650008820F2F7B2FF07E001218220F2F7ADFF98
:1086600002E03000F3F719F869B0BDE8F0830000CC
:10867000000000002821290078B5A9B00400206C72
:10868000F1F780FC5FF480000021F1F770FC206CB2
:10869000F5F769FC162201A9F4F79CFA002802D12B
:1086A000F2F7E3FFA3E001A80090236CDFF8DC27DA
:1086B000162107A8F2F78DFE07A90020F3F764FA48
:1086C000DFF8CC2716210DA8F2F783FEDFF8C437B8
:1086D000DFF8C42716210DF14A00F2F77AFEDFF821
:1086E000BC37DFF8BC27162118A8F2F772FEDFF8B6
:1086F000B437DFF8B42716210DF17600F2F769FEE2
:10870000DFF8A837DFF8A827162123A8F2F761FEC3
:108710000520F2F7E9FE0320F3F701FA0420F3F74E
:1087200056FA0220F2F70FFF050016260DA806FBE9
:1087300005F101440120F3F727FA0DA806FB05F126
:10874000084410F116010220F3F71EFA0DA806FBEB
:1087500005F1084410F12C010320F3F715FA0DA8D8
:108760007543284410F142010420F3F70DFA00206C
:10877000F2F7E9FE401CF3F7D6F90120F3F7DCF835
:10878000002802D0F2F771FF31E00820F3F7D4F8A7
:10879000002829D00120F2F7D6FE002804D10121BB
:1087A0008320F2F70AFF1CE0012804D10121852073
:1087B000F2F703FF15E0022804D101218420F2F72B
:1087C000FCFE0EE0032804D101218620F2F7F5FE1D
:1087D00007E0206CF5F7E0FB206301218720F2F72A
:1087E000ECFE206BE06302E00520F2F756FF2AB0B2
:1087F00070BD0000282A29002DE9F043CFB0070002
:10880000386CF1F7BFFB5FF480000021F1F7AFFB9C
:10881000386CF5F7A8FB162201A9F4F7DBF901A8DB
:1088200000903B6CDFF86426162107A8F2F7D1FD13
:1088300007A90020F3F7A8F900200AE000220DABF9
:10884000162404FB00F423445A54491C1629F5D37A
:10885000401C0C2801D20021F8E701240025002645
:10886000386CF5F721FB8046894617E018EA0400CA
:1088700019EA050100220023994201D1904209D052
:1088800022002B000DA8162101FB06F10844F5F784
:10889000D9FC761C6D0045EAD47564000C2E05D217
:1088A000002000218D42E1D18442DFD13000F2F777
:1088B0001BFE0320F3F733F90420F3F788F907A927
:1088C0000020F3F761F900200021894505D180459A
:1088D00003D10020F3F727F905E00020F2F733FE7B
:1088E000401CF3F720F90220F2F72DFE04001625B4
:1088F0000DA805FB04F101440120F3F745F90DA88B
:1089000005FB04F1084410F116010220F3F73CF9CD
:108910000DA805FB04F1084410F12C010320F3F726
:1089200033F90DA86C43204410F142010420F3F701
:108930002BF90820F3F700F8002804D10120F2F702
:10894000FBFF002802D0F2F790FE02E03000F2F7C1
:10895000A4FE4FB0BDE8F083F0B5B9B00400206CC0
:10896000F1F710FB5FF480000021F1F700FB206CB1
:10897000F5F7F9FA162201A9F4F72CF901A80090ED
:10898000236CDFF80825162107A8F2F722FD07A9B6
:108990000020F3F7F9F80320F3F7C1F80420F3F708
:1089A00016F900200AE000220DAB162505FB00F5A4
:1089B0002B445A54491C1629F5D3401C082801D2CF
:1089C0000021F8E7206CF5F761FA0500206CF5F757
:1089D000CAFA062801D1012700E000270124002659
:1089E0000CE0254209D03A0021000DA8162303FB14
:1089F00006F31844F5F7CEFB761C6400082E01D26E
:108A0000002CEED13000F2F76FFD002D03D10020D5
:108A1000F3F789F805E00020F2F795FD401CF3F725
:108A200082F80220F2F78FFD040016250DA805FB41
:108A300004F101440120F3F7A7F80DA805FB04F1A8
:108A4000084410F116010220F3F79EF80DA805FB6B
:108A500004F1084410F12C010320F3F795F80DA858
:108A60006C43204410F142010420F3F78DF80820F4
:108A7000F2F762FF002804D10120F2F75DFF002821
:108A800002D0F2F7F2FD02E03000F2F706FE39B054
:108A9000F0BD18B58DB00400206CF1F773FA5FF4E7
:108AA00080000021F1F763FA206CF5F75CFA1622DA
:108AB00007A9F4F78FF807A80090236CDFF8CC2300
:108AC000162101A8F2F785FC01A90020F3F75CF854
:108AD0000420F3F724F80120F3F779F80A2315228C
:108AE00007A9DFF8D003F2F7EDFE206CF5F7F7F9F0
:108AF000009007ABDFF8C023162101A8F2F769FC4C
:108B000001A90120F3F740F887A421000220F3F720
:108B10003BF821000320F3F737F821000420F3F796
:108B200033F821000520F3F72FF821000620F3F792
:108B30002BF821000720F3F727F821000820F3F78E
:108B400023F80020F2F7EFFF0820F2F7F5FE0028E7
:108B500001D0F2F78AFD0EB010BD30B5A5B004000B
:108B600002A8D6490A680260206CF1F70BFA5FF49C
:108B700080000021F1F7FBF9206CF5F7F4F91622DB
:108B800009A9F4F727F809A80090236CBF4A162119
:108B900003A8F2F71EFC03A90020F2F7F5FF03205B
:108BA000F2F7BDFF0120F3F712F80121206CF5F771
:108BB000B8F905000021206CF5F7B3F90195009094
:108BC00002ABBF4A16210FA8F2F703FC0FA9012040
:108BD000F2F7DAFF206CF5F7C6F910280DD152A490
:108BE00021000220F2F7D0FF21000320F2F7CCFF92
:108BF00021000420F2F7C8FF7DE0206CF5F754F95E
:108C000010F0000011F4807100220023994201D17C
:108C1000904218D0206C012801D103200AE0206C7A
:108C2000032801D1012005E0206C052801D107208F
:108C300000E005200090A34BA34A16210DF152003D
:108C4000F2F7C7FB06E09F4BA04A16210DF1520038
:108C5000F2F7BFFB94F84000C00702D4256C6D1EEC
:108C600001E0256C6D1C206CF5F71EF910F000007A
:108C700011F0800100220023994201D1904207D0D7
:108C80000095934B934A16211AA8F2F7A2FB05E030
:108C90008F4B914A16211AA8F2F79BFB256C0835D9
:108CA000206CF5F701F910F0000011F040010022EE
:108CB0000023994201D1904208D00095874B884A01
:108CC00016210DF17E00F2F784FB06E0834B854A06
:108CD00016210DF17E00F2F77CFB0DF1520102200E
:108CE000F2F752FF1AA90320F2F74EFF0DF17E01B1
:108CF0000420F2F749FF0CA421000620F2F744FFFC
:108D000021000720F2F740FF21000820F2F73CFF86
:108D10000020F2F708FF0820F2F70EFE002801D02D
:108D2000F2F7A3FC25B030BD0000000038B58EB0CE
:108D30000400206CF1F726F95FF480000021F1F7C0
:108D400016F9206CF5F70FF9162202A9F3F742FF86
:108D500002A80090236C4D4A162108A8F2F739FBAF
:108D600008A90020F2F710FF236C5F4A162102A821
:108D7000F2F72FFB02A90020F2F706FF206B002874
:108D800005D11622594902A8F2F7C8F90DE0206B67
:108D9000012805D11622564902A8F2F7BFF904E0CE
:108DA0001622544902A8F2F7B9F90420F2F7B7FEE7
:108DB0000420F2F70CFF0020F2F7B5FE02A9012013
:108DC000F2F7E2FE2BA529000220F2F7DDFE2900D2
:108DD0000320F2F7D9FE29000420F2F7D5FE29007E
:108DE0000520F2F7D1FE29000620F2F7CDFE29007A
:108DF0000720F2F7C9FE29000820F2F7C5FE082077
:108E0000F2F79AFD00281BD0E06B216B884214D04A
:108E1000206C012808D1216B5920F3F7DDFD0020DB
:108E20000821F1F7A4F808E0216B206CF5F7CAF8E7
:108E300000204FF48061F1F79AF8F2F716FC17E082
:108E40000120F2F779FD002802D0F2F70EFC0FE0C6
:108E5000206C012801D1012100E0022100200190B5
:108E60000120009001230022206BF2F789FC20638F
:108E70000FB030BD000000004000300028E70100C6
:108E800044E8010098EB010020F6030050E80100DF
:108E9000A0EB010060D20300A8EB010080D2030028
:108EA000B0EB010000ED0300B8EB010020ED030082
:108EB000C0EB0100E0EC0300C8EB010078F001001A
:108EC00040E6010080F4030038E701005CE801009F
:108ED000A0F4030068E80100D0EB010008E80100FD
:108EE00048E7010074E8010080E8010080E6030023
:108EF00060E40300E0F5030078B59DB00400206C49
:108F0000F1F740F85FF480000021F1F730F8206CB1
:108F1000012807D1DFF8C4339FA2162101A8F2F778
:108F200058FA09E0DFF8B4030090236CDFF8B023AF
:108F3000162101A8F2F74DFA01A90020F2F724FE4C
:108F4000DFF8A023162107A8F2F743FADFF89833D9
:108F5000DFF8982316210DF13200F2F73AFADFF824
:108F600090532B00DFF88C23162112A8F2F731FA68
:108F70002B00DFF8842316210DF15E00F2F729FAA9
:108F80000420F2F7B1FA0320F2F7C9FD0420F2F74A
:108F90001EFE0220F2F7D7FA0500162607A806FBE8
:108FA00005F101440120F2F7EFFD07A806FB05F1EA
:108FB000084410F116010220F2F7E6FD07A806FBAF
:108FC00005F1084410F12C010320F2F7DDFD07A89C
:108FD0007543284410F142010420F2F7D5FD00202A
:108FE000F2F7B1FA401CF2F79EFD206CF4F78BFF0C
:108FF00005000120F2F7A0FC002802D0F2F735FBB3
:1090000039E00820F2F798FC002831D00120F2F76F
:109010009AFAFF2D29D0002804D101218320F2F7EC
:10902000CCFA22E001280DD101218920F2F7C5FAFE
:10903000A80702D40120206301E000202063206BF8
:10904000E06312E0022808D101218A20F2F7B5FA84
:10905000C5F38200401C206307E001218B20F2F75A
:10906000ACFAC5F34210401C2063206BE06302E0C1
:109070000420F2F712FB1EB070BD38B588B00400B2
:10908000206CF0F77FFF5FF480000021F0F76FFFA6
:10909000206C012806D1914B3FA2162102A8F2F7BD
:1090A00098F907E08D480090236C8D4A162102A89C
:1090B000F2F78FF902A90020F2F766FD206B002875
:1090C00005D116228D4902A8F2F728F804E01622ED
:1090D0008B4902A8F2F722F80420F2F720FD0420C1
:1090E000F2F775FD0020F2F71EFD02A90120F2F74C
:1090F0004BFD77A529000220F2F746FD2900032049
:10910000F2F742FD29000420F2F73EFD2900052078
:10911000F2F73AFD29000620F2F736FD2900072074
:10912000F2F732FD29000820F2F72EFD206CF4F74B
:10913000EAFE05000820F2F7FFFB002816D0206B9E
:10914000E16B88420FD035F00205206B002801D179
:1091500055F002052900206CF4F7DEFE00204FF4E4
:109160008061F0F704FFF2F780FA12E00120F2F7D5
:10917000E3FB002802D0F2F778FA0AE00020019021
:1091800001200090012300220121206BF2F7F8FA60
:10919000206309B030BD00002573000070B588B0B1
:1091A00004000D00206CF0F7EDFE5FF4800000215C
:1091B000F0F7DDFE206C012806D1484B45A21621B0
:1091C00002A8F2F706F907E044480090236C444AED
:1091D000162102A8F2F7FDF802A90020F2F7D4FC4C
:1091E000236B3DA2162102A8F2F7F3F80420F2F750
:1091F00096FC0420F2F7EBFC02A90120F2F7C4FC74
:1092000033A631000220F2F7BFFC31000320F2F751
:10921000BBFC31000420F2F7B7FC31000520F2F767
:10922000B3FC31000620F2F7AFFC31000720F2F763
:10923000ABFC31000820F2F7A7FC0020F2F773FC2A
:109240000820F2F779FB00282DD0206BE16B8842D3
:1092500026D0206CF4F757FE022D0CD1216B491E4D
:109260002163216B490111F0E001216330F0E0003E
:10927000216B08430BE0216B491E2163216B8900A0
:1092800011F01C01216330F01C00216B0843010028
:10929000206CF4F741FE00204FF48061F0F767FE88
:1092A000F2F7E3F912E00120F2F746FB002802D0C2
:1092B000F2F7DBF90AE00020019000200090012382
:1092C00001220421206BF2F75BFA206308B070BD25
:1092D00000000000257300002564000008E801007C
:1092E00038E8010078EB010040D8030080EB010072
:1092F000C0D5030088EB010090EB010080E603007D
:10930000E0D9030078B59DB0040070200021F0F78B
:109310002EFE0420F2F7E8F81622DFF8FC1501A86B
:10932000F1F7FCFEDFF8F4552B00DFF8F4251621E9
:1093300007A8F2F74EF8DFF8EC35DFF8EC25162138
:109340000DF13200F2F745F8DFF8E00500902B0050
:10935000DFF8DC25162112A8F2F73BF8DFF8D43548
:10936000DFF8D42516210DF15E00F2F732F8032064
:10937000F2F7D5FB0420F2F72AFC0020F2F7E3F81D
:10938000401CF2F7D0FB01A90020F2F7FDFB022000
:10939000F2F7D9F80500162607A806FB05F10144E7
:1093A0000120F2F7F1FB07A806FB05F1084410F1D4
:1093B00016010220F2F7E8FB07A806FB05F10844B6
:1093C00010F12C010320F2F7DFFB07A875432844B6
:1093D00010F142010420F2F7D7FB0820F2F7ACFAB3
:1093E000002869D00120F2F7AEF8002816D101213B
:1093F0002720F2F7E2F84E20F3F7CFFAC00702D4A5
:109400000020206355E04E20F3F7C7FA800702D50D
:10941000012020634DE0022020634AE0012817D19B
:109420004E20F3F7BAFA10F001002063206B0028F9
:109430003FD001212820F2F7C0F84E20F3F7ADFA13
:10944000000602D40020206333E00120206330E0D6
:10945000022817D14E20F3F7A0FA10F00100206384
:10946000206B002825D001212920F2F7A6F84E20F4
:10947000F3F793FA400702D50120206319E000209A
:10948000206316E04E20F3F788FA10F00100206305
:10949000206B00280DD001212A20F2F78EF84E20F3
:1094A000F3F77BFA400602D40020206301E001209C
:1094B0002063206BE0630AE00120F2F73DFA002808
:1094C00002D0F2F7D2F802E00420F2F7E6F81EB07C
:1094D00070BD38B58EB0040070200021F0F747FD54
:1094E0001622DFF8381408A8F1F718FE206B0128BF
:1094F00006D11622DFF8441402A8F1F70FFE11E09E
:10950000206B022806D11622DFF8341402A8F1F7E6
:1095100005FE07E01622DFF82C1402A8F1F7FEFD85
:10952000002020630420F2F7FAFAF3F7E8FA0128A2
:1095300003D10120F2F74BFB02E00420F2F747FBD6
:109540000020F2F7F0FA08A90020F2F71DFB02A9AB
:109550000120F2F719FBB0A529000220F2F714FB55
:1095600029000320F2F710FB29000420F2F70CFB7E
:1095700029000520F2F708FB29000620F2F704FB7A
:1095800029000720F2F700FB29000820F2F7FCFA77
:109590000820F2F7D1F900281ED0206BE16B884239
:1095A00017D04E20F3F7F9F9010089088900206BE4
:1095B000012802D151F0030104E0206B022801D1FF
:1095C00051F001014E20F3F707FA00200821F0F7CF
:1095D000CEFCF2F74AF818E00120F2F7ADF90028C6
:1095E00002D0F2F742F810E0002001900120009034
:1095F000012300220221206BF2F7C2F82063F3F767
:109600007EFA012801D1012020630FB030BD38B5AA
:109610008EB0040070200021F0F7A9FC1622CA4980
:1096200008A8F1F77BFD206B002805D11622C4495C
:1096300002A8F1F773FD04E01622C04902A8F1F771
:109640006DFD0420F2F76BFA0420F2F7C0FA002057
:10965000F2F769FA08A90020F2F796FA02A90120A8
:10966000F2F792FA6CA529000220F2F78DFA290090
:109670000320F2F789FA29000420F2F785FA29007D
:109680000520F2F781FA29000620F2F77DFA290079
:109690000720F2F779FA29000820F2F775FA082076
:1096A000F2F74AF9002818D0206BE16B884211D0FC
:1096B0004E20F3F772F9010031F00401206B01280C
:1096C00001D151F004014E20F3F786F90020082162
:1096D000F0F74DFCF1F7C9FF12E00120F2F72CF989
:1096E000002802D0F1F7C1FF0AE00020019001201C
:1096F0000090012300220121206BF2F741F8206342
:109700000FB030BD38B58EB0040070200021F0F7E6
:109710002EFC1622834908A8F1F700FD206B0028D3
:1097200005D11622894902A8F1F7F8FC04E01622B7
:10973000874902A8F1F7F2FC0420F2F7F0F9F3F7F9
:10974000DEF9012803D10120F2F741FA02E00420FA
:10975000F2F73DFA0020F2F7E6F908A90020F2F747
:1097600013FA02A90120F2F70FFA2BA52900022013
:10977000F2F70AFA29000320F2F706FA290004207A
:10978000F2F702FA29000520F2F7FEF92900062077
:10979000F2F7FAF929000720F2F7F6F92900082074
:1097A000F2F7F2F90820F2F7C7F8002818D0206B7A
:1097B000E16B884211D04E20F3F7EFF8010031F051
:1097C0008001206B002801D051F080014E20F3F77A
:1097D00003F900200821F0F7CAFBF1F746FF18E073
:1097E0000120F2F7A9F8002802D0F1F73EFF10E0BF
:1097F0000020019001200090012300220121206B14
:10980000F1F7BEFF2063F3F77AF9012801D10020B8
:1098100020630FB030BD00000000000038B58EB0EE
:10982000040070200021F0F7A2FB1622414908A88D
:10983000F1F774FC206B002805D11622434902A8D9
:10984000F1F76CFC04E01622414902A8F1F766FC2E
:109850000420F2F764F90420F2F7B9F90020F2F7D6
:1098600062F908A90020F2F78FF902A90120F2F7A6
:109870008BF928A529000220F2F786F92900032098
:10988000F2F782F929000420F2F77EF92900052079
:10989000F2F77AF929000620F2F776F92900072075
:1098A000F2F772F929000820F2F76EF90820F2F7B2
:1098B00043F8002818D0206BE16B884211D04E206D
:1098C000F3F76BF8010031F04001206B002801D064
:1098D00051F040014E20F3F77FF800200821F0F707
:1098E00046FBF1F7C2FE12E00120F2F725F800284E
:1098F00002D0F1F7BAFE0AE00020019001200090AA
:10990000012300220121206BF1F73AFF20630FB001
:1099100030BD000000000000A0D3030040D80300C9
:1099200030EB010060D8030038EB010080E4030055
:1099300040EB010060F3030048EB0100E0D80300B6
:10994000C0D8030080E6030080F3030080D5030045
:10995000A0D5030010B59CB0040070200021F0F7E2
:1099600006FB0420F1F7C0FDDFF8F43672A21621E1
:109970006846F1F72EFD69460020F2F705F9DFF899
:10998000E436DFF8E426162106A8F1F722FDDFF819
:10999000DC36DFF8DC2616210DF12E00F1F719FD7B
:1099A000DFF8D036DFF8D026162111A8F1F711FD27
:1099B000DFF8C836DFF8C82616210DF15A00F1F796
:1099C00008FD0320F2F7ABF80420F2F700F90020BD
:1099D000F1F7B9FD401CF2F7A6F806A90120F2F74D
:1099E000D3F80DF12E010220F2F7CEF811A90320D1
:1099F000F2F7CAF80DF15A010420F2F7C5F8082071
:109A0000F1F79AFF002800F089800120F1F79BFD13
:109A1000002818D101212C20F1F7CFFD4D20F2F7BD
:109A2000BCFF10F0C0002063206B802802D1012011
:109A3000206370E0206B402802D1022020636AE09E
:109A40000020206367E001282AD101212D20F1F7B1
:109A5000B4FD4D20F2F7A1FF10F00F002063206B42
:109A6000012802D10120206355E0206B032802D198
:109A7000022020634FE0206B052802D103202063E1
:109A800049E0206B092802D10420206343E0206BC9
:109A90000F2802D1052020633DE0002020633AE03A
:109AA000022817D14D20F2F778FF10F00F00206345
:109AB000206B00282FD001212E20F1F77EFD2020E1
:109AC000F2F75CFF002802D10020206323E0012090
:109AD000206320E04D20F2F760FF10F00F002063BC
:109AE000206B002817D001212F20F1F766FD4D20B3
:109AF000F2F753FF10F030002063206B002802D1F2
:109B00000020206307E0206B102802D10120206391
:109B100001E002202063206BE0630AE00120F1F7FE
:109B20000BFF002802D0F1F7A0FD02E00420F1F7BE
:109B3000B4FD1CB010BD00002573000038B58EB018
:109B4000040070200021F0F712FA1622DFF8141535
:109B500008A8F1F7E3FA206B002806D1DFF82425E6
:109B6000162102A8F1F735FC0FE0206B012806D181
:109B7000DFF81425162102A8F1F72BFC05E0DFF829
:109B80000C25162102A8F1F724FC0420F1F7C7FFE9
:109B90000420F2F71CF80020F1F7C5FF08A9002007
:109BA000F1F7F2FF02A90120F1F7EEFFA2A52900CB
:109BB0000220F1F7E9FF29000320F1F7E5FF290072
:109BC0000420F1F7E1FF29000520F1F7DDFF29006E
:109BD0000620F1F7D9FF29000720F1F7D5FF29006A
:109BE0000820F1F7D1FF0820F1F7A6FE002822D0C7
:109BF000206BE16B88421BD0206B002804D120240D
:109C00002020F2F7C4FE0BE0206B012804D1802451
